:100000000C94A40A0C94D50A0C94D50A0C94D50A25
:100010000C94D50A0C94D50A0C94D50A0C94D50AE4
:100020000C94D50A0C94D50A0C94D50A0C94D50AD4
:100030000C94D50A0C94AA570C94D50A0C94D50AA2
:100040000C94D50A0C94D50A0C94D50A0C94D50AB4
:100050000C94D50A0C94D50A0C94D50A0C94C19929
:100060000C94D50A0C94BD4E0C94944E0C94D50A65
:100070000C94D50A0C94D50A0C94D50A0C94D50A84
:100080000C94D50A0C94D50A0C94D50A0C94D50A74
:100090000C946A4E0C94414E0C94D50A0C94D05892
:1000A0000C94D50A0C94D50A0C94D50A0C94D50A54
:1000B0000C94D50A0C94D50A0C94D50A0C94D50A44
:1000C0000C94D50A0C94D50A0C94D50A0C94174EAE
:1000D0000C94EE4D0C94D50A0C94C44D0C949B4D8D
:1000E0000C94D50A021CE91C511C4A1C1A1C0A1C3F
:1000F000E91C061CE91CE91CE91CE91CE91C610B54
:10010000CA0B5B0C980DA00D7A0F34105211F4122B
:10011000F0134F1464146814E91CAA14AE141916D1
:10012000D417EE1715197419501AD01AD71AC31B01
:100130001940B240C440CD40D640DF40F140FA40C3
:1001400029413B4144414D415641F141FA4103426D
:1001500058845B844A844E84548492845F8463848C
:1001600069846D84718477847B847F8492848584A0
:1001700089848D84084AD73B3BCE016E84BCBFFD89
:10018000C12F3D6C74319ABD56833DDA3D00C77F67
:1001900011BED9E4BB4C3E916BAAAABE0000008000
:1001A0003F07634236B79BD8A71A39685618AEBACC
:1001B000AB558C1D3CB7CC5763BD6DEDFD753EF660
:1001C000177231BF000000803F08000000BE92247B
:1001D00049123EABAAAA2ABECDCCCC4C3E000000B0
:1001E00080BEABAAAAAA3E00000000BF00000080AB
:1001F0003F0000000000084178D3BB4387D1133D86
:10020000190E3CC3BD4282AD2B3E68EC8276BED94E
:100210008FE1A93E4C80EFFFBE01C4FF7F3F00008D
:10022000000000004E414E494E495459494E46CDBA
:10023000CCCC3D0AD7233C17B7D13877CC2B32959D
:1002400095E6241FB14F0A000020410000C842007B
:10025000401C4620BCBE4CCA1B0E5AAEC59D740045
:10026000407A10F35A00A0724E18090010A5D4E885
:100270000000E87648170000E40B54020000CA9A18
:100280003B000000E1F5050000809698000000406A
:10029000420F000000A086010000001027000000AF
:1002A00000E803000000006400000000000A0000F5
:1002B0000000000100000000002C76D888DC674FA9
:1002C0000823DFC1DFAE59E1B1B796E5E3E453C6D9
:1002D0003AE651997696E8E6C28426EB898C9B62D1
:1002E000ED407C6FFCEFBC9C9F40F2BAA56FA5F47B
:1002F00090055A2AF75C936B6CF9676DC11BFCE0A3
:10030000E40D47FEF520E6B500D0ED902E030094F5
:100310003577050080841E080000204E0A0000008A
:10032000C80C333333330F986E12831141EF8D2194
:1003300014893BE65516CFFEE6DB18D1844B381BFB
:10034000F77C1D901DA4BBE424203284725E2281C0
:1003500000C9F124ECA1E53D274D6F74696F6E0073
:10036000555620496E742E00555620496E74656EA0
:1003700073697479004F3220436F6E6300434F32CC
:1003800020436F6E630053656E736F7220657272E7
:100390006F722100234E6F2073656E736F722100A0
:1003A000434F3220436F6E63004D65617375726910
:1003B0006E6700234E6F2073656E736F7220666FD9
:1003C0007220504D21004E6F2073656E736F722145
:1003D00000206E672F4C00504D313A322E353A31A5
:1003E00030004D6561737572696E672E2E00234E65
:1003F0006F2054422073656E736F723F00234E6FFF
:100400002073656E736F722100536F756E64204C9C
:100410006576656C004D6561737572696E672E2E29
:1004200000234E6F2073656E736F722100536F75DA
:100430006E64204C6576656C00234E6F2073656E8C
:10044000736F7220666F722074656D70202620684D
:10045000756D696469747921004E6F2053656E7300
:100460006F72210020666F722074656D70202620E7
:1004700068756D696469747921002353656E736FC3
:1004800072204572726F72200053656E736F722016
:100490004572726F7221002357726F6E6720736509
:1004A0006E736F7220666F722074656D70202620E7
:1004B00068756D6964697479210057726F6E672081
:1004C00053656E736F72210054656D702048756DB1
:1004D0006964697479004C6967687420496E746551
:1004E0006E7369747900466C616D652049520048ED
:1004F0002D6669656C6400536561726368204469A8
:1005000072656374696F6E00234E6F2070482073AC
:10051000656E736F72210070482076616C7565009E
:1005200023496E76616C6964206B65792100204DEA
:10053000756C746973656E736F7273004D756C744E
:100540006973656E736F72730044697361626C6581
:1005500000456E61626C65005265626F6F74696E12
:10056000672E2E2E002344413A2D3233002372652C
:10057000706C6965733D002353657474696E6773AD
:10058000206F6620616C6C2073656E736F72733AB6
:10059000002353697A65206F66206865616465721F
:1005A000202B20616C6C2073656E736F72733A2020
:1005B000002353697A65206F6620686561646572FF
:1005C0003A20002320616E64207265616479207492
:1005D0006F207573652100206D6F62696C65206CFA
:1005E0006F6767657220737461727465642000437D
:1005F000616C6962726174696F6E205072657373A9
:100600007572653D00536561206C6576656C2050A0
:100610002863616C63293D00234572726F723A70E2
:100620007265737375726520424D503038352C20D9
:10063000636865636B20776972696E672100495250
:100640002054656D702073656E736F7220666F75D0
:100650006E6400504D322E352073656E736F7220BC
:100660006C696B656C7920666F756E6400206D6FC8
:1006700062696C65206C6F67676572207374617264
:10068000746564202E2E2E2000576946692049503B
:100690003A002357694669204950206164647265B5
:1006A00073733A2000456455484B205345534C6FB3
:1006B000676765720053656E736F7220736C6F7439
:1006C00020616E6420747970653A0057656C636FC1
:1006D0006D6520746F20456455484B0023456E645A
:1006E000206F66204D756C746973656E736F722030
:1006F0004379636C6523002354696D6520647572CA
:100700006174696F6E3D002354696D6520696E7474
:10071000657276616C3D00576946692049503A0020
:10072000234D5320456E61626C656400234D532058
:1007300044697361626C6564002352657374207050
:100740006172616D657465727320746F2064656693
:1007500061756C742076616C756573004C6F6767AA
:100760006572204E616D653A200067657453656C53
:10077000665465737442697428293A200069734984
:100780006E74657272757074456E61626C65642812
:1007900031293A2000676574496E7465727275700C
:1007A000744D617070696E672831293A2000676561
:1007B00074496E74657272757074536F7572636587
:1007C0002831293A2000676574496E746572727524
:1007D0007074536F7572636528293A2000676574D9
:1007E0005261746528293A20332E31343135393F2E
:1007F00000616363656C2E69734C6F77506F77652A
:100800007228293A2000616363656C2E6973417315
:100810006C65657028293A2000616363656C2E69F8
:1008200073546170536F757263654F6E5A28293A1D
:100830002000616363656C2E6973546170536F753A
:100840007263654F6E5928293A2000616363656CB5
:100850002E6973546170536F757263654F6E5828BB
:10086000293A2000616363656C2E69734163746982
:1008700076697479536F757263654F6E5A28293A99
:100880002000616363656C2E6973416374697669E6
:100890007479536F757263654F6E5928293A200039
:1008A00069734163746976697479536F75726365AE
:1008B0004F6E5828293A200069735461704465745A
:1008C000656374696F6E4F6E5A28293B2066616CB0
:1008D00073653F2000697354617044657465637487
:1008E000696F6E4F6E5A28293B20747275653F20E0
:1008F000006973546170446574656374696F6E4F09
:100900006E5928293B2066616C73653F200069732E
:10091000546170446574656374696F6E4F6E5928D5
:10092000293B20747275653F2000697354617044DF
:100930006574656374696F6E4F6E5828293B206635
:10094000616C73653F200069735461704465746520
:100950006374696F6E4F6E5828293B2074727565F9
:100960003F200067657453757070726573734269D8
:100970007428293B2066616C73653F2000676574AD
:10098000537570707265737342697428293B2074C3
:100990007275653F20006973416374697669747983
:1009A000416328293A20006973496E61637469764E
:1009B0006974795A456E61626C656428293A200031
:1009C0006973496E616374697669747959456E61BA
:1009D000626C656428293A20006973496E6163740A
:1009E000697669747958456E61626C656428293A44
:1009F0002000697341637469766974795A456E6140
:100A0000626C656428293A200069734163746976D1
:100A100069747959456E61626C656428293A2000D1
:100A20006973416374697669747958456E61626C63
:100A3000656428293A2000676574467265654661D9
:100A40006C6C4475726174696F6E28293A20006776
:100A500065744672656546616C6C5468726573684E
:100A60006F6C6428293A200067657454696D654984
:100A70006E616374697669747928293A2000676524
:100A800074496E61637469766974795468726573C8
:100A9000686F6C6428292000676574416374697607
:100AA0006974795468726573686F6C6428292000D2
:100AB000676574446F75626C6554617057696E64E4
:100AC0006F7728292000676574446F75626C6554E0
:100AD00061704C6174656E637928293A20006765FE
:100AE000745461704475726174696F6E28293A207C
:100AF00000676574417869734F666673657428266C
:100B0000782C2026792C20267A293A2000676574D3
:100B10005461705468726573686F6C6428293A2058
:100B20000058595A2047733A200058595A20434FC9
:100B3000554E54533A2000736574206761696E7393
:100B40005B5D3A006761696E735F6F7269675B5DD9
:100B50003A00696E7075742044535463616C696225
:100B6000726174653A0020766F6C746167653D0050
:100B70002354757262696469747920557070657266
:100B8000204C696D69743A200020766F6C7461673F
:100B9000653D0023547572626964697479204C6FF5
:100BA000776572204C696D69743A20002354757220
:100BB000626964697479204C6F776572204C696D45
:100BC00069742056696E663A20004D617820726122
:100BD0006E67653D0023566F6C74616765207365B1
:100BE0006E736F723A00342D32306D4100414353C1
:100BF000373132204D61783D004143533731322047
:100C00004D61783D3541002343757272656E7420E5
:100C100073656E736F723A00234453205468657293
:100C20006D6F6D657465722063616C696272617469
:100C3000656420666F72202300234E6F206E656509
:100C40006420746F2063616C6962726174652063F3
:100C5000757272656E742073656E736F72210023F6
:100C60004143533731322063757272656E7420735D
:100C7000656E736F72206F666673657420563D00F3
:100C8000235556207A65726F20766F6C74616765A4
:100C9000203D00234F3220766F6C253D00234F32DC
:100CA0002063616C6962726174696F6E3A2000231F
:100CB000566F6C746167652870483D3130293A0081
:100CC00023566F6C746167652870483D34293A007B
:100CD000232D2D2D2D2D2D2D2D2D2D2D2D2D2D2D4E
:100CE0002D2D2D2D2D2D2D2D2D2D2D2D2D2D2D2D34
:100CF0002D2D2D2D2D00235265736F6C7574696F2A
:100D00006E3A20202000234D696E2056616C756577
:100D10003A2020202000234D61782056616C7565B3
:100D20003A202020200023556E69717565204944C2
:100D30003A2020202000234472697665722056658F
:100D4000723A202020002353656E736F723A202080
:100D5000202020202000232D2D2D2D204D61676E79
:100D6000657469632053656E736F72202D2D2D2D70
:100D70002D2D2D2D2D2D2D2D2D2D2D2D2D2D2D2DA3
:100D800000482D6669656C643A20280020202020E8
:100D90002020202020202020202020002020202073
:100DA000202020202020202020202000233A5368CB
:100DB0006F772F48696465204C4344002A3A546891
:100DC00069732048656C700044233A43616C696222
:100DD000726174696F6E00442A3A53657474696E67
:100DE00067730044423A5265736574204C6F6767BD
:100DF00065720044433A436C656172204C43440081
:100E000044443A4D756C746953656E736F72730028
:100E100044393A43757272656E7400566F6C746132
:100E200067652B43757272656E740044383A456C81
:100E30006563747269630044373A4D6F74696F6E0D
:100E40000044363A44532054656D700044353A5599
:100E50005620496E74656E736974790044343A4F54
:100E60003220636F6E632E0044333A434F32206367
:100E70006F6E632E0044323A504D28313A322E358F
:100E80003A3130290044323A504D28313A322E3529
:100E90003A3130292A0044313A54757262696469E2
:100EA00074790044303A566F6C7461676500393A62
:100EB0006F7220334420616363656C2E00393A49B8
:100EC0006E636C2E20616E672E00383A7048207673
:100ED000616C756500373A49522054656D70003772
:100EE0003A49522054656D702A00363A4D61676E5A
:100EF00065746963206669656C6400353A4761739F
:100F0000204C6576656C00343A495220466C616D20
:100F10006500333A4C6967687420496E742E00325C
:100F20003A616E642048656967687400323A5465B6
:100F30006D7020507265737375726500313A546537
:100F40006D702048756D696469747900303A536F2B
:100F5000756E64204C6576656C00303A536F756E23
:100F600064204C6576656C2A0054696D65206C615F
:100F70007073653A00576946692049503A00005E2F
:100F8000BCE2613FDD83C29C7E20A3FD1F41009D2A
:100F900023BE46DB65F88C11AF32CA57E974697419
:100FA00065726174696F6E3D0073656E736F722355
:100FB0003D0043757272656E74207374617475734D
:100FC0003A206379636C653D006E6379636C653DBF
:100FD000006E73656E736F72733D006D61786E7332
:100FE000656E736F72733D00656E61626C65643D22
:100FF00000234D756C746973656E736F7273206D29
:101000006561737572656D656E742073657474695E
:101010006E67733A0046696E64696E672057694669
:1010200069204950007365703D006976616C3D0030
:101030006E697465723D00230043616C2E20466129
:10104000696C65640043616C2E20446F6E65004ED0
:101050006F206E6565642100496E76616C6964205D
:101060005028506129005365614C6576656C2050AD
:10107000285061293A0043616C696272617465208D
:1010800050004453542054656D702073656E736F27
:10109000720043757272656E742073656E736F7241
:1010A000004F322073656E736F7200555620736562
:1010B0006E736F720043616C6962726174650046A1
:1010C00061696C65640054422063616C2E20646F1A
:1010D0006E65005570706572204C696D69743A3E9A
:1010E000004C6F776572204C696D69743A3E00540C
:1010F0007572626964697479004661696C6564003F
:1011000070482063616C2E20646F6E6500704831FA
:101110003020507265737320420070483420507242
:1011200065737320410043616C696272617465008C
:10113000416E676C65732F003E6128782C792C7A9C
:10114000292F673A004E6F2073656E736F7221000E
:1011500049522054656D7065726174757265004DF9
:101160006561737572696E672E2E004E6F20736510
:101170006E736F723F0049522054656D70657261E5
:1011800074757265004D6561737572696E672E2E98
:10119000004F6666206169722D636F6E642100499D
:1011A00074277320746F6F20636F6F6C2100546518
:1011B0006D702069732066696E6521004973206136
:1011C00069722D636F6E64206F6E3F0049742773E0
:1011D00020717569746520686F74210049742773E4
:1011E000207665727920686F742120004F66662032
:1011F0006169722D636F6E642100497427732074D6
:101200006F6F20636F6F6C210054656D7020697380
:101210002066696E6521004973206169722D636FD4
:101220006E64206F6E3F0049742773207175697476
:101230006520686F74210049742773207665727980
:1012400020686F74210054656D702048756D696465
:10125000697479004E6F2053656E736F7221004E72
:101260006F20445320546865726D6F6D65746572AC
:101270002100445320546865726D2E004D6F7469CF
:101280006F6E00556E6B6E6F776E00496E6475738E
:10129000747269616C20342D32306D4100414353CA
:1012A000373132204D61783D3541002343757272EC
:1012B000656E742073656E736F723A0000002100D2
:1012C000240027002A002D00300033000101000017
:1012D000040107010A0100002200250028002B005C
:1012E0002E003100340002010000050108010B014D
:1012F000000020002300260029002C002F003200CF
:1013000000010000030106010901050505050705A7
:1013100008080808020202020A0A08080404040471
:10132000010101010101010103030303030303039D
:10133000040707070C0C0C0C0C0C0C0C020202022C
:1013400006060606060606060B0B0B0B0B0B0B0B15
:1013500001021020200808102040102040800201C7
:1013600002010804020101020408102040808040AC
:1013700020100804020180040201804020100804AB
:101380000201080402010102040810204080010249
:1013900004081020408000000A0B02090C0D0E0802
:1013A000070304010000000000000000000000002E
:1013B000000000000000000000000000000000002D
:1013C00000001211100000000000000000000000EA
:1013D000000000000000000000000000496E76617F
:1013E0006C6964206B65792100202020202020205A
:1013F000202020202020202020002020202020200D
:1014000020202020202020202020002020202020FC
:1014100020202020202020202020200020202020EC
:10142000202020202020202020202020004E455455
:101430003D426C7565746F6F7468204C45004E4575
:10144000543D426C7565746F6F7468004E45543D31
:10145000576946690053657474696E67204661690F
:101460006C65640053657474696E6720446F6E65C3
:10147000004368616E6765204E6574776F726B3EDE
:1014800000547970653A0042542F57694669204EDE
:101490006574776F726B004368616E676520536592
:1014A0006E736F723E0043757272656E7420536581
:1014B0006E736F72004F7468657200496E642E20FF
:1014C000342D32306D4100414353373132203C33AB
:1014D000304100414353373132203C3230410041EA
:1014E0004353373132203C3541003E4D6178205620
:1014F0006F6C743A3E004368616E676520766F6C6E
:10150000746167653E00547970652000566F6C7495
:101510006167652053656E736F72004368616E6723
:1015200065207479706520746F0053656E736F72F7
:101530003D4448540054656D702048756D69646978
:10154000747900003FA70FA711241FBECFEFD1E28F
:10155000DEBFCDBF00E00CBF1BE0A0E0B2E0E8EBD7
:10156000FCE601E00BBF02C007900D92AC3EB10754
:10157000D9F723E1ACEEBBE001C01D92A23AB2075D
:10158000E1F71AE0C3EADAE000E006C021970109BA
:10159000802FFE010E9496B3C23AD10780E008076F
:1015A000A9F70E94509A0C944BB60C9400002F920D
:1015B0003F924F925F926F927F928F929F92AF92E3
:1015C000BF92CF92DF92EF92FF920F931F93CF9330
:1015D000DF93CDB7DEB7C554D1090FB6F894DEBF9F
:1015E0000FBECDBF8C01E0900B0CF0900C0C8091E5
:1015F0009A13882349F06DE675E082E19FE00E942E
:10160000CF4CC8010E948651680125E0C20ED11C52
:1016100035E0C316D10420F180910B0C90910C0C95
:101620000817190729F10E94E93E0E947B760C3EBB
:101630004FEF140724F010930C0C00930B0CB8011F
:10164000CE0101960E948950BE016F5F7F4F8FE2ED
:1016500092E10E941C4BCE0101960E94FF4B08C0F4
:101660000E3F5FEF150721F40E948B760C94DD1D71
:101670006EEB79E083E292E10E94D54BF5E0CF1664
:10168000D10490F069ED7BE0CE0101960E94634C9D
:101690004AE050E06FEF7FEFCE0101960E94649028
:1016A000CE0101960E94FF4BF8017C96E632F105CF
:1016B00010F00C94E91C8827EE58FF4F8F4F0C94C4
:1016C00096B30E94E93E89E390E00E94447120E0D5
:1016D00030E04AE754E40E941DAFAB01BC0121E0B9
:1016E000CE0101960E94044C60E178E0CE01809624
:1016F0000E94634CBE016F5F7F4FCE0180960E94B7
:101700007F4B61EC75E00E94684BBC0183E292E183
:101710000E94EA4BCE0180960E94FF4BCE010196BB
:101720000E94FF4B65EC75E08DE192E10E94D54B84
:101730006DE172E1CE0101960E945B4C4AE050E0FF
:1017400068E070E0CE0101960E94BF8FCE01019645
:101750000E94FF4B63E272E1CE0101960E945B4C56
:101760004AE050E06FEF7FEFCE0101960E94778D47
:10177000CE0101960E94FF4B6DE172E183E292E19E
:101780000E94164B8091470C882311F40C941B1D6A
:101790000C946917E090B902F090BA020E94E93EF9
:1017A00089E390E00E94447120E030E04AE754E48D
:1017B0000E941DAF0E94A7B1CE0101960E948950E0
:1017C00060E178E0CE0180960E94634CBE016F5FBD
:1017D0007F4FCE0180960E947F4B61EC75E00E94A6
:1017E000684BBC0183E292E10E94EA4BCE018096F5
:1017F0000E94FF4BCE0101960E94FF4B8091271261
:1018000090912812099718F423E0D22E02C092E09A
:10181000D92E8091BA1083302CF5C7010E94E4784C
:101820007C016091BB107091BC10072E000C880BDE
:10183000990B0E94BEAE4B015C01B701FF0C880BF7
:10184000990B0E94BEAE9B01AC01C501B4010E9480
:101850001DAF20E030EC4FE754E40E940EB1AB0125
:10186000BC0103C040E050E0BA012D2DCE0101962D
:101870000E94044C6AEF75E0CE0180960E94634C92
:10188000BE016F5F7F4FCE0180960E947F4B6DEC53
:1018900075E00E94684BBC0183E292E10E94164B06
:1018A000CE0180960E94FF4BCE0101960E94FF4B15
:1018B00060ED75E039CF8091470C882309F42CC185
:1018C00088ED9DE00E94118E61E0809102020E94ED
:1018D000A98560E0809100020E94A9850E949E97E0
:1018E0000E94FF5B0E941C5CAB01BC0123E0CE01A7
:1018F00080960E94044CBE01605E7F4FCE0101962F
:101900000E945B4C67EF75E0CE0101960E94684B28
:10191000BC018DE192E10E94EA4BCE0101960E944A
:10192000FF4BCE0180960E94FF4B6AEF79E0CE011B
:1019300001960E94634C6DE172E1CE0101960E9416
:101940007F4BBC0183E292E10E94EA4BCE010196FB
:101950000E94FF4B0E941C5C6B017C010E940A8666
:101960004B015C016EE170E080E090E00E942F8608
:101970000E941C5C2B013C010E940A869B01AC0169
:10198000281939094A095B0949015A0131ED8316C1
:1019900037E09306A104B1040CF441C0A7019601FD
:1019A000C301B2010E9447B06B017C0120E030E02E
:1019B000A9010E94FDB118165CF426EA3BE944EC4B
:1019C0005BE3C701B6010E94B8AE87FF0BC027C01A
:1019D00026EA3BE944EC5BEBC701B6010E94FDB18E
:1019E0001816ECF0C501B40128EE33E040E050E0F9
:1019F0000E94EAAFCA01B9010E94BEAE4B015C0170
:101A000020E030E04AE754E4C701B6010E941DAF70
:101A1000A50194010E940EB1AB01BC0103C040E0DE
:101A200050E0BA0122E0CE0180960E94044CBE0133
:101A3000605E7F4FCE0101960E945B4C69ED75E0C0
:101A4000CE0101960E94684BBC0187E192E10E94A1
:101A5000EA4BCE0101960E94FF4BCE0180960E9478
:101A6000FF4B6DED75E0CE0101960E94634C67E17E
:101A700072E1CE0101960E947F4BBC0183E292E1AC
:101A80000E94164BCE0101960E94FF4B69ED7BE050
:101A9000CE0101960E94634C67E172E1CE0101968E
:101AA0000E947F4BBC018DE192E10E94164BCE015A
:101AB00001960E94FF4B69E573E0CE0101960E94FA
:101AC000534C4AE050E060E070E0CE0101960E9485
:101AD000BF8FCE0101960E94FF4B6DE172E1CE01F6
:101AE00001960E945B4C45E050E06FEF7FEFCE0126
:101AF00001960E94778DCE0101960E94FF4B61EE08
:101B000075E083E292E10E94084B60E0809102025E
:101B10000E94A9850C941B1D60915502709156027C
:101B200080915702909158020E94047A0C941B1DD8
:101B300080915B0290915C020E94077C0C941B1DBB
:101B400040915D0226964FAF269760E0842F0E9459
:101B5000A9858091470C811109C0809118118111CC
:101B60000EC08FE090E0A0E0B0E00DC023E030E0D8
:101B700040E050E02CAF3DAF4EAF5FAF08C083E018
:101B800090E0A0E0B0E08CAF9DAFAEAFBFAF68E635
:101B900073E083E292E10E94904B63E272E1CE0136
:101BA00001960E945B4C4AE050E06FEF7FEFCE0160
:101BB00001960E94BF8FCE0101960E94FF4B219695
:101BC0001FAE219725961FAE2597212C312CC12CB5
:101BD000D12C760182E3682E712C812C912C54013A
:101BE00026968FAD26970E94E585092E000CAA0B3C
:101BF000BB0B880E991EAA1EBB1E65E070E080E03C
:101C000090E00E942F8691E0691A710849F7409090
:101C10002102509022026090230270902402C5019C
:101C2000B4010E94BEAE20E030E040EA50E40E94E1
:101C30001DAF20E030E040E85AE30E941DAF20E0F5
:101C400030E048E452E40E940EB1A30192010E94E8
:101C500047B020E030E040E751E40E941DAF4B0167
:101C60005C01A30192016AE979E989E390E40E94A9
:101C700047B09B01AC01C501B4010E940EB120E048
:101C800030E0A9010E9448B020E030E040E251E499
:101C90000E941DAF4B015C0121962FAD2197259627
:101CA0003FAD2597A1010E94FDB118163CF4219685
:101CB0008FAE219725969FAE2597150120E030E045
:101CC000A901B401C5010E94B8AE87FF04C0812CF0
:101CD000912CA12CB12C22E0A401B501CE0180965B
:101CE0000E94044CBE01605E7F4FCE0101960E94AF
:101CF0005B4C64EF75E0CE0101960E94684BBC011D
:101D00008DE192E10E94EA4BCE0101960E94FF4BC9
:101D1000CE0180960E94FF4B6DE172E1CE010196EB
:101D20000E945B4C4AE050E060E070E0CE0101961A
:101D30000E94778DCE0101960E94FF4B0E948B87F7
:101D40008090921390909313A0909413B090951359
:101D5000A4E68A0E911CA11CB11C86169706A80643
:101D6000B90610F40C943C1D0E948B870E94BCAEF7
:101D70004B015C01609192137091931380919413C5
:101D8000909195130E94BEAE20E030E048EC51E403
:101D90000E9448B09B01AC01C501B4010E94B8AEDD
:101DA00087FF02C00C943C1D6CE370E080E090E083
:101DB0000E942F86BFEFCB1ADB0AEB0AFB0A2CAD81
:101DC0003DAD4EAD5FAD2C153D054E055F050CF0EC
:101DD00001CF64E670E080E090E00E942F860E94D0
:101DE000E93E64E670E080E090E00E942F8660E6C5
:101DF00073E08DE192E10E94904B6DE172E1CE01C2
:101E000001960E945B4C44E150E060E070E0CE013E
:101E100001960E94BF8FCE0101960E94FF4B22E0E7
:101E200021964FAD219725965FAD2597B101CE0143
:101E300080960E94044CBE01605E7F4FCE010196E9
:101E40000E945B4C64EF75E0CE0101960E94684BE6
:101E5000BC018DE192E10E94EA4BCE0101960E9405
:101E6000FF4BCE0180960E94FF4B6DE172E1CE01E7
:101E700001960E945B4C42E350E06FEF7FEFCE0192
:101E800001960E94778DCE0101960E94FF4B64E17E
:101E900070E080E090E00E942F860E940D3F6EE18E
:101EA00070E080E090E00E942F866EE170E080E0BC
:101EB00090E00E942F8669EF75E0CE0101960E94A6
:101EC000634C6DE172E1CE0101960E947F4B6DEF94
:101ED00075E00E94684B63E272E10E947F4BBC0197
:101EE00083E292E10E94EA4BCE0101960E94FF4BF1
:101EF0000C941B1D80915F029091600299270E94B3
:101F0000E478BC01990F880B990B0E94BEAE2DE0BE
:101F100038E643E55BE30E941DAF6B017C01209135
:101F200083023091840240918502509186020E9482
:101F3000B8AE18164CF060916B0270916C028091F3
:101F40006D0290916E021BC0209197023091980211
:101F50004091990250919A02C701B6010E94FDB1C9
:101F600087FF05C0C701B6010E94106D08C06091CF
:101F70007F0270918002809181029091820220E024
:101F800030E048EC52E40E941DAF20E030E048EA27
:101F900051E40E941DAF209125023091260240910C
:101FA0002702509128020E940EB16B017C0165E767
:101FB00073E08DE192E10E94904B6DE172E1CE0100
:101FC00001960E945B4C42E350E060E070E0CE017D
:101FD00001960E94BF8FCE0101960E94FF4B22E026
:101FE000B701A601CE0101960E94044C67E076E09D
:101FF000CE0180960E94634CBE016F5F7F4FCE0181
:1020000080960E947F4B61E076E00E94684BBC01A5
:1020100083E292E10E94EA4BCE0180960E94FF4B40
:10202000CE0101960E94FF4B63E272E1CE01019660
:102030000E945B4C42E350E06FEF7FEFCE010196D0
:102040000E94778DCE0101960E94FF4B8091470C34
:10205000882311F40C941B1D60E273E080E090E093
:102060000E942F860C941B1D0E94E93E69EA73E0D2
:1020700083E292E10E94904B63E272E1CE0101960D
:102080000E945B4C4AE050E060E070E0CE010196B7
:102090000E94BF8FCE0101960E94FF4B60EA73E061
:1020A0008DE192E10E94904B6DE172E1CE010196CB
:1020B0000E945B4C44E150E06FEF7FEFCE01019650
:1020C0000E94778DCE0101960E94FF4B8091F00B0C
:1020D0009091F10B8230910549F40E94678681113D
:1020E0001AC01092F10B1092F00B15C0892BC9F495
:1020F0000E946786882339F082E090E09093F10B8C
:102100008093F00B08C00E9467868111F5CF0E9472
:1021100067868111F1CF8091F00B9091F10B0297BE
:1021200041F164E973E083E292E10E94904B63E243
:1021300072E1CE0101960E945B4C4AE050E060E003
:1021400070E0CE0101960E94BF8FCE0101960E94E1
:10215000FF4B63E272E1CE0101960E945B4C69ED98
:102160007BE0CE0101960E94684B6DE172E10C9418
:10217000431A8AE090E00E94B7766B017C0120E070
:1021800030E0A9010E94B8AE181634F08AE090E061
:102190000E94B7766B017C01BBE0AB2EB12C20E036
:1021A00030E042ED53E4C701B6010E94B8AE181604
:1021B0008CF031E0A31AB10869F068EC70E080E0BF
:1021C00090E00E942F8683E090E00E94B7766B013A
:1021D0007C01E5CF20E030E0A901C701B6010E94F3
:1021E000B8AE18163CF066E873E083E292E10E9414
:1021F000904B31C020E030E048EC52E4C701B6011A
:102200000E94B8AE87FF02C021E001C020E0B70104
:10221000A601CE0101960E94044C66E076E0CE0154
:1022200080960E94634CBE016F5F7F4FCE01809607
:102230000E947F4B6BE076E00E94684BBC0183E21A
:1022400092E10E94EA4BCE0180960E94FF4BCE01A4
:1022500001960E94FF4B63E272E1CE0101960E945B
:102260005B4C42E350E06FEF7FEFCE0101960E949E
:10227000778DCE0101960E94FF4B6DE773E08DE1F3
:1022800092E10E94904B6DE172E1CE0101960E94B5
:102290005B4C42E350E060E070E0CE0101960E94AA
:1022A000BF8FD0CE0E948B872B013C0188ED9DE033
:1022B0000E94118E64E670E080E090E00E942F861C
:1022C00040E855E260E070E088ED9DE00E94EF6D2F
:1022D00064E670E080E090E00E942F8662EE73E09A
:1022E0008DE192E10E94904B6DE172E1CE01019689
:1022F0000E945B4C42E350E06FEF7FEFCE0101960E
:102300000E94BF8FCE0101960E94FF4B67ED73E0E4
:102310008DE192E10E94904B6DE172E1CE01019658
:102320000E945B4C42E350E06FEF7FEFCE010196DD
:102330000E94778DCE0101960E94FF4B8091110C77
:102340009091120C8D7F1CAEA12CB12CC12CD12CE4
:10235000E12CF12C019709F46FC0AE01405E5F4F94
:1023600059AF48AFCE014E969BAF8AAF0E948B8784
:10237000DC01CB0184199509A609B709883B9B406C
:10238000A105B10508F058C088ED9DE00E94B9474D
:10239000892B09F44AC02CED35E040E050E0209351
:1023A000DC0D3093DD0D4093DE0D5093DF0D0E9468
:1023B000BB6D97FD06C082349105C9F780E090E0BF
:1023C00002C08FEF9FEF892B81F5AE014F5F5F4F0A
:1023D0001A014A010E94BB6D97FF06C089818D34A6
:1023E00021F520E030E009C0D4018D934D01E8AD26
:1023F000F9ADEA17FB0771F7F1CFD1018D911D01FE
:10240000280F311DEAADFBADAE17BF07B1F72E5B4C
:102410003F4F8E8D90E0982F88274F8D840F911D10
:102420002817390711F40C94401D62E370E080E036
:1024300090E00E942F869ACF0E948B87DC01CB010F
:1024400084199509A609B709883B9B40A105B105E8
:1024500018F42CAD2111BDC00E94E93E6DE172E17E
:10246000CE0180960E945B4C42E350E066E070E053
:10247000CE0180960E94BF8FCE0180960E94FF4BB6
:102480003CAD332311F40C94591D82E090E09093FD
:10249000120C8093110CB501CE0180960E948950D8
:1024A000B601CE0186960E948950B701CE01C29630
:1024B0000E948950BE016E5C7F4FCE018C960E94B7
:1024C0005B4C66E177E0CE018C960E94684BBE01C2
:1024D0006A5D7F4F0E947F4B66E177E00E94684B08
:1024E000BE01605E7F4F0E947F4BBC0183E292E1A0
:1024F0000E94EA4BCE018C960E94FF4BCE01C29601
:102500000E94FF4BCE0186960E94FF4BCE01809623
:102510000E94FF4B63E272E1CE0180960E945B4C09
:102520004AE050E06FEF7FEFCE0180960E94778DFA
:10253000CE0180960E94FF4B61ED73E084E293E14F
:102540000E94CF4CB501CE0180960E948950B60101
:10255000CE0186960E948950B701CE018C960E94CA
:1025600089506FE076E0CE01C2960E94634CBE01B6
:10257000645D7F4FCE01C2960E947F4B69ED7BE088
:102580000E94684BBE016A5D7F4F0E947F4B69EDE0
:102590007BE00E94684BBE01605E7F4F0E947F4BD4
:1025A0006FE176E00E94684BBC0183E292E10E94F9
:1025B000EA4BCE01C2960E94FF4BCE018C960E9440
:1025C000FF4BCE0186960E94FF4BCE0180960E9463
:1025D000FF4B62E370E080E090E00E942F8688ED80
:1025E0009DE00E94118E1BC6E0905902F0905A02A5
:1025F00065E276E08DE192E10E94D54B0E94E93ED2
:102600006DE172E1CE0101960E945B4C4AE050E020
:102610006FEF7FEFCE0101960E94BF8FCE01019632
:102620000E94FF4BC7010E94DD7924966CAF7DAFFD
:102630008EAF9FAF249780902F0290903002A09091
:102640003102B0903202A501940160912B02709189
:102650002C0280912D0290912E020E9447B02B01F6
:102660003C0120E030E0A9010E94B8AE882309F4C3
:1026700053C0C0903702D0903802E0903902F090F9
:102680003A0220E030E0A901C701B6010E94B8AECD
:1026900018160CF041C08091330290913402A09141
:1026A0003502B09136028CAF9DAFAEAFBFAF9C018B
:1026B000AD01C701B6010E94B8AE882369F1A70138
:1026C00096016CAD7DAD8EAD9FAD0E940EB10E94A6
:1026D00043B26CAF7DAF8EAF9FAFA501940124963E
:1026E0006CAD7DAD8EAD9FAD24970E9447B0A30128
:1026F00092010E940EB12CAD3DAD4EAD5FAD0E947A
:102700001DAF0E947BB19B01AC01C701B6010E94C5
:102710001DAF6B017C0103C0C12CD12C76016DE192
:1027200072E1CE0101960E945B4C4AE050E060E00D
:1027300070E0CE0101960E94BF8FCE0101960E94EB
:10274000FF4B20E030E64AEE56E4C701B6010E9496
:10275000FDB118163CF46EEE73E083E292E10E9444
:10276000904B25C021E0B701A601CE0180960E94C2
:10277000044C6FE276E0CE0101960E94634CBE01EC
:10278000605E7F4FCE0101960E947F4B63E376E04F
:102790000E94684BBC0183E292E10E94EA4BCE01A9
:1027A00001960E94FF4BCE0180960E94FF4B63E290
:1027B00072E1CE0101960E945B4C4AE050E06FEF5F
:1027C0007FEFCE0101960E94778DCE0101960E9487
:1027D000FF4B64E670E080E090E00E942F8636CCEC
:1027E000E090B902F090BA020E94E93E65E070E024
:1027F00080E090E00E942F868091BA1083302CF503
:10280000C7010E94E4787C016091BB107091BC10FC
:10281000072E000C880B990B0E94BEAE4B015C0189
:10282000B701FF0C880B990B0E94BEAE9B01AC0157
:10283000C501B4010E941DAF20E030EC4FE754E425
:102840000E940EB1AB01BC0103C040E050E0BA01F0
:1028500023E0CE0101960E94044C6AEF75E0CE01A0
:1028600080960E94634CBE016F5F7F4FCE018096C1
:102870000E947F4B6DEC75E00E94684BBC0183E2C7
:1028800092E10E94EA4BCE0180960E94FF4BCE015E
:1028900001960E94FF4B67E376E00C94940B9091B5
:1028A0000A0C81E0892780930A0C8091470C8823C9
:1028B00031F063E272E18BE39DE00E94E66968EC2F
:1028C00070E080E090E0CCCB1092470C0C941B1D84
:1028D00081E08093470C8093261180911D118823FD
:1028E00049F16FEE77E08FE292E10E94D54B86EEE0
:1028F0009FEF90930C0C80930B0C20912011309142
:10290000211180912211909123118217930724F0B5
:10291000109223111092221110921411109215117D
:1029200010921611109217116CE271E080E090E0A5
:102930000E942F866FE272E185E392E10E94EA4BEA
:1029400080910B0C90910C0C9093420C8093410C55
:102950000C941B1D0E94403F0C941B1D85E79EE0BC
:102960000E94118E40E052EC61E070E085E79EE04D
:102970000E94EF6D8CED95E0A0E0B0E08093790EC1
:1029800090937A0EA0937B0EB0937C0E64E670E079
:1029900080E090E00E942F868091F00B9091F10BE7
:1029A000019759F483E090E00E944079811140C082
:1029B0001092F10B1092F00B1AC081E090E00E948F
:1029C0004079882339F081E090E09093F10B809377
:1029D000F00B0DC083E090E00E9440798111F3CFAD
:1029E00083E090E00E9440798111EDCF06C0809194
:1029F000F00B9091F10B0197D9F06DE274E08DE14D
:102A000092E10E94904B6DE172E1CE0101960E942D
:102A10005B4C44E150E06FEF7FEFCE0101960E94E6
:102A2000778DCE0101960E94FF4B61E274E0CDC02C
:102A300065E174E083E292E10E94904B63E272E10F
:102A4000CE0101960E945B4CCE0101960E94938FAD
:102A5000CE0101960E94FF4B62E370E080E090E0BF
:102A60000E942F8663E272E1CE0101960E945B4CC8
:102A700042E350E06FEF7FEFCE0101960E94BF8FDF
:102A8000CE0101960E94FF4B69E074E08DE192E176
:102A90000E94904B6DE172E1CE0101960E945B4C69
:102AA00044E150E06FEF7FEFCE0101960E94778DF9
:102AB000CE0101960E94FF4B8BEB88A38AEA89A383
:102AC00081E08AA3C12CD12C412C512C3201212C24
:102AD000312CC6016AE070E00E9483B3892B49F46F
:102AE00043E050E0BE01605E7F4F85E79EE00E94BC
:102AF0005E4765E070E080E090E00E942F86BFEFC7
:102B0000CB1ADB0AE12CF12C812C912C540185E7A6
:102B10009EE00E94B947892B81F4E4E08E1691046F
:102B2000A104B10454F094E02916310464F4A0E93E
:102B3000CA16A1E0DA0669F606C0F6E0EF16F1045F
:102B40000CF4E3C7F0CFC301B2010E94BEAE20E097
:102B500030E040E251E40E940EB120E030E040E875
:102B60005EE30E941DAF6B017C0120E030E040EA93
:102B700051E40E94FDB1181634F521E0B701A60119
:102B8000CE0101960E94044C61E677E0CE0180966A
:102B90000E94634CBE016F5F7F4FCE0180960E9402
:102BA0007F4B6FE376E00E94684BBC0183E292E1C9
:102BB0000E94EA4BCE0180960E94FF4BCE01019607
:102BC0000E94FF4B06C06DEF73E083E292E10E942A
:102BD000904B63E272E1CE0101960E945B4C4AE0A9
:102BE00050E060E070E0CE0101960E94BF8FCE0100
:102BF00001960E94FF4B63E272E1CE0101960E94B2
:102C00005B4C69ED7BE0CE0101960E94684B6DE163
:102C100072E10E947F4BBC0183E292E10E94EA4B89
:102C2000CE0101960E94FF4B85E79EE00E94118E27
:102C30000DCA68EC74E0CE0101960E94534C4AE044
:102C400050E06FEF7FEFCE0101960E94778DCE01AD
:102C500001960E94FF4B6091B7027091B80280917B
:102C6000290290912A020E94F66EE4E18E2E912CA8
:102C7000A12CB12CC12CD12CAFEFCA1ADA0AC50194
:102C8000B4010E942F866091B7027091B8028091C2
:102C9000290290912A020E94F66E7C01B3E0CB16C5
:102CA000D10434F08EE1C816D10444F4EF2851F079
:102CB00094E1890E911CA11CB11CDECFE114F1043A
:102CC00009F00CC18091290290912A028B30910564
:102CD000C9F48091811290918212A0918312B091D7
:102CE00084128093421390934313A0934413B093A0
:102CF000451380917D1290917E12A0917F12B09128
:102D000080121DC08631910521F30C9701F5809149
:102D1000351390913613A0913713B09138138093E7
:102D2000421390934313A0934413B093451380919F
:102D3000311390913213A0913313B09134138093D7
:102D40003E1390933F13A0934013B09341134091CF
:102D5000421350914313609144137091451321E045
:102D6000CE0101960E94044C6CE07AE0CE01809680
:102D70000E94634CBE016F5F7F4FCE0180960E9420
:102D80007F4BBC0183E292E10E94EA4BCE01809628
:102D90000E94FF4BCE0101960E94FF4B40913E13D3
:102DA00050913F13609140137091411321E0CE0187
:102DB00001960E94044C62E476E0CE0180960E9467
:102DC000634CBE016F5F7F4FCE0180960E947F4BA8
:102DD000BC0183E292E10E94164BCE0180960E94D4
:102DE000FF4BCE0101960E94FF4B64E076E083E248
:102DF00092E10E94084B6EEB79E0CE0101960E94B1
:102E0000634C44E150E060E070E0CE0101960E9426
:102E1000BF8FCE0101960E94FF4BC0904213D0900D
:102E20004313E0904413F090451320E030E0A901F3
:102E3000C701B6010E94FDB120E030E040E05FE351
:102E400087FD05C0C701B6010E9448B004C0C70194
:102E5000B6010E9447B00E94A7B1AB01BC01CE01F0
:102E600001960E94A06ABE016F5F7F4F8DE192E1E3
:102E70000E941C4BCE0101960E94FF4B60E087E050
:102E80000E94756A6DE172E184E293E10E94C14C97
:102E90006FED84E293E10E94BA4C68E476E084E24C
:102EA00093E10E949A4D60913E1370913F1380917F
:102EB0004013909141130E94A7B14AE050E084E290
:102EC00093E10E94504D64E076E084E293E10E9439
:102ED0009A4D64E670E080E090E0C2C8EFEFEE1635
:102EE000FE06ACF06AEB74E0CE0101960E94534CF2
:102EF0004AE050E060E070E0CE0101960E94BF8F92
:102F0000CE0101960E94FF4B67E974E048C0FEEFD6
:102F1000EF16FFEFFF0679F169E874E0CE01019644
:102F20000E94534C4AE050E060E070E0CE01019610
:102F30000E94BF8FCE0101960E94FF4B6AE774E0AA
:102F400083E292E10E94904BB701CE0101960E946C
:102F50008950BE016F5F7F4F83E292E10E94164B62
:102F6000CE0101960E94FF4B64E674E083E292E199
:102F70000E94C64A60C569E574E0CE0101960E94D0
:102F8000534C4AE050E060E070E0CE0101960E94B0
:102F9000BF8FCE0101960E94FF4B69E374E083E28C
:102FA00092E10E94904B47C580910402882309F466
:102FB00042C56EEB79E0CE0101960E94634C4AE077
:102FC00050E061E070E0CE0101960E94BF8FCE011B
:102FD00001960E94FF4B0E94FD8B2DC58091470CEE
:102FE00081110AC080911811811106C07EE1472E1F
:102FF000512C612C712C05C063E0462E512C612CA4
:10300000712C66ED74E083E292E10E94904B63E2E2
:1030100072E1CE0101960E945B4C4AE050E06FEFF6
:103020007FEFCE0101960E94778DCE0101960E941E
:10303000FF4B812C912C54011CAE1DAE1EAE1FAE59
:1030400083E20E945A6A87E090E00E94556A0E94DB
:10305000536A66E970E080E090E00E942F8683E288
:103060000E945A6A80E290E00E94556A0E94536A68
:1030700066E970E080E090E00E942F8662E070E0F8
:1030800083E290E00E942D8FC12CD12C760180919B
:10309000701390E020917113821B91091816190684
:1030A0006CF48FEA9FE00E940956FE2CED2CDC2C7C
:1030B000CC24C80ED11CE11CF11CE9CFC701B6011C
:1030C0000E94BEAE2AE939E949E95FE30E940EB1E8
:1030D0000E94A7B1AB01BC0184169506A606B706EF
:1030E00014F44A015B01CE0180960E94A06ABE01E1
:1030F000605E7F4FCE0101960E945B4C6BE476E0F0
:10310000CE0101960E94684BBC018DE192E10E94C4
:10311000EA4BCE0101960E94FF4BCE0180960E94A1
:10312000FF4B6DE172E1CE0101960E945B4C4EE1D6
:1031300050E060E070E0CE0101960E946490CE0104
:1031400001960E94FF4B2CAD3DAD4EAD5FAD2F5FA4
:103150003F4F4F4F5F4F2CAF3DAF4EAF5FAF42166B
:103160005306640675060CF06BCFB501A401CE01C1
:1031700080960E94A06ABE01605E7F4FCE010196DC
:103180000E945B4C6BE476E0CE0101960E94684B96
:10319000BC018DE192E10E94EA4BCE0101960E94B2
:1031A000FF4BCE0180960E94FF4B6DE172E1CE0194
:1031B00001960E945B4C4AE050E060E070E0CE0176
:1031C00001960E94BF8FCE0101960E94FF4BB50170
:1031D000A401CE0101960E94A06A65E279E0CE01C9
:1031E00080960E94634CBE016F5F7F4FCE01809638
:1031F0000E947F4B6FE476E00E94684B63E272E1CD
:103200000E947F4BBC0183E292E10E94EA4BCE0117
:1032100080960E94FF4BCE0101960E94FF4B62E315
:1032200070E080E090E00C943010E090B502F090F7
:10323000B60281E080932C0564E670E080E090E0C7
:103240000E942F860E94E93EC7010E94E47860E058
:1032500074E0681B790BCE0101960E94895064E5E9
:1032600076E0CE0180960E94634CBE016F5F7F4F77
:10327000CE0180960E947F4BBC0183E292E10E94C6
:10328000EA4BCE0180960E94FF4BCE0101960E9430
:10329000FF4B60E087E00E94756A66EE74E0CE0145
:1032A00001960E94534C42E350E068E070E0CE018A
:1032B00001960E94BF8FCE0101960E94FF4B63E2F0
:1032C00072E1CE0101960E945B4C42E350E06FEF49
:1032D0007FEFCE0101960E94778DCE0101960E946C
:1032E000FF4B6BE576E0C7C08091B3029091B402CA
:1032F0000E94E4787C019093F30B8093F20B62E3DD
:1033000070E080E090E00E942F86B701CE01019628
:103310000E948950BE016F5F7F4F83E292E10E945D
:103320001C4BCE0101960E94FF4B80917B12909125
:103330007C12892B09F45EC067E772E1CE018096AA
:103340000E945B4CBE01605E7F4FCE0101960E94E1
:103350005B4C44E150E060E070E0CE0101960E94D9
:10336000BF8FCE0101960E94FF4B65E676E0CE014D
:1033700001960E94634C63E272E1CE0101960E94C5
:103380007F4BBC018DE192E10E94EA4BCE01019698
:103390000E94FF4B6DE172E1CE0101960E945B4CF1
:1033A00044E150E06FEF7FEFCE0101960E94778DF0
:1033B000CE0101960E94FF4BBE01605E7F4FCE01A1
:1033C00001960E945B4C69ED7BE0CE0101960E9464
:1033D000684B6DE172E10E947F4BBC0183E292E198
:1033E0000E94EA4BCE0101960E94FF4BCE018096CF
:1033F0000C94241060E776E08DE192E10E94D54BB9
:103400006DE172E1CE0101960E945B4C44E150E017
:1034100060E070E0CE0101960E94BF8FCE01019660
:103420000E94FF4B64E576E0CE0101960E94634C5A
:1034300063E272E1CE0101960E947F4BBC018DE1F7
:1034400092E10E94EA4BCE0101960E94FF4B6DE192
:1034500072E1CE0101960E945B4C44E150E06FEFB7
:103460007FEFCE0101960E94778DCE0101960E94DA
:10347000FF4B65E676E0CE0101960E94634C63E265
:1034800072E1CE0101960E947F4BBC0183E292E182
:103490000E94EA4BCE0101960E94FF4B0C9426102D
:1034A00080910402882309F4C6C28091470C8111DF
:1034B00004C080911811882329F082E090E00E94D6
:1034C000C442B9C2C0905502D0905602E090570253
:1034D000F090580220E030E040E450E4C701B6012B
:1034E0000E94FDB118166CF420E030E04AEF54E47D
:1034F000C701B6010E941DAF0E94A7B16B017C01FC
:1035000006C040E3C42E45E7D42EE12CF12C0E94E6
:10351000E93E60E080E00E94756A67EF74E084E253
:1035200093E10E94CF4C61E080E00E94756A6FEEEB
:1035300074E084E293E10E94CF4C64E670E080E0A6
:1035400090E00E942F860E948B876093EC0B709313
:10355000ED0B8093EE0B9093EF0B0E948B87809086
:10356000EC0B9090ED0BA090EE0BB090EF0BDC010C
:10357000CB0188199909AA09BB098C159D05AE05CF
:10358000BF050CF058C283E090E00E94C4420E9444
:103590008B8764E170E080E090E00E942F86DDCFB1
:1035A0000E9467628BE39DE00E94574844C267E136
:1035B00075E08DE192E10E94904B6DE172E1CE01E8
:1035C00001960E945B4C4AE050E060E070E0CE0162
:1035D00001960E94BF8FCE0101960E94FF4B309151
:1035E00061023CAF8091020C811105C00E948B8763
:1035F00081E08093020C8091FA0B811105C00E943A
:103600008B8781E08093FA0B1092F90B1092F80BE4
:103610002090F80B3090F90B48E2241631040CF09E
:103620007CC08CAD0E94E585F101EE0FFF1FEF55C8
:10363000F34F918380830E94EB6B20E030E040EAFF
:1036400050E40E941DAF20E030E040E85AE30E94C1
:103650001DAF2B013C0180901D0290901E02A09096
:103660001F02B0902002A50194016091190270918F
:103670001A0280911B0290911C020E9447B09B018C
:10368000AC0160E070E080EC90E40E9447B06B0118
:103690007C0120E030E0A9010E94B8AE20E030E0DB
:1036A00040E650E4811105C0C301B2010E941DAF84
:1036B0001EC0C301B2010E941DAFA50194010E946A
:1036C00048B020E030E040E850E40E9447B0A70155
:1036D00096010E940EB120E030E040EC50E40E94E0
:1036E0001DAF20E030E040E850E40E9448B0609315
:1036F000F40B7093F50B8093F60B9093F70B64E14A
:1037000070E080E090E00E942F865FEF251A350A76
:103710003092F90B2092F80B7BCFC090F40BD09035
:10372000F50BE090F60BF090F70B20E030E0A901EC
:10373000C701B6010E94FDB187FD1EC022E0B7019E
:10374000A601CE0101960E94044C64E776E0CE010A
:1037500080960E94634CBE016F5F7F4FCE018096C2
:103760000E947F4BBC0183E292E10E94EA4BCE01B2
:1037700080960E94FF4B49C168E075E083E292E1C8
:103780000E94904B46C180910402882309F453C1E2
:103790008091470C81112BC080911811811127C095
:1037A000C0905502D0905602E0905702F090580217
:1037B00020E030E04AE754E4C701B6010E941DAFA3
:1037C0000E94A7B14B015C0120E030E040EA50E4E8
:1037D000C701B6010E941DAF20E030E040EA50E48E
:1037E0000E9448B00E94A7B1A501940108C021E041
:1037F00030E040E050E06AE070E080E090E00E945D
:10380000BC6519C1C7010E94ED9115C1C7010E9495
:10381000795D11C180919A13882309F40CC165E682
:1038200075E0CE0101960E94534CCE0101960E9494
:103830002971FDC080919F0C9091A00C892BA1F45F
:1038400081E090E09093A00C80939F0C8EED93E02C
:1038500090933C0C80933B0C0E94526E68EC70E09D
:1038600080E090E00E942F8668E575E0CE01019629
:103870000E94534C44E650E06FEF7FEFCE0101967B
:103880000E94778DCE0101960E94FF4BE0E0F0E0B0
:103890001995D1C00E9423870E94E93E0E947B7641
:1038A000CAC090911D1181E0892780931D11882342
:1038B00069F161E575E083E292E10E94904B0E941C
:1038C0008B87609314117093151180931611909348
:1038D00017118091201190912111181619065CF48E
:1038E00020912211309123112817390724F01092CA
:1038F0002311109222119091241180911F11981779
:103900005CF0109224111092251106C069E475E054
:1039100083E292E10E94904B80911D1180931811D7
:1039200063E272E1CE0101960E945B4C4AE050E0F6
:1039300068E070E0CE0101960E94BF8FCE01019633
:103940000E94FF4B6CE375E0CE0101960E94534C40
:103950004AE050E06FEF7FEFCE0101960E94778D35
:10396000CE0101960E94FF4B6EE275E083E292E188
:103970000E94C64A61E179E0CE0101960E94634C43
:1039800063E272E1CE0101960E947F4BBC0183E2AB
:1039900092E10E94EA4BCE0101960E94FF4B80917A
:1039A000470C809326118CE291E00E94786E809102
:1039B000470C882309F43FC06FEE77E08FE292E175
:1039C0000E94D54B86EE9FEF90930C0C80930B0CCE
:1039D00032C0F0920C0CE0920B0C8BE39DE00E9445
:1039E000574860E275E083E292E10E94904B6EEBF3
:1039F00079E0CE0101960E94634C4AE050E060E01D
:103A000070E0CE0101960E94BF8FCE0101960E9408
:103A1000FF4B63E272E1CE0101960E945B4C4AE0EB
:103A200050E06FEF7FEFCE0101960E94778DCE01BF
:103A300001960E94FF4B80912712909128120097C7
:103A4000A1F0419720F4023011050CF0A3C063E20D
:103A500072E1CE0101960E945B4CCE0101960E945C
:103A60002971CE0101960E94FF4B64E670E080E070
:103A700090E00E942F86A1C00E940D3F0C94D40EAE
:103A8000EC80F12CFE2CEE248D81E80EF11CCE8012
:103A9000D12CDC2CCC248F81C80ED11CA884B12C55
:103AA000BA2CAA248985A80EB11C21E02CAF0C9455
:103AB000151266EC73E083E292E10E94904B63E2A0
:103AC00072E1CE0180960E945B4C4AE050E060E0DB
:103AD00070E0CE0180960E94778DCE0180960E9484
:103AE000FF4B63EB73E083E292E10E94904B809185
:103AF000110C9091120C029711F00C94E912109293
:103B0000120C1092110C0C94E91285E79EE00E94B1
:103B1000B947892B71F085E79EE00E949747E1E065
:103B2000F0E0EC0FFD1FEE0DFF1D80832FEFE21A7A
:103B3000F20A65E070E080E090E00E942F8636E0B7
:103B4000E316F10401F5998188A198131CC09A81AC
:103B500089A1981318C09B818AA1981314C08D81E4
:103B600090E0A0E0B0E0BA2FA92F982F88272C81F1
:103B7000820F911DA11DB11D480E591E6A1E7B1E8C
:103B80004FEF241A340A5FEF851A950AA50AB50A81
:103B90000C94871563E272E1CE0101960E945B4CA2
:103BA0004AE050E06FEF7FEFCE0101960E94778DE3
:103BB000CE0101960E94FF4B4ACFCB5BDF4F0FB681
:103BC000F894DEBF0FBECDBFDF91CF911F910F9153
:103BD000FF90EF90DF90CF90BF90AF909F908F902D
:103BE0007F906F905F904F903F902F9008952F920D
:103BF0003F924F925F926F927F928F929F92AF927D
:103C0000BF92CF92DF92EF92FF920F931F93CF93C9
:103C1000DF93CDB7DEB728970FB6F894DEBF0FBE9F
:103C2000CDBFFC0182EC9FE0938782878091BF0F1C
:103C300090E09587848780918C1090E097878687A5
:103C40008091BB0F853009F063C68091C40F9091BD
:103C5000C50F885891098D35910588F48091BF0F63
:103C6000843041F48091C60F9091C70F8097479799
:103C700008F47DC08091BF0F843408F05EC080914D
:103C8000BF0F8A3108F4D5C08091C20F9091C30F45
:103C9000843F914050F4118610868FEF9FEFDC0136
:103CA00084839583A683B7833CC08091C40F909191
:103CB000C50F85974B9708F0BCC008ECE02E0FE0CD
:103CC000F02E82E090E040E050E0BA018C010F5FFE
:103CD0001F4F2091BF0F30E0021713076CF49701BC
:103CE00022503109D9012D913C91275031092730BB
:103CF000310508F47FC0C801019795958795918794
:103D000080870C971CF41186108693C044835583DA
:103D10006683778384E090E00DC044835583668397
:103D200077838BE090E006C0448355836683778376
:103D30008CE090E0918380831EC58091C60F9091A6
:103D4000C70F825491098E9708F099CF20E030E098
:103D5000C12CD12C7601A9014853504FDA014D9165
:103D60005C91495051094930510598F088CF8091B4
:103D7000C80F9091C90F0997099708F07BCF11865A
:103D800010868FEF9FEFDC0184839583A683B78332
:103D9000C2C5B9016653704FDB014D915C9147512B
:103DA000510942315105C0F4D701C601880F991F4E
:103DB000AA1FBB1F6C017D016894C0F82C5F3F4FA8
:103DC0002038310541F620E230E031872087C48277
:103DD000D582E682F7829FC5DB014D915C9146500A
:103DE00051094730510508F04ACFCC0CDD1CEE1CC0
:103DF000FF1CE4CFD7012D913C91235131092F3085
:103E0000310550F4440F551F661F771F416002961D
:103E1000B4E0EB0EF11C5ACFD7012D913C912A5002
:103E200031092930310528F4440F551F661F771FCB
:103E3000EECF8091BF0F8A3108F460C08091C20F2D
:103E40009091C30F8032934008F425CF8091C40F26
:103E50009091C50FC697869708F050C08091C60F05
:103E60009091C70FC697869708F048C0BAECEB2E22
:103E7000BFE0FB2E83E090E040E050E0BA018C010F
:103E80000F5F1F4F2091BF0F30E00217130764F43C
:103E9000970122503109D9012D913C912C503109C3
:103EA0002B30310560F0C801019795958795918772
:103EB00080870C970CF031CF118610861FC0D70178
:103EC0002D913C91255231092B31310550F4440F8D
:103ED000551F661F771F41600296B4E0EB0EF11C80
:103EE000CECFD7012D913C912C5031092A3031058C
:103EF00028F4440F551F661F771FEECF8091BF0F28
:103F0000823208F452C08091C40F9091C50F069779
:103F1000079708F04AC048ECC42E4FE0D42E82E048
:103F200090E040E050E0BA018C010F5F1F4F2091FC
:103F3000BF0F30E002171307F4F4D6011297ED908B
:103F4000FC9011979D01BEE1EB1AF108A7E1EA167A
:103F5000F104E0F4440F551F661F771F4160D6013E
:103F60002D913C91B4E0CB0ED11C2350310925306A
:103F70003105C8F0C801019795958795918780878D
:103F800040970CF0D1CE118610860FC0D9012D912B
:103F90003C912C5031092B30310538F4440F551F1A
:103FA000661F771FDCCF0296BFCF7F011C821B826A
:103FB00081E090E09A8389838091BF0F8D3070F407
:103FC0001C821B8281E090E09A838983F7018485BB
:103FD0009585181619060CF474C0D1C029E733E092
:103FE000AE014D5F5F4FBE016F5F7F4FC7010E9403
:103FF0004999892B29F729E733E0AE014D5F5F4FDF
:10400000BE016F5F7F4FC7010E9449990197C1F6BA
:1040100029E733E0AE014D5F5F4FBE016F5F7F4F19
:10402000C7010E944999892B59F6812C912C540182
:1040300000E010E08091BF0F90E029813A812817BD
:10404000390794F529E733E0AE014D5F5F4FBE01BC
:104050006F5F7F4FC7010E9449996C0129E733E0E8
:10406000AE014D5F5F4FBE016F5F7F4FC7010E9482
:104070004999F1E0CF16D10451F4892B09F0A0CF72
:10408000880C991CAA1CBB1C689480F80AC0CD2817
:1040900009F096CF019709F093CF880C991CAA1CC0
:1040A000BB1C0F5F1F4FC6CFD70119961C930E93F1
:1040B0001897F70184829582A682B78281E090E00A
:1040C00039CE0284F385E02D82E090E09A838983E3
:1040D0008281938189974E9708F051C083E090E0E8
:1040E0009A838983848195810B970A9708F047C04A
:1040F0002CEB31E0AE014D5F5F4FBE016F5F7F4F34
:10410000C7010E944999892BD1F52CEB31E0AE0112
:104110004D5F5F4FBE016F5F7F4FC7010E9449999E
:10412000019769F5412C512C320100E010E0F701B4
:104130002485358589819A81821793070CF02FC1D8
:104140002CEB31E0AE014D5F5F4FBE016F5F7F4FE3
:10415000C7010E9449995C010330110509F0E5C0CF
:104160002CEB31E0AE014D5F5F4FBE016F5F7F4FC3
:10417000C7010E944999A816B90609F4D6C0D7010B
:104180001A96ED91FC911B9782819381C697869731
:10419000E0F4848195814B974597B8F4DF0116963A
:1041A0006F0126ECC20ED11C20E030E040E050E070
:1041B00060E070E080E090E00D911C911197095053
:1041C00011090830110508F4F4C08091BF0F89333C
:1041D00070F182819381895791098335910508F4A3
:1041E0001BC125C0D90112966D917C911397665120
:1041F00071096131710508F037C1D501C401880F1B
:10420000991FAA1FBB1F4C015D01689480F84E5F87
:104210005F4F2C5F3F4F4B33510509F40CC1D9015F
:104220006D917C916A50710969307105D8F2809165
:10423000BF0F823231F4828193810A97099708F483
:1042400023C1828193818957910983359105D0F4E7
:104250008091BF0F8132B0F084819581CA97899790
:1042600088F49F012A5F3F4F812C912C540143E039
:1042700050E0D9016D917C916A50710969307105E6
:1042800008F41EC1828193818C549109C59778F4FA
:104290008091BF0F843031F4848195818097479756
:1042A00008F46CC18091BF0F843408F04EC1809136
:1042B000BF0F863460F1828193810C970B9708F4CD
:1042C000A9C125C0D90112966D917C9113976E51A9
:1042D00071096731710508F0D1C1D501C401880F9A
:1042E000991FAA1FBB1F4C015D01689480F84E5FA7
:1042F0005F4F2C5F3F4F4534510509F4A6C1D901EA
:104300006D917C916C5071096B307105D8F2809180
:10431000BF0F883508F4E4C18281938185589109E3
:104320008B35910508F4BAC1DBC12CEB31E0AE014D
:104330004D5F5F4FBE016F5F7F4FC7010E9449997C
:104340006C010330110579F42CEB31E0AE014D5FC7
:104350005F4FBE016F5F7F4FC7010E944999C8162A
:10436000D90609F00CCFA114B10459F4CA94CD2890
:1043700009F005CF440C551C661C771C689440F866
:104380000BC0AA94AB2809F0FACECD2809F0F7CEDD
:10439000440C551C661C771C0F5F1F4FC8CE11873D
:1043A0000087F701448255826682778282E090E03E
:1043B000C1CC12960D911C911397015111090D302A
:1043C0001105E0F401E00E949EB321601496AC1543
:1043D000BD0509F0F1CEF701248335834683578369
:1043E00000E20E94B9B32283338385E090E0918399
:1043F000808380E390E091878087BDC112960D9104
:104400001C911397045011090530110508F0DDCEF9
:1044100001E00E949EB3DACF84819581CA97899783
:1044200008F005CF9F012A5F3F4F812C912C54014A
:1044300043E050E0F4CE9F012A583F4FD9012D911F
:104440003C912A5031092930310508F0F0CE2CE199
:1044500030E0F70131872087D70184829582A682D8
:10446000B7828AE090E085C1D90112966D917C9166
:104470001397665071096730710508F0D8CE880C23
:10448000991CAA1CBB1CC3CE2091BF0FCF01820F69
:10449000911D820F911DDC0112978D919C910A97BD
:1044A000099708F0CECEF701118610868FEF9FEFA7
:1044B000DC0184839583A683B78386E090E03ACCC1
:1044C000D90112966D917C911397665171096131F2
:1044D000710558F5D501C401880F991FAA1FBB1F8C
:1044E0004C015D01689480F84E5F5F4F2C5F3F4F39
:1044F0004332510509F0BDCE9F012A5B3F4FD901E0
:104500002D913C912A5031092930310508F0BACE5D
:1045100020E130E0F70131872087D701848295823E
:10452000A682B78286E090E024C1D90112966D91EF
:104530007C911397665071096730710508F0A2CE1F
:10454000880C991CAA1CBB1CCFCF848195818954EF
:104550009109C39708F0ABCE9F012A5F3F4FAF018F
:104560004A575F4F812C912C5401D9016D917C9158
:104570006950710969307105B8F099CE86819781CB
:104580000997099708F08ECED70119961C921E92B2
:1045900018978FEF9FEFDC01F70184839583A68343
:1045A000B78387E090E0C6CBD90112966D917C91DC
:1045B00013976651710961317105E0F4D501C401A9
:1045C000880F991FAA1FBB1F4C015D01689480F8DA
:1045D0002C5F3F4F2417350741F620E230E0F7010A
:1045E00031872087D70184829582A682B78287E0AF
:1045F00090E0BFC0D90112966D917C9113976650DF
:1046000071096730710508F052CE880C991CAA1CFC
:10461000BB1CDECF848195810997099708F077CE7E
:10462000868197818C974F9708F071CE8085918510
:1046300089974D9708F06BCE9F01265F3F4F812CE5
:10464000912C540145E050E05ACE9F0126573F4F30
:10465000D9012D913C912C5031092B30310508F0B6
:1046600056CE20E230E0F70131872087D7018482DF
:104670009582A682B78288E090E07BC0D90112962D
:104680006D917C911397695071096930710508F03B
:104690003ECE880C991CAA1CBB1C29CE8481958116
:1046A000825491098E97E0F48F01045C1F4F8DE1D5
:1046B00090E040E050E02091BF0F30E024503109FD
:1046C000821793070CF063C0980122503109D90179
:1046D0002D913C91295031092830310508F46EC0E4
:1046E0008091BF0F803209F07EC08281938106974E
:1046F000069708F078C0848195810997099708F09A
:1047000072C09F012A5F3F4FAF01425C5F4F812C17
:10471000912C5401D9016D917C91665071096630DC
:10472000710508F060C0D90112966D917C911397C4
:10473000695171096331710508F0D5C0D501C40113
:10474000880F991FAA1FBB1F4C015D01689480F858
:104750002C5F3F4F24173507E9F62EE030E0F701D4
:1047600031872087D70184829582A682B7828FE025
:1047700090E08D939C9381E090E0D0C0D8012D9182
:104780003C91285131092231310550F1CB0101977B
:1047900095958795D70119969C938E9318978A972C
:1047A0000CF49ECF052E000C660B770BF7014483AB
:1047B00055836683778389E090E0BCCABC016F5F54
:1047C0007F4FD8012D913C91275031092730310579
:1047D000A8F6440F551F416002960C5F1F4F6BCF28
:1047E000440F551FF9CFD7011C962D903C901D9773
:1047F000B6E02B1631040CF486C08F010E5F1F4FFC
:1048000075EC872E7DE9972E7CE1A72E71E8B72EF7
:10481000E3E0CE2ED12CF801648175816080718037
:1048200080E090E00E94BCAE6D837E838F8398878A
:10483000B30180E090E00E94BCAE2B013C012DEC66
:104840003CEC4CE45FE30E941DAF9B01AC016D8129
:104850007E818F8198850E94B8AE87FD19C02DECAE
:104860003CEC4CE45FE36D817E818F8198850E94F2
:104870001DAF9B01AC01C301B2010E94B8AEE82F8D
:10488000880FFF0BEE27FF0FEE1FFF27319602C0A8
:10489000E0E0F0E0A501940163E971E080E091E0DF
:1048A0000E9460B34F01FF0FAA08BB088626972617
:1048B000A826B926FFEFCF1ADF0A0E5F1F4F2C1470
:1048C0003D0409F0A8CFD70114968D929D92AD9228
:1048D000BC92179780E290E019969C938E9318975C
:1048E0008FEF9FEF46CFD90112966D917C91139770
:1048F000695071096930710508F075CF880C991CF1
:10490000AA1CBB1C25CF82E08093BB0F1092BF0F67
:1049100080E090E003C083E090E00CCA28960FB6D8
:10492000F894DEBF0FBECDBFDF91CF911F910F91E5
:10493000FF90EF90DF90CF90BF90AF909F908F90BF
:104940007F906F905F904F903F902F9008955F926F
:104950006F927F928F929F92AF92BF92CF92DF928F
:10496000EF92FF920F931F93CF93DF93CDB7DEB7F4
:10497000E4970FB6F894DEBF0FBECDBF63E277E0D9
:10498000CE0101960E94634CBE016F5F7F4F8BE3A7
:1049900092E10E941F85182FCE0101960E94FF4BC5
:1049A000112309F476C026E030E045E050E061E4F0
:1049B00072E1CE0101960E94774CBE016F5F7F4F7E
:1049C0008DE192E10E941C4BCE0101960E94FF4BAB
:1049D0008DE192E10E944A4A6B017C0163ED7AE02D
:1049E000CE0101960E94634CBE016F5F7F4F81E450
:1049F00092E10E94CF84AC014F5F5F4F61E472E1AE
:104A0000CE010B960E94343FBE01655F7F4F8DE162
:104A100092E10E941C4BCE010B960E94FF4BCE01EF
:104A200001960E94FF4B8DE192E10E944A4A9B0150
:104A3000E7E0F2E041E050E0A0910702B091080207
:104A4000A417B5075CF0A281B3812A173B0711F4C4
:104A5000138212824F5F5F4F3296EECF9601220F84
:104A6000331FF901E95FFD4F7183608382E090E0BD
:104A70000E94D57761E472E1CE0101960E945B4C01
:104A8000CE0101960E94938FCE0101960E94FF4BAA
:104A900031C069E277E0CE0101960E94634CBE010D
:104AA0006F5F7F4F8BE392E10E941F85182FCE012D
:104AB00001960E94FF4B112349F1E7E0F2E081E00B
:104AC00090E020910702309108022817390774F00E
:104AD000863091051CF49383828305C09C012E5F70
:104AE0003F4F3383228301963296EBCF82E090E0F2
:104AF0000E94D57710923C0C10923B0C80E090E025
:104B00000E94A26E109254020C94572F6FE277E02D
:104B1000CE0101960E94634CBE016F5F7F4F8BE315
:104B200092E10E941F85182FCE0101960E94FF4B33
:104B30001123F9F080919F0C9091A00C892BA1F486
:104B400081E090E09093A00C80939F0C8EED93E019
:104B500090933C0C80933B0C0E94526E68EC70E08A
:104B600080E090E00E942F86E0E0F0E019950C9440
:104B7000572F66E377E0CE0101960E94634CBE0199
:104B80006F5F7F4F8BE392E10E941F85182FCE014C
:104B900001960E94FF4B1123B1F06EE377E0CE0146
:104BA00001960E94634C62E173E1CE0101960E947E
:104BB0007F4BBC0183E292E10E94EA4BCE01019659
:104BC0000E94FF4B20C068E477E0CE0101960E946E
:104BD000634CBE016F5F7F4F8BE392E10E941F85A4
:104BE000182FCE0101960E94FF4B112351F16CE565
:104BF00077E083E292E10E94904B68E173E183E207
:104C000092E10E94164B61E179E0CE0101960E948B
:104C1000634C63E272E1CE0101960E947F4BBC01BE
:104C2000CE010B960E945B4CCE010B960E9429711F
:104C3000CE010B960E94FF4BCE0101960E94FF4BC6
:104C400061CF6FE477E0CE0101960E94634CBE0114
:104C50006F5F7F4F8BE392E10E941F85182FCE017B
:104C600001960E94FF4B112311F169E377E083E283
:104C700092E10E94904B63E272E1CE0101960E94A4
:104C80005B4CCE0101960E942971CE0101960E94D3
:104C9000FF4B0E94025A1092540265E577E081E4CE
:104CA00092E10E94D54B0E949C7E0C94572F69E59F
:104CB00077E0CE0101960E94634CBE016F5F7F4F8B
:104CC0008BE392E10E941F85182FCE0101960E946E
:104CD000FF4B112309F48CC063ED7AE0CE010196FD
:104CE0000E94634CBE016F5F7F4F81E492E10E949E
:104CF000CF84AC014F5F5F4F61E472E1CE010B9650
:104D00000E94343FBE01655F7F4F8DE192E10E94BA
:104D10001C4BCE010B960E94FF4BCE0101960E94C8
:104D2000FF4B8DE192E10E944A4A8B016CE277E0F1
:104D300083E292E10E94904B80911D11882331F013
:104D400060E277E083E292E10E94904B0115110549
:104D500011F40C94432FCE0101960E94555ACE01B6
:104D600001960E942971CE0101960E94FF4B0230EC
:104D700011050CF4C7CE67E775E0CE010B960E94D3
:104D8000534CBE01655F7F4FCE0101960E945B4C84
:104D9000CE0101960E942971CE0101960E94FF4B1F
:104DA000E12CF12C80911F11082E000C990BE816B4
:104DB000F9068CF4B701CE0101960E945E5CCE012B
:104DC00001960E942971CE0101960E94FF4BFFEFD0
:104DD000EF1AFF0AE7CFCE010B960E94FF4B02307D
:104DE000110509F48FCE8CE291E00E94CC6E8ACE40
:104DF00060E677E0CE0101960E94634CBE016F5FD2
:104E00007F4F8BE392E10E941F85182FCE01019600
:104E10000E94FF4B112309F488C361E472E1CE01C3
:104E20008F960E945B4C63ED7AE0CE0101960E9462
:104E3000634CBE016F5F7F4FCE018F960E94CF847F
:104E4000AC014F5F5F4FBE01615D7F4FCE01899620
:104E50000E94343FCE0101960E94FF4BBE01615D6E
:104E60007F4FCE0101960E945B4CCE0101960E94BD
:104E7000938FCE0101960E94FF4B64E677E0CE014E
:104E800001960E94634CBE016F5F7F4FCE018996F1
:104E90000E9493848C01CE0101960E94FF4B6EEB21
:104EA00079E0CE0183960E94634C6EEB79E0CE01EF
:104EB0004D960E94634C1016110684F5A8014F5FB1
:104EC0005F4F8DA59EA54817590790F4BE01675DF9
:104ED0007F4FCE0101960E94343FBE016F5F7F4F2E
:104EE000CE0183960E941C4BCE0101960E94FF4B7F
:104EF000980140E050E0BE01675D7F4FCE01019612
:104F00000E94774CBE016F5F7F4FCE014D960E948D
:104F10001C4BCE0101960E94FF4B0DC06EEB79E059
:104F2000CE0183960E94D54BBE01675D7F4FCE01B7
:104F30004D960E94EA4B89A19AA1892B09F4E6C2F9
:104F4000CE014D960E944A4A8B0101501109083149
:104F5000110514F007E110E017FF02C00FEF1FEF7B
:104F6000B801CE010B960E94895066E677E0CE012B
:104F700001960E94634CBE01655F7F4FCE01019692
:104F80000E947F4BBC01CE0141960E945B4CCE013A
:104F900041960E94938FCE0141960E94FF4BCE0115
:104FA00001960E94FF4BCE010B960E94FF4BBE0163
:104FB0006D5D7F4FCE0189960E94EA4B64E677E0F3
:104FC000CE0101960E94634CBE016F5F7F4FCE0100
:104FD00089960E9493847C01CE0101960E94FF4B2A
:104FE0006EEB79E0CE0183960E94D54B6EEB79E0B3
:104FF000CE014D960E94D54B1E141F040CF04EC0DE
:10500000A7014F5F5F4F8DA59EA54817590790F4E4
:10501000BE01675D7F4FCE0101960E94343FBE0105
:105020006F5F7F4FCE0183960E941C4BCE0101968D
:105030000E94FF4B970140E050E0BE01675D7F4F4B
:10504000CE0101960E94774CBE016F5F7F4FCE016B
:105050004D960E941C4BCE0101960E94FF4BAE0163
:105060004F5F5F4F5A01E12CF12CA8014F5F5F4F5A
:105070008AE0849F9001859F300D1124F901E35E41
:10508000FE4E6F01809F9001819F300D1124A90178
:10509000455D5E4E3A018AE2582EC1C06EEB79E062
:1050A000CE0183960E94D54BBE01675D7F4FCE0136
:1050B0004D960E94EA4BD3CFE114F10409F0BCC035
:1050C0000F3F8FEF180709F4B7C0CE014D960E942D
:1050D000554AC114D10439F044E050E0B601CE0184
:1050E0004D960E94AD84B601CE0141960E94634C5C
:1050F0006BE677E0CE010B960E94634CBE016F5EBB
:105100007F4FCE010B960E947F4BBC01CE0147968C
:105110000E945B4CCE0147960E94938FCE0147962A
:105120000E94FF4BCE010B960E94FF4BCE01419691
:105130000E94FF4B89A19AA1029708F476C061E012
:1051400070E0CE014D960E94B54A082E000C990BD6
:10515000803391050CF44C96E52DE81B8E2FF3015E
:105160008083FFEFEF1AFF0ABE016D5D7F4FCE0116
:1051700089960E94EA4B64E677E0CE010B960E9486
:10518000634CBE01655F7F4FCE0189960E94938478
:105190004C01CE010B960E94FF4B6EEB79E0CE01E5
:1051A00083960E94D54B6EEB79E0CE014D960E941E
:1051B000D54B181419040CF047C0A4014F5F5F4F82
:1051C0008DA59EA54817590790F4BE01675D7F4FD6
:1051D000CE010B960E94343FBE01655F7F4FCE012A
:1051E00083960E941C4BCE010B960E94FF4B9401AC
:1051F00040E050E0BE01675D7F4FCE010B960E94FC
:10520000774CBE01655F7F4FCE014D960E941C4BCF
:10521000CE010B960E94FF4B52E0A50EB11C89A156
:105220009AA1892B09F048CF1DC0CE014D960E944E
:105230004A4AF301608395CFCE014D960E944A4AB7
:10524000F501718360838DCF6EEB79E0CE0183969B
:105250000E94D54BBE01675D7F4FCE014D960E94E7
:10526000EA4BDACF0F3F2FEF120709F07DC064E65B
:1052700077E0CE010B960E94634CBE01655F7F4FC5
:10528000CE0183960E9493848C01CE010B960E94DE
:10529000FF4B17FF3BC109811A811016110634F428
:1052A000093111052CF008E110E002C001E010E026
:1052B00000931F11B801CE0141960E94895069E701
:1052C00077E0CE010B960E94634CBE016F5E7F4F6C
:1052D000CE010B960E947F4BBC01CE0147960E94E7
:1052E0005B4CCE0147960E94938FCE0147960E9459
:1052F000FF4BCE010B960E94FF4BCE0141960E94C0
:10530000FF4BE114F10459F18B819C8197FF02C09E
:1053100080E090E0909321118093201141E0E41609
:10532000F104E9F08D819E81181619062CF480177E
:10533000910724F48C0102C001E010E001500093B9
:10534000241152E0E516F10451F08F81988518166A
:10535000190614F081E090E08150809325118CE2D1
:1053600091E00E94786ED2C080911E11082E000C30
:10537000990B081719070CF083C0B701CE014196AD
:105380000E94895063E877E0CE010B960E94634C3F
:10539000BE016F5E7F4FCE010B960E947F4BBC011A
:1053A000CE0147960E945B4CCE0147960E94938F98
:1053B000CE0147960E94FF4BCE010B960E94FF4BF9
:1053C000CE0141960E94FF4B8AE0809FF001819FB1
:1053D000F00D1124E35EFE4E81E0878783E090E0CC
:1053E000918B808B938B828BE114F10409F48EC036
:1053F0008B819C818038910514F08FE790E0803894
:105400002FEF920714F480E89FEF878741E0E416BE
:10541000F10409F47BC08AE0809FF001819FF00DC8
:105420001124E35EFE4E8D819E8197FF02C080E0D5
:1054300090E0918B808B52E0E516F10409F466C090
:105440008AE0809FF001819FF00D1124E35EFE4E03
:105450008F81988597FF02C080E090E0938B828BCC
:1054600080911F11082E000C990B081719071CF0CA
:105470000F5F00931F118CE291E00E94CC6E46C03A
:10548000BE016D5D7F4FCE0147960E945B4C6091DF
:105490001E11062E000C770BCE0141960E948950FA
:1054A0006BE877E0CE010B960E94634CBE01695E0B
:1054B0007F4FCE010B960E947F4B6CE977E00E94F4
:1054C000684BBE016F5E7F4F0E947F4BBC01CE01D7
:1054D00047960E94EA4BCE010B960E94FF4BCE01ED
:1054E00041960E94FF4BBE01695E7F4FCE010B9635
:1054F0000E945B4CCE010B960E942971CE010B9647
:105500000E94FF4BCE0147960E94FF4BCE014D9665
:105510000E94FF4BCE0183960E94FF4BCE018996DD
:105520000E94FF4BCE018F9650C260EA77E0CE0119
:1055300001960E94634CBE016F5F7F4F8BE392E147
:105540000E941F85182FCE0101960E94FF4B112348
:10555000C9F163ED7AE0CE0101960E94634CBE0171
:105560006F5F7F4F81E492E10E94CF84AC014F5F77
:105570005F4F61E472E1CE010B960E94343FBE01A1
:10558000655F7F4F8DE192E10E941C4BCE010B962F
:105590000E94FF4BCE0101960E94FF4B8DE192E1EC
:1055A0000E944A4A6115710521F481E080932E051D
:1055B00006C06130710509F0A5CA10922E050E943F
:1055C0008B76A0CA65EA77E0CE0101960E94634C13
:1055D000BE016F5F7F4F8BE392E10E941F85182F02
:1055E000CE0101960E94FF4B112309F452C143E002
:1055F00050E061E472E1CE0101960E94343FBE01A9
:105600006F5F7F4F8DE192E10E941C4BCE010196AE
:105610000E94FF4B6DE172E1CE0101960E945B4C4E
:10562000CE0101960E94938FCE0101960E94FF4BFE
:1056300010923C0C10923B0C6DE172E1CE01019690
:105640000E945B4C60E0CE0101960E94F54A8111F8
:1056500004C0CE0101960E94564BBE016F5F7F4F82
:105660008EE193E10E94EA4BCE0101960E94FF4B2E
:105670006DE172E1CE0101960E945B4C60E0CE01CB
:1056800001960E94F54A811104C0CE0101960E9444
:10569000564BBE016F5F7F4F88E193E10E94EA4B5A
:1056A000CE0101960E94FF4B40912213509123138B
:1056B0004115510549F08AEA90E1009729F0BC01B3
:1056C0008EE193E10E94AD8440911C1350911D1313
:1056D0004115510549F088E091E1009729F0BC019E
:1056E00088E193E10E94AD8480913B0C90913C0C49
:1056F0000E94A26E6AEF76E0CE0101960E94634C92
:105700006DE172E1CE0101960E947F4BBC01CE019A
:1057100041960E945B4CCE0101960E94FF4B809106
:10572000041190910511892B39F4BE016F5E7F4FF2
:105730008BE39DE00E94C14C68EB7BE080E090E051
:105740000E942F868091041190910511029709F013
:1057500087C06DE172E1CE0147960E945B4C69EA19
:1057600077E0CE0101960E94634CCE0101960E9423
:10577000A5A9CE0101960E94FF4B64EF71E080E085
:1057800090E00E942F866CEA77E0CE0101960E949D
:10579000634CCE0101960E94A5A9CE0101960E94FC
:1057A000FF4B6CED75E080E090E00E942F8665EB8A
:1057B00077E0CE0101960E94634CCE0101960E94D3
:1057C000A5A9CE0101960E94FF4B64EF71E080E035
:1057D00090E00E942F8663EC77E0CE0101960E9454
:1057E000634CCE0101960E94A5A9CE0101960E94AC
:1057F000FF4B64EF71E080E090E00E942F866AEF3B
:1058000076E0CE0101960E94634CBE01695E7F4F37
:10581000CE0101960E947F4BBC01CE010B960E94E7
:105820005B4CCE0101960E94FF4BCE010B960E946D
:10583000554ABE01655F7F4FCE0101960E945B4CC9
:10584000CE0101960E94A5A9CE0101960E94FF4BB0
:10585000CE010B960E94FF4BCE0147960E94FF4B54
:1058600068EB7BE080E090E00E942F866AEA70E1BE
:10587000CE0101960E94634CCE0101960E94938F47
:10588000CE0101960E94FF4B10925402CE01419628
:105890009CC061ED77E0CE0101960E94634CBE0191
:1058A0006F5F7F4F8BE392E10E941F85182FCE011F
:1058B00001960E94FF4B112309F48AC044E050E096
:1058C00061E472E1CE0101960E94343FBE016F5F38
:1058D0007F4F8DE192E10E941C4BCE0101960E9408
:1058E000FF4B62E077E0CE0101960E94634C6DE1D0
:1058F00072E1CE0101960E947F4BBC01CE010B9656
:105900000E945B4CCE0101960E94FF4B80910411D6
:1059100090910511892B69F4BE01655F7F4F8BE380
:105920009DE00E94C14C68E873E180E090E00E9435
:105930002F868091041190910511029709F041C0C2
:1059400066ED77E0CE0101960E94634C80912112B2
:1059500090912212892B39F46FED77E0CE010196F8
:105960000E94D54B15C0BE016F5F7F4FCE0141969F
:105970000E945B4CCE0141960E94A5A9CE014196A2
:105980000E94FF4B60ED77E080E090E00E942F8660
:10599000BE01655F7F4FCE0141960E945B4CCE01F8
:1059A00041960E94A5A9CE0141960E94FF4B60ED51
:1059B00077E080E090E00E942F86CE0101960E9461
:1059C000FF4B10925402CE010B960E94FF4B6FC208
:1059D00068EE77E0CE0101960E94634CBE016F5FD6
:1059E0007F4F8BE392E10E941F85182FCE01019615
:1059F0000E94FF4B112309F462C061E472E18DE162
:105A000092E10E94EA4B81E08093540261E472E1EA
:105A1000CE0101960E945B4CCE0101960E94938FAD
:105A2000CE0101960E94FF4B8091041190910511C7
:105A3000029709F16DE172E18BE39DE00E94C14C98
:105A400068EB7BE080E090E00E942F86CE0101961B
:105A50000E94EB75BE016F5F7F4F81E492E10E946F
:105A60001C4BCE0101960E94FF4B60ED77E080E079
:105A700090E00E942F868091041190910511029769
:105A800071F46DE172E1CE0101960E945B4CCE0192
:105A900001960E94A5A9CE0101960E94FF4B80911C
:105AA000451290914612892B09F42CC861E179E0E6
:105AB000CE0101960E94634C61E472E1ACC86CEEC9
:105AC00077E0CE0101960E94634CBE016F5F7F4F6D
:105AD0008BE392E10E941F85182FCE0101960E9450
:105AE000FF4B112309F45CC08091041190910511C2
:105AF000019709F007C8CE0101960E94E8608D81E8
:105B00009E81009709F4C9C1E981FA81208122238D
:105B100009F4C3C1079708F4C0C167E177E0CE017B
:105B20000B960E94534C48EC50E06FEF7FEFCE0194
:105B30000B960E946490CE010B960E94FF4BBE0113
:105B40006F5F7F4FCE010B960E945B4C40ED57E09C
:105B50006FEF7FEFCE010B960E94778DCE010B96F3
:105B60000E94FF4B62EF77E0CE010B960E94634CE0
:105B700061E472E1CE010B960E947F4BBC01CE0125
:105B800041960E945B4CCE0141960E942971CE0144
:105B900041960E94FF4BCE010B960E94FF4B7DC1A8
:105BA00060E078E0CE0101960E94634CBE016F5F19
:105BB0007F4F8BE392E10E941F85182FCE01019643
:105BC0000E94FF4B112361F125E030E044E050E0FA
:105BD00061E472E1CE0101960E94774CBE016F5FD5
:105BE0007F4F8DE192E10E941C4BCE0101960E94F5
:105BF000FF4B61E472E1CE0101960E945B4CCE0145
:105C000001960E94938FCE0101960E94FF4B8DE179
:105C100092E10E944A4ACB010E941D910C94822578
:105C200065E078E0CE0101960E94634CBE016F5F93
:105C30007F4F8BE392E10E941F85182FCE010196C2
:105C40000E94FF4B112361F127E030E046E050E075
:105C500061E472E1CE0101960E94774CBE016F5F54
:105C60007F4F8DE192E10E941C4BCE0101960E9474
:105C7000FF4B8DE192E10E944A4A672B19F4109282
:105C80009A1303C081E080939A1361E472E1CE011C
:105C900001960E945B4CCE0101960E94938FFDC03D
:105CA0006CE078E0CE0101960E94634CBE016F5F0C
:105CB0007F4F8BE392E10E941F85182FCE01019642
:105CC0000E94FF4B112309F476C0809145129091F8
:105CD0004612079708F4EBC046E050E061E472E139
:105CE000CE0101960E94343FBE016F5F7F4F8DE170
:105CF00092E10E941C4BCE0101960E94FF4B8DE168
:105D000092E10E943F4A6093500270935102809347
:105D100052029093530267E077E083E292E10E949F
:105D2000904B4091500250915102609152027091FB
:105D3000530221E0CE0101960E94044CBE016F5F28
:105D40007F4FCE010B960E945B4C6BED75E0CE0150
:105D50000B960E94684BBC0183E292E10E94164BB5
:105D6000CE010B960E94FF4BCE0101960E94FF4B85
:105D700063E272E1CE0101960E945B4CCE01019676
:105D80000E942971CE0101960E94FF4B0E948B87D1
:105D900028EE33E040E050E00E9416B0CA01B9019D
:105DA0000E94BCAE6093430C7093440C8093450CEE
:105DB0009093460C7CC063E178E0CE0101960E948E
:105DC000634CBE016F5F7F4F8BE392E10E941F85A2
:105DD000182FCE0101960E94FF4B112309F463C0D6
:105DE0008091451290914612079708F460C046E0F2
:105DF00050E061E472E1CE0101960E94343FBE01A1
:105E00006F5F7F4F8DE192E10E941C4BCE010196A6
:105E10000E94FF4B8DE192E10E943F4A6093550240
:105E200070935602809357029093580267EF76E082
:105E300083E292E10E94904B4091550250915602AC
:105E4000609157027091580221E0CE0101960E94A4
:105E5000044CBE016F5F7F4FCE010B960E945B4CDE
:105E60006BED75E0CE010B960E94684BBC0183E29E
:105E700092E10E94164BCE010B960E94FF4BCE0181
:105E800001960E94FF4B63E272E1CE0101960E94EF
:105E90005B4CCE0101960E942971CE0101960E94B1
:105EA000FF4B0C948225E9D5182F8823A1F010917F
:105EB0005402112379F061E472E1CE0101960E944F
:105EC0005B4CCE0101960E94938FCE0101960E94F9
:105ED000FF4B01C011E0812FE4960FB6F894DEBFAE
:105EE0000FBECDBFDF91CF911F910F91FF90EF902B
:105EF000DF90CF90BF90AF909F908F907F906F90EA
:105F00005F9008954F925F926F927F929F92AF92AF
:105F1000BF92CF92DF92EF92FF920F931F93CF9396
:105F2000DF93CDB7DEB7A9970FB6F894DEBF0FBEEB
:105F3000CDBF982E882351F080919A13882331F099
:105F40006EEB79E082E19FE00E94CD6A0E9457509B
:105F500060E08DE20E94B25160E18DE20E94B25198
:105F600068E08DE20E94B25140908D1250908E12E6
:105F700060908F1270909012498E5A8E6B8E7C8E2C
:105F8000C0909112D0909212E0909312F0909412DF
:105F9000CD8EDE8EEF8EF8A28091951290919612A2
:105FA000A0919712B09198128EA39FA3A8A7B9A70A
:105FB00089A39AA3ABA3BCA39920C9F180919A139A
:105FC0008823A9F164E47BE0CE0101960E94534C42
:105FD000CE0101960E94938FCE0101960E94FF4B45
:105FE0008E01075E1F4F5E0195E2A90EB11CD8011C
:105FF0006D917D918D919D918D0146E00E94116B77
:1060000069ED7BE082E19FE00E949A4DA016B10607
:1060100071F76EEB79E0CE0101960E94634CCE01E0
:1060200001960E94938FCE0101960E94FF4B23E9B7
:1060300038E144E85FE3C301B2010E941DAF2B01C8
:106040003C016D877E878F87988B22E430E645E898
:106050005FE3C701B6010E941DAF6B017C01698B34
:106060007A8B8B8B9C8B25E83BEE41E95FE36EA13D
:106070007FA188A599A50E941DAF6D8B7E8B8F8B0C
:10608000988F40928D1250928E1260928F12709261
:106090009012C0929112D0929212E0929312F092CA
:1060A0009412609395127093961280939712909326
:1060B0009812992009F4A0C080919A13882309F4BA
:1060C0009BC067E37BE0CE0101960E94534CCE015A
:1060D00001960E94938FCE0101960E94FF4B8E0184
:1060E000035F1F4F6E01B9E1CB0ED11C7801F8019F
:1060F00061917191819191918F0142E00E94116BA8
:1061000069ED7BE082E19FE00E949A4DC016D106C6
:1061100071F76EEB79E0CE0101960E94634CCE01DF
:1061200001960E94938FCE0101960E94FF4B49E990
:1061300052E166E070E082E30E944D51A090991216
:10614000B0909A12C0909B12D0909C1200919D1218
:1061500010919E126AE27BE082E19FE00E94CF4CA8
:106160004AE050E0B50182E19FE00E94504D69EDA8
:106170007BE082E19FE00E949A4D4AE050E0B60148
:1061800082E19FE00E94504D69ED7BE082E19FE05B
:106190000E949A4D4AE050E0B80182E19FE00E94DF
:1061A000504D6EEB79E082E19FE00E94CD6ACE0116
:1061B00001960E941F5261E27BE082E19FE00E9413
:1061C000CF4C8E010F5F1F4FD8016D917D918D9146
:1061D0009D918D014AE00E94116B69ED7BE082E1A7
:1061E0009FE00E949A4D0E151F0571F76EEB79E046
:1061F00082E19FE00E94CD6A61E08DE10E94B25190
:106200009920B1F080919A13882391F06DE07BE0A2
:1062100082E19FE00E94CF4CAE014B5D5F4F61E099
:1062200070E08DE10E944D518DA190E00E94865159
:1062300062E08EE10E94B25163E08FE10E94B251B0
:1062400064E080E20E94B251992009F450C080912C
:106250009A13882309F44BC061EF7AE082E19FE052
:106260000E94CF4CAE014B5D5F4F61E070E08EE16C
:106270000E944D51CDA0D12CAE014B5D5F4F61E02E
:1062800070E08FE10E944D51EDA0F12CAE014B5D0D
:106290005F4F61E070E080E20E944D510DA110E07F
:1062A0004AE050E0B60182E19FE00E94504D69ED66
:1062B0007BE082E19FE00E949A4D4AE050E0B70106
:1062C00082E19FE00E94504D69ED7BE082E19FE01A
:1062D0000E949A4D4AE050E0B80182E19FE00E949E
:1062E000504D6EEB79E082E19FE00E94CD6A65E05F
:1062F00081E20E94B2519920B1F080919A138823D3
:1063000091F06EED7AE082E19FE00E94CF4CAE0109
:106310004B5D5F4F61E070E081E20E944D518DA1C5
:1063200090E00E94865166E082E20E94B25199207C
:10633000B1F080919A13882391F066EC7AE082E1C3
:106340009FE00E94CF4CAE014B5D5F4F61E070E07B
:1063500082E20E944D518DA190E00E94865167E03B
:1063600083E20E94B2519920B1F080919A13882360
:1063700091F060EB7AE082E19FE00E94CF4CAE01A9
:106380004B5D5F4F61E070E083E20E944D518DA153
:1063900090E00E94865168E084E20E94B251992008
:1063A000B1F080919A13882391F068E97AE082E154
:1063B0009FE00E94CF4CAE014B5D5F4F61E070E00B
:1063C00084E20E944D518DA190E00E94865169E0C7
:1063D00085E20E94B2519920B1F080919A138823EE
:1063E00091F06EE77AE082E19FE00E94CF4CAE012F
:1063F0004B5D5F4F61E070E085E20E944D518DA1E1
:1064000090E00E9486516AE086E20E94B251992093
:10641000B1F080919A13882391F068E67AE082E1E6
:106420009FE00E94CF4CAE014B5D5F4F61E070E09A
:1064300086E20E944D518DA190E00E9486516BE052
:1064400088E20E94B2519920B1F080919A1388237A
:1064500091F06FE47AE082E19FE00E94CF4CAE01C0
:106460004B5D5F4F61E070E088E20E944D518DA16D
:1064700090E00E9486516CE089E20E94B25199201E
:1064800009F479C080919A13882309F474C067E3F2
:106490007AE082E19FE00E94CF4CAE014B5D5F4FFE
:1064A00061E070E089E20E944D518DA190E00E9470
:1064B000865160E27AE082E19FE00E94CF4C66E084
:1064C00070E087E20E94985190E00E94865169E056
:1064D0007AE082E19FE00E94CF4C65E070E087E2C5
:1064E0000E94985190E00E94865162EF79E082E12B
:1064F0009FE00E94CF4C64E070E087E20E949851D8
:1065000090E00E94865169ED79E082E19FE00E946F
:10651000CF4C62E070E087E20E94985190E00E94C8
:10652000865160EC79E082E19FE00E94CF4C61E00F
:1065300070E087E20E94985190E00E94865167EADD
:1065400079E082E19FE00E94CF4C60E070E087E25A
:106550000E94985190E00E94865166E979E082E1BC
:106560009FE00E94CF4C63E070E087E20E94985168
:1065700090E00E94865141E067E070E087E20E946F
:10658000C55141E063E070E087E20E94C55141E0FF
:1065900063E070E08AE20E94C551992091F08091F9
:1065A0009A13882371F06DE779E082E19FE00E9401
:1065B000CF4C63E070E08AE20E94985190E00E9424
:1065C000865140E063E070E08AE20E94C551992064
:1065D00091F080919A13882371F063E679E082E16B
:1065E0009FE00E94CF4C63E070E08AE20E949851E5
:1065F00090E00E94865141E062E070E08AE20E94F1
:10660000C551992091F080919A13882371F067E425
:1066100079E082E19FE00E94CF4C62E070E08AE284
:106620000E94985190E00E94865140E062E070E044
:106630008AE20E94C551992091F080919A13882393
:1066400071F06AE279E082E19FE00E94CF4C62E063
:1066500070E08AE20E94985190E00E94865141E0E9
:1066600061E070E08AE20E94C551992091F080912A
:106670009A13882371F06EE079E082E19FE00E9436
:10668000CF4C61E070E08AE20E94985190E00E9455
:10669000865140E061E070E08AE20E94C551992095
:1066A00091F080919A13882371F061EF78E082E194
:1066B0009FE00E94CF4C61E070E08AE20E94985116
:1066C00090E00E94865141E060E070E08AE20E9422
:1066D000C551992091F080919A13882371F065ED4E
:1066E00078E082E19FE00E94CF4C60E070E08AE2B7
:1066F0000E94985190E00E94865140E060E070E076
:106700008AE20E94C551992091F080919A138823C2
:1067100071F068EB78E082E19FE00E94CF4C60E08E
:1067200070E08AE20E94985190E00E94865141E018
:1067300066E070E087E20E94C55141E065E070E0EC
:1067400087E20E94C55141E064E070E087E20E9468
:10675000C55140E062E070E087E20E94C55140E030
:1067600061E070E087E20E94C55140E060E070E0C7
:1067700087E20E94C551992009F475C080919A134F
:10678000882309F470C060EA78E082E19FE00E940B
:10679000CF4C66E070E08BE20E94985190E00E943E
:1067A000865162E878E082E19FE00E94CF4C65E08C
:1067B00070E08BE20E94985190E00E94865164E65E
:1067C00078E082E19FE00E94CF4C64E070E08BE2D1
:1067D0000E94985190E00E9486516BE478E082E13B
:1067E0009FE00E94CF4C62E070E08BE20E949851E3
:1067F00090E00E94865162E378E082E19FE00E948F
:10680000CF4C61E070E08BE20E94985190E00E94D2
:10681000865169E178E082E19FE00E94CF4C60E020
:1068200070E08BE20E94985190E00E94865166E0F1
:1068300078E082E19FE00E94CF4C63E070E08BE261
:106840000E94985190E00E94865161EF77E082E1CA
:106850009FE00E94CF4C64E070E08CE20E9498516F
:1068600090E00E94865140E064E070E08CE20E947B
:10687000C551AE014B5D5F4F61E070E08CE20E945C
:106880004D516DA1607F66608CE20E94B2519920EB
:1068900009F45FC080919A13882309F45AC06DED02
:1068A00077E082E19FE00E94CF4CAE014B5D5F4FED
:1068B00061E070E08CE20E944D516DA16F7070E05C
:1068C00066507109072E000C880B990B0E94BEAE12
:1068D0009B01AC0160E070E080E090E40E94B6B201
:1068E00020E030E048EC50E40E941DAF0E941052BE
:1068F00066EC77E082E19FE00E94CF4CAE014B5DF9
:106900005F4F61E070E080E30E944D516DA14AE06D
:1069100050E082E19FE00E94F5516EEA77E082E16B
:106920009FE00E94CF4C61E070E080E30E949851AC
:1069300090E00E94865165E977E082E19FE00E9445
:10694000CF4C61E070E08FE20E94985190E00E948D
:10695000865141E061E070E08FE20E94C5519920CC
:1069600091F080919A13882371F06DE777E082E1CE
:106970009FE00E94CF4C61E070E08EE20E9498514F
:1069800090E00E94865141E061E070E08EE20E945A
:10699000C55140E067E070E081E30E94C551992055
:1069A00009F455C080919A13882309F450C06AE60F
:1069B00077E082E19FE00E94CF4C67E070E081E3E6
:1069C0000E94985190E00E9486516AE178E082E14D
:1069D0009FE00E949A4DAE014B5D5F4F61E070E019
:1069E00080E00E944D518DA10E94AC586EEB79E081
:1069F00082E19FE00E94CD6A0DE110E06DE976E052
:106A000082E19FE00E949A4D40E150E0B80182E1AE
:106A10009FE00E94504D6EE178E082E19FE00E948D
:106A20009A4DAE014B5D5F4F61E070E0802F0E9498
:106A30004D518DA10E94AC586EEB79E082E19FE050
:106A40000E94CD6A0F5F1F4F0A331105B9F6A99650
:106A50000FB6F894DEBF0FBECDBFDF91CF911F916F
:106A60000F91FF90EF90DF90CF90BF90AF909F90ED
:106A70007F906F905F904F9008954F925F926F92CA
:106A80007F929F92AF92BF92CF92DF92EF92FF924E
:106A90000F931F93CF93DF93CDB7DEB7A8970FB6B1
:106AA000F894DEBF0FBECDBF6EE478E0CE01019654
:106AB0000E94634CBE016F5F7F4F8BE392E10E94A7
:106AC0001F85182FCE0101960E94FF4B112309F458
:106AD000E6C08091451290914612409718F080E0F0
:106AE0000C94D23E42E050E061E472E1CE010196A6
:106AF0000E94343FBE016F5F7F4F8DE192E10E94A3
:106B00001C4BCE0101960E94FF4B6DE172E1CE015C
:106B100001960E945B4CCE0101960E94938FCE019C
:106B200001960E94FF4B8DE192E10E943F4A20E0D6
:106B300030E048EC52E40E941DAF0E94A7B1AB01C7
:106B4000BC0140934302509344026093450270930A
:106B50004602CE0101960E94A06ACE0101960E94D3
:106B6000938FCE0101960E94FF4B6091430270917A
:106B7000440280914502909146028B019C0100598C
:106B80001F452140310901341C4921053105D0F050
:106B900061E278E0CE0101960E94634C6DE172E102
:106BA000CE0101960E947F4B64E378E00E94684B1F
:106BB000BC0183E292E10E94EA4BCE0101960E9461
:106BC000FF4B4EC01A821982FE01339626E0DF0188
:106BD0001D922A95E9F70E94BEAE20E030E048EC15
:106BE00052E40E940EB18E010F5F1F4F22E047E07A
:106BF0000E9428AABC0183E292E10E94D54B64E482
:106C000078E0CE0145960E94634C63E272E1CE01CA
:106C100045960E947F4B61E578E00E94684BBC017D
:106C200083E292E10E94EA4BCE0145960E94FF4B1F
:106C300010923C0C10923B0C8091430290914402C4
:106C4000A0914502B091460280938E1090938F10D0
:106C5000A0939010B093911080E090E00E94A26EFB
:106C600061E179E0CE0101960E94634C63E272E13A
:106C7000CE0101960E947F4BBC01CE0145960E9439
:106C80005B4CCE0145960E942971CE0145960E942B
:106C9000FF4BCE0101960E94FF4B0C94CF3E66E560
:106CA00078E0CE0101960E94634CBE016F5F7F4F7A
:106CB0008BE392E10E941F85182FCE0101960E945E
:106CC000FF4B1123C9F126E030E044E050E061E4DD
:106CD00072E1CE0101960E94774CBE016F5F7F4F3B
:106CE0008DE192E10E941C4BCE0101960E94FF4B68
:106CF0008DE192E10E944A4A709307116093061158
:106D000070932A026093290261E472E1CE01019638
:106D10000E945B4CCE0101960E94938FCE0101969A
:106D20000E94FF4B10923C0C10923B0C80E090E0D4
:106D30000E94A26E0C94CF3E6BE578E0CE010196E6
:106D40000E94634CBE016F5F7F4F8BE392E10E9414
:106D50001F85182FCE0101960E94FF4B112309F4C5
:106D600011C10AE010E0C12CD12C7601AA24AA940A
:106D700043E0B42E6EE170E080E090E00E942F8648
:106D8000809161020E94E585B5010E9483B3072EC0
:106D9000000C880B990B0E94BEAE20E030E040EA68
:106DA00050E40E941DAF9B01AC01C701B6010E94D7
:106DB00048B06B017C0101501109E1F620E030E0A0
:106DC00040E251E40E940EB16B017C016EE578E077
:106DD000CE0101960E94634CBE016F5F7F4F8BE333
:106DE00092E10E941F85182FCE0101960E94FF4B51
:106DF000112309F446C020E030E040E650E4C7012A
:106E0000B6010E941DAF9B01AC0160E070E080E81C
:106E100090E40E9447B060931D0270931E0280931D
:106E20001F029093200260EC7CE083E292E10E94DA
:106E3000904B40911D0250911E0260911F02709173
:106E4000200222E0CE0101960E94044CBE016F5F39
:106E50007F4F83E292E10E94164BCE0101960E9481
:106E6000FF4B80911D0290911E02A0911F02B091D4
:106E700020028093B2109093B310A093B410B093FB
:106E8000B51062E678E0CE0101960E94634CBE0127
:106E90006F5F7F4F8BE392E10E941F85182FCE0119
:106EA00001960E94FF4B112309F44EC020E030E010
:106EB00040E650E4C701B6010E941DAF9B01AC0142
:106EC00060E070E080E291E40E9447B060931902B4
:106ED00070931A0280931B0290931C026FEA7CE06D
:106EE00083E292E10E94904B4091190250911A0264
:106EF00060911B0270911C0222E0CE0101960E945B
:106F0000044CBE016F5F7F4F83E292E10E94164BFB
:106F1000CE0101960E94FF4B8091190290911A02B6
:106F2000A0911B02B0911C028093B6109093B710F1
:106F3000A093B810B093B91010923C0C10923B0C77
:106F400080E090E00E94A26E61E179E0CE010196BE
:106F50000E94634C63E272E1CE0101960E947F4B76
:106F6000BC01CE0145960E945B4CCE0145960E9425
:106F70002971CE0145960E94FF4BCE0101960E94D9
:106F8000FF4B0FC767E678E0CE0101960E94634C85
:106F9000BE016F5F7F4F8BE392E10E941F85182F28
:106FA000CE0101960E94FF4B112309F4BEC08091CF
:106FB0004512909146120797F0F046E050E061E4E8
:106FC00072E1CE01019650D7BE016F5F7F4F8DE118
:106FD00092E10E941C4BCE0101960E94FF4B8DE175
:106FE00092E10E943F4A60932502709326028093AB
:106FF00027029093280280915F0290916002992766
:107000000E94E478BC01990F880B990B0E94BEAED8
:107010002DE038E643E55BE30E941DAF6B017C0188
:107020002091830230918402409185025091860222
:107030000E94B8AE18164CF060916B0270916C0211
:1070400080916D0290916E021BC020919702309149
:1070500098024091990250919A02C701B6010E948C
:10706000FDB187FF05C0C701B6010E94106D08C0C1
:1070700060917F02709180028091810290918202E2
:1070800020E030E048EC52E40E941DAF6B017C012F
:1070900020E030E0A9010E94B8AE181634F0C12CEF
:1070A000D12C38EAE32E31E4F32EC0922502D0929F
:1070B0002602E0922702F0922802C092C210D092DB
:1070C000C310E092C410F092C51080919A138823E7
:1070D00081F06DE97CE082E19FE00E94CF4C6091FD
:1070E00025027091260280912702909128020E9429
:1070F000105210923C0C10923B0C80E090E00E94E9
:10710000A26E63E97CE083E292E10E94904B4091A1
:10711000250250912602609127027091280222E0F8
:10712000CE0101960E94044C4AC26DE678E0CE0181
:1071300001960E94634CBE016F5F7F4F8BE392E12B
:107140000E941F85182FCE0101960E94FF4B11232C
:1071500009F46EC0B0905D0260E08B2D0E94A9859D
:1071600009E110E0C12CD12C76018B2D0E94E58520
:10717000BC01990F880B990B0E94BEAE9B01AC011C
:10718000C701B6010E9448B06B017C016AE070E063
:1071900080E090E00E942F860150110931F720E035
:1071A00030E040EA50E4C701B6010E941DAF20E084
:1071B00030EC4FE754E40E940EB120E030E048ECA0
:1071C00051E40E940EB160932102709322028093D9
:1071D0002302909324026093D8107093D910809367
:1071E000DA109093DB1010923C0C10923B0C80E074
:1071F00090E00E94A26E60E87CE083E292E10E944F
:10720000904B409121025091220260912302709193
:10721000240222E0CE0101960E94044CBE016F5F61
:107220007F4FCE0145960E945B4C6DEC75E05AC0D5
:1072300061E778E0CE0101960E94634CBE016F5F6A
:107240007F4F8BE392E10E941F85182FCE0101969C
:107250000E94FF4B112309F45AC08091BD10082EE3
:10726000000C990B0197039708F04AC089E390E05E
:107270000E94E478BC01990F880B990B0E94BEAE66
:107280002AE137E64CE950E40E941DAF6093BE103E
:107290007093BF108093C0109093C11010923C0C5B
:1072A00010923B0C80E090E00E94A26E6FE57CE0C3
:1072B00083E292E10E94904B4091BE105091BF102A
:1072C0006091C0107091C11022E0CE0101960E9421
:1072D000044CBE016F5F7F4FCE0145960E945B4C10
:1072E00067E778E0CE0145960E94684BBC0183E2D7
:1072F00092E10E94164BCE0145960E94FF4B66C15B
:1073000069E37CE083E292E10E94904B3AC56AE730
:1073100078E0CE0101960E94634CBE016F5F7F4F03
:107320008BE392E10E941F85182FCE0101960E94E7
:10733000FF4B112309F44DC126E030E044E050E05A
:1073400061E472E1CE0101960E94774CBE016F5F4D
:107350007F4F8DE192E10E941C4BCE0101960E946D
:10736000FF4B8DE192E10E944A4A6B017C015B0177
:1073700063ED7AE0CE0101960E94634CBE016F5F1F
:107380007F4F81E492E10E94CF848E010B5E1F4FFC
:10739000AC014F5F5F4F61E472E1C80165D5B80190
:1073A0008DE192E10E941C4BC8010E94FF4BCE016F
:1073B00001960E94FF4B90905B028DE192E10E944A
:1073C0003F4A2B013C0180919A138823B9F062E572
:1073D0007BE082E19FE00E94CF4C4AE050E0B601A2
:1073E00082E19FE00E94504D69ED7BE082E19FE0E9
:1073F0000E949A4DC301B2010E941052692DC8012A
:107400000E94415718870F831D821E82198289E0CE
:107410008A8381E08B838C831C8A1B8ACE01019630
:107420000E944E54CE0101960E94E253CE01019675
:107430000E9413530E8110E00B30110514F00AE086
:1074400010E0BBE5CB16D10408F44CC023E1C22EFA
:107450002CE0D22E5601412C512C3201E12CF12C82
:10746000E016F106BCF46E2DCE0101960E94A452E6
:107470009B01AC01F50161937193819391935F013D
:10748000C301B2010E9448B02B013C01FFEFEF1A8B
:10749000FF0AE6CFB801012E000C880B990B0E9461
:1074A000BEAE9B01AC01C301B2010E940EB12B0123
:1074B0003C01E12CF12CE016F1060CF05AC0D6018B
:1074C0002D913D914D915C91C301B2010E9447B055
:1074D000F60161937193819391936F01FFEFEF1A1E
:1074E000FF0AE9CF1A141B0424F50A151B0524F022
:1074F00041E0C41AD10804C0680181E0C81AD1086B
:107500006C2DCE0101960E94A4529B01AC01860114
:10751000000F111F000F111F0D5E134FC301B201A9
:107520000E9447B0D8016D937D938D939C931397E0
:1075300020C0AB28F1F483E1C82E8CE0D82EE12CDA
:10754000F12CE016F106ACF46E2DCE0101960E94EE
:10755000A4529B01AC01C301B2010E9447B0F601E5
:1075600061937193819391936F01FFEFEF1AFF0A7B
:10757000E8CFE3E1FCE0ACEDB0E18BE39CE04191CE
:107580005191619171914D935D936D937D938E17A0
:107590009F07A9F710923C0C10923B0C80E090E002
:1075A0000E94A26E68E17CE083E292E10E94904B2F
:1075B00044E050E061E472E1CE01019655D4BE0191
:1075C0006F5F7F4F83E292E10E94164BCE010196DE
:1075D000D6C36EE778E0CE0101960E94634CBE01EF
:1075E0006F5F7F4F8BE392E10E941F85182FCE01C2
:1075F00001960E94FF4B112309F424C127E030E0DB
:1076000046E050E061E472E1CE0101960E94774CC1
:10761000BE016F5F7F4F8DE192E10E941C4BCE0156
:1076200001960E94FF4B8DE192E10E944A4A8B0134
:107630006093BD1081E492E10E94554A69ED7BE0C0
:10764000CE0101960E94634CBE016F5F7F4F81E4C3
:1076500092E10E94CF84AC014F5F5F4F61E472E121
:10766000CE01459601D4CE0145960E943F4A6093D3
:10767000BE107093BF108093C0109093C110CE01C4
:1076800045960E94FF4BCE0101960E94FF4B67E09A
:107690007CE083E292E10E94904B0430110594F467
:1076A000023011050CF05BC001151105B1F001307D
:1076B000110509F09BC069EF7BE083E292E10E9433
:1076C000C64A77C00430110509F090C066EE7BE031
:1076D00083E292E10E94C64AACC020E030E0A901FA
:1076E0006091BE107091BF108091C0109091C11038
:1076F0000E94B8AE181664F080E090E0A0E8BFE306
:107700008093BE109093BF10A093C010B093C1108F
:107710002091BE103091BF104091C0105091C11007
:1077200060E070E080EA90E40E940EB1AB01BC0121
:1077300022E0CE0145960E94044C65E878E0CE0137
:1077400001960E94634CBE016B5E7F4FCE01019695
:107750000E947F4B64ED78E00E94684B5DC06DEE47
:107760007BE083E292E10E94C64A8AE0809FB001FA
:10777000819F700D1124CE0101960E948950BE0197
:107780006F5F7F4FCE0145960E945B4C6DEC78E0B9
:10779000CE0145960E94684BBC0183E292E10E94B3
:1077A000164BCE0145960E94FF4BCE0101960E94DA
:1077B000FF4B20E030E048E453E46091BE1070914C
:1077C000BF108091C0109091C1100E94B8AE1816E1
:1077D00084F180E090E4ACE1B5E48093BE10909336
:1077E000BF10A093C010B093C11023C06091BD1012
:1077F000062E000C770BCE0145960E94895060E959
:1078000078E0CE0101960E94634CBE016B5E7F4F13
:10781000CE0101960E947F4BBC0183E292E10E945F
:10782000164BCE0101960E94FF4BCE0145960E9459
:10783000FF4B10923C0C10923B0C80E090E00E94B9
:10784000A26E9FC267E978E0CE0101960E94634C68
:10785000BE016F5F7F4F8BE392E10E941F85182F5F
:10786000CE0101960E94FF4B112309F4CEC027E000
:1078700030E046E050E061E472E1CE0101960E9402
:10788000774CBE016F5F7F4F8DE192E10E941C4BF0
:10789000CE0101960E94FF4B8DE192E10E944A4A7F
:1078A0006093BA1081E492E10E94554A8DE192E121
:1078B0000E944A4A611571058105910519F485E018
:1078C00090E007C0613071058105910539F489E1C7
:1078D00090E09093BC108093BB1025C069ED7BE0D5
:1078E000CE0101960E94634CBE016F5F7F4F81E421
:1078F00092E10E94CF84AC014F5F5F4F61E472E17F
:10790000CE014596B1D2CE0145960E944A4A709367
:10791000BC106093BB10CE0145960E94FF4BCE0178
:1079200001960E94FF4B10923C0C10923B0C80E0A1
:1079300090E00E94A26E65ED7BE083E292E10E94FE
:10794000904B8091BA10833044F56AEC7BE083E27F
:1079500092E10E94C64A6091BB107091BC10CE01AA
:1079600001960E948950BE016F5F7F4FCE01459600
:107970000E945B4C63EB7BE0CE0145960E94684B16
:10798000BC0183E292E10E94164BCE0145960E9413
:10799000FF4BCE0101960E94FF4B8091BA108330BD
:1079A0000CF4EFC16091BB107091BC10CE018396B6
:1079B0000E9489506091BA10062E000C770BCE0100
:1079C00045960E94895060E978E0CE0101960E94B8
:1079D000634CBE016B5E7F4FCE0101960E947F4BD0
:1079E000BE016D5D7F4F0E947F4BBC0183E292E13F
:1079F0000E94164BCE0101960E94FF4BCE01459688
:107A00000E94FF4BCE018396BAC16EE978E0CE01A9
:107A100001960E94634CBE016F5F7F4F8BE392E142
:107A20000E941F85182FCE0101960E94FF4B112343
:107A300009F456C08091590290915A020E94DD7952
:107A400060932B0270932C0280932D0290932E0250
:107A50006093A6107093A7108093A8109093A9101C
:107A600080E090E5A3ECB7E4809333029093340276
:107A7000A0933502B093360280939E1090939F108E
:107A8000A093A010B093A11080919A13882381F045
:107A90006CEA7BE082E19FE00E94CF4C60912B0278
:107AA00070912C0280912D0290912E020E94105212
:107AB00010923C0C10923B0C80E090E00E94A26E71
:107AC00040912B0250912C0260912D0270912E0258
:107AD00022E0CE0145960E94044C62EA78E039C16A
:107AE0006DEA78E0CE0101960E94634CBE016F5FA3
:107AF0007F4F8BE392E10E941F85182FCE010196E4
:107B00000E94FF4B112309F484C08091451290918B
:107B100046120497F0F044E050E061E472E1CE01D7
:107B20000196A2D1BE016F5F7F4F8DE192E10E946D
:107B30001C4BCE0101960E94FF4B8DE192E10E9409
:107B40003F4A6093370270933802809339029093D2
:107B50003A028091370290913802A0913902B09197
:107B60003A0280939A1090939B10A0939C10B0932C
:107B70009D1080919A13882389F063E97BE082E16C
:107B80009FE00E94CF4C6091370270913802809143
:107B9000390290913A0242E00E94116B80915902A1
:107BA00090915A020E94DD7960932F027093300207
:107BB00080933102909332026093A2107093A310CD
:107BC0008093A4109093A51080919A13882381F03C
:107BD00069E87BE082E19FE00E94CF4C60912F0238
:107BE0007091300280913102909132020E941052C5
:107BF00010923C0C10923B0C80E090E00E94A26E30
:107C000040912F0250913002609131027091320206
:107C100099C069EB78E0CE0101960E94634CBE01E9
:107C20006F5F7F4F8BE392E10E941F85182FCE017B
:107C300001960E94FF4B112311F40C946F35809133
:107C40004512909146120497F0F044E050E061E450
:107C500072E1CE01019608D1BE016F5F7F4F8DE1C9
:107C600092E10E941C4BCE0101960E94FF4B8DE1D8
:107C700092E10E943F4A60933302709334028093F2
:107C80003502909336028091330290913402A09194
:107C90003502B091360280939E1090939F10A0936E
:107CA000A010B093A11080919A13882389F060E707
:107CB0007BE082E19FE00E94CF4C609133027091A3
:107CC0003402809135029091360242E00E94116B9D
:107CD0008091590290915A020E94DD7960932B02A3
:107CE00070932C0280932D0290932E026093A61025
:107CF0007093A7108093A8109093A91080919A1365
:107D0000882381F066E67BE082E19FE00E94CF4C11
:107D100060912B0270912C0280912D0290912E0285
:107D20000E94105210923C0C10923B0C80E090E0AC
:107D30000E94A26E40912B0250912C0260912D0264
:107D400070912E0222E0CE0145960E94044C61EB18
:107D500078E0CE0101960E94634CBE016B5E7F4FBE
:107D6000CE0101960E947F4BBC0183E292E10E940A
:107D7000EA4BCE0101960E94FF4BCE0145960E9430
:107D8000FF4B63E272E1CE0101960E945B4CCE0193
:107D900001960E942971CE0101960E94FF4B10921C
:107DA000540281E0A8960FB6F894DEBF0FBECDBF97
:107DB000DF91CF911F910F91FF90EF90DF90CF90C7
:107DC000BF90AF909F907F906F905F904F9008957D
:107DD000089580912E058823F9F080912D05882340
:107DE000D9F081E00E94646A8BE39FE10197F1F78B
:107DF00060E080E00E94756A6CE97DE084E293E1D6
:107E00000E94CF4C61E080E00E94756A6CE87DE0E2
:107E100084E293E10C94CF4C089580912E05882341
:107E200049F080912D05882329F060E084E293E1F8
:107E30000C9495570895FF920F931F93CF93DF9360
:107E4000EC01F62E08811981C8010E94D4AFF81602
:107E500021F06F2DC8010E94DCAFCE01DF91CF91E0
:107E60001F910F91FF900895CF93DF93EC01FB01D9
:107E7000248135810E94774CCE01DF91CF91089506
:107E80003F924F925F926F927F928F929F92AF92AA
:107E9000BF92CF92DF92EF92FF920F931F93CF93F7
:107EA000DF93CDB7DEB7E4970FB6F894DEBF0FBE11
:107EB000CDBF80914713882319F0109247134CC30C
:107EC00081E0809347136EEB79E0CE0185960E94A6
:107ED000634C6EEB79E0CE018B960E94634C00E020
:107EE00010E082E0382E98EEC92E93E0D92EE12CD6
:107EF000F12CF8013197E031F10530F48827E8568C
:107F0000FF4F8F4F0C9496B36EEB79E0CE018596C0
:107F10000E94D54B8091041190910511892B31F469
:107F200069E077E0CE0185960E94D54B80910411DF
:107F300090910511019731F46DE077E0CE018596BF
:107F40000E94D54B8091041190910511029731F454
:107F500063E177E0CE0185960E94D54B89A59AA56D
:107F6000892B31F068E173E1CE0185960E94164BB2
:107F70006DEB78E0CE0101960E94634C62E173E103
:107F8000CE0101960E947F4BBC01CE018B960E94D0
:107F9000EA4BCE0101960E94FF4B80910411909113
:107FA0000511019709F03BC2BE016B5D7F4FCE0109
:107FB00001960E945B4C48EC50E06FEF7FEFCE01E2
:107FC00001960E94BF8FCE0101960E94FF4BBE0119
:107FD000655D7F4FCE0101960E945B4C40ED57E0FE
:107FE0006FEF7FEFCE0101960E94778DCE01019653
:107FF0000E94FF4BCE0101960E94E8608D819E8118
:108000000097A1F0E981FA812081222379F0079776
:1080100068F065E77FE0CE0185960E94904BBE0137
:108020006F5F7F4FCE018B960E94EA4BCE01019687
:1080300096C069E67FE0CE0185960E94904B0E9433
:108040008B874B015C010E948B87A70196010E94E0
:1080500016B0CA01B90120E831E541E050E00E94C4
:1080600016B020E13EE040E050E00E94EAAF29ABCC
:108070003AAB4BAB5CAB2CE330E040E050E00E940D
:10808000EAAF29013A01AB01BC01CE0101960E9481
:10809000A06AB301A201CE0107960E94A06A49A975
:1080A0005AA96BA97CA9CE010D960E94A06AC501B0
:1080B000B40120E03CE546E255E00E9416B0BA016A
:1080C000A901CE0149960E94A06ABE01675E7F4F5A
:1080D000CE0143960E945B4C62EC78E0CE01439661
:1080E0000E94684BBE01635F7F4F0E947F4B65EC2F
:1080F00078E00E94684BBE01695F7F4F0E947F4B12
:1081000068EC78E00E94684BBE016F5F7F4F0E9471
:108110007F4B6BED75E00E94684BBC01CE014F9622
:108120000E945B4CCE0143960E94FF4BCE014996C4
:108130000E94FF4BCE010D960E94FF4BCE01079689
:108140000E94FF4BCE0101960E94FF4BBE01615E73
:108150007F4FCE018B960E941C4BCE014F960E9402
:10816000FF4B5DC18091110C9091120C019719F495
:108170006AE57FE002C06CE47FE0CE0185960E9454
:10818000904B6CE37FE047C16CE27FE0CE018596C7
:108190000E94904B6FE17FE03EC162E17FE0CE0143
:1081A00085960E94904B67E07FE035C16BEF7EE0E3
:1081B000CE0185960E94904B6AEE7EE02CC18091A4
:1081C000110C9091120C039719F46FED7EE002C030
:1081D00065ED7EE0CE0185960E94904B6AEC7EE0D4
:1081E0001AC16DEB7EE0CE0185960E94904B6EEA3F
:1081F0007EE011C163EA7EE0CE0185960E94904B3D
:108200006091BB107091BC10CE0107960E948950FE
:1082100062EE7BE0CE0101960E94634CBE01695F75
:108220007F4FCE0101960E947F4B63EB7BE00E9463
:10823000684BBC01CE0185960E94164BCE0101967B
:108240000E94FF4BCE0107960E94FF4B66E97EE03D
:10825000E2C08091110C9091120C029719F465E81C
:108260007EE002C065E77EE0CE0185960E94904BDD
:1082700068E67EE0D0C06CE57EE0CE0185960E9487
:10828000904B6CE47EE0C7C061E47EE0CE01859651
:108290000E94904B67E37EE0BEC06BE27EE0CE01C1
:1082A00085960E94904B6BE17EE0B5C0B090BD100A
:1082B00060E17EE0CE0185960E94904B83E08B15B5
:1082C00074F092E0B9160CF045C0BB2081F081E05B
:1082D000B81261C06BEC78E0CE01859659C094E08D
:1082E000B91259C06FEC78E083E292E151C08090FE
:1082F000BE109090BF10A090C010B090C11020E0B0
:1083000030E048E452E4C501B4010E94B8AE87FFF2
:1083100002C033243394A501940160E070E080EA48
:1083200090E40E940EB1AB01BC01232DCE01079653
:108330000E94044C69EF78E0CE0101960E94634CE4
:10834000BE01695F7F4FCE0101960E947F4B64EDB5
:1083500078E018C08B2D9AE08902B0011124CE017B
:1083600007960E94895062EE7BE0CE0101960E9442
:10837000634CBE01695F7F4FCE0101960E947F4B27
:108380006DEC78E00E94684BBC01CE0185961CC064
:108390000E94084B23C06091BD10062E000C770B85
:1083A000CE0107960E94895066E97AE0CE010196D7
:1083B0000E94634CBE01695F7F4FCE0101960E940F
:1083C0007F4BBC0183E292E10E94164BCE010196E5
:1083D0000E94FF4BCE0107960E94FF4B60E07EE0BB
:1083E0001AC063EF7DE0CE0185960E94904B63EE4C
:1083F0007DE011C067ED7DE0CE0185960E94904B37
:1084000068EC7DE008C06CEB7DE0CE0185960E94B3
:10841000904B6CEA7DE0CE018B960E94904BBE01A2
:108420006B5D7F4FCE0101960E945B4C48EC50E0A3
:108430006FEF7FEFCE0101960E946490CE0101960E
:108440000E94FF4BBE01655D7F4FCE0101960E94E9
:108450005B4C48EC50E06FEF7FEFCE0101960E943D
:10846000778DCE0101960E94FF4B0E94FE97982EB9
:10847000A12CB12C91106DC08FEFA81AB80A95E607
:10848000A916B10451F00E94FE97982E64E170E0A5
:1084900080E090E00E942F86EDCF6EEB79E081E4E2
:1084A00092E10E94D54BCE0101960E94A274BE01BA
:1084B0006F5F7F4F81E492E10E941C4BCE010196D9
:1084C0000E94FF4B8091451290914612892B89F4AE
:1084D00061E070E0CE0101960E94338BBE016F5FB8
:1084E0007F4F81E492E10E941C4BCE0101960E94D5
:1084F000FF4B8091451290914612892B89F461E0DF
:1085000070E0CE0101960E94D189BE016F5F7F4F5E
:1085100081E492E10E941C4BCE0101960E94FF4B28
:108520008091451290914612892B51F48091471306
:10853000882331F00F5F1F4F0131110509F0D9CCAD
:10854000CE018B960E94FF4BCE0185960E94FF4B79
:1085500003C010924713F4CFE4960FB6F894DEBF31
:108560000FBECDBFDF91CF911F910F91FF90EF9084
:10857000DF90CF90BF90AF909F908F907F906F9043
:108580005F904F903F9008954F925F926F927F92CD
:108590008F929F92AF92BF92CF92DF92EF92FF9213
:1085A0000F931F93CF93DF93CDB7DEB7C654D10996
:1085B0000FB6F894DEBF0FBECDBF8C016EEB79E035
:1085C000CE01C7960E94634C6EEB79E0CE01CD964A
:1085D0000E94634CBE016F5F7F4F8EE592E154D6DF
:1085E0008D889E88AF88B88C498C5A8C6B8C7C8C1B
:1085F0008D8D9E8DAF8DB8A127968CAF9DAFAEAF00
:10860000BFAF2797C8010197039708F0ADC1A30139
:108610009201C501B40190580E94BBB02BED3FE020
:1086200049EC5FE30E9448B020913F023091400244
:1086300040914102509142020E9448B06B017C017E
:1086400020E030E0A9010E94B8AE87FD09C0C092C9
:10865000500CD092510CE092520CF092530C10C07E
:108660002BED3FE049EC50E4C701B6010E9448B051
:108670006093500C7093510C8093520C9093530C58
:10868000C090500CD090510CE090520CF090530CD4
:108690002BED3FE049EC50E4C701B6010E94FDB16B
:1086A000181684F42BED3FE049EC50E4C701B60105
:1086B0000E9447B06093500C7093510C8093520C01
:1086C0009093530C20E030E044E353E46091500C6D
:1086D0007091510C8091520C9091530C0E941DAFDF
:1086E0002BED3FE049E450E40E940EB160934C0C46
:1086F00070934D0C80934E0C90934F0C0E94A7B139
:10870000CE018B960E94895067ED78E0CE01859668
:108710000E94634CBE01655D7F4FCE018596EFD709
:1087200061EE78E0D5D7BC0189E292E10E94EA4B84
:10873000CE0185960E94FF4BCE018B960E94FF4B87
:10874000C0904C0CD0904D0CE0904E0CF0904F0C23
:1087500020E030E044EB52E4C701B6010E94B8AE1D
:1087600018168CF020E030E040E05FE3C701B6016E
:108770000E9448B00E94A7B1CE018B960E948950FA
:1087800068EE78E022C020E030E044E353E4C70123
:10879000B6010E94B8AE18168CF1A701960160E0F0
:1087A00070E884E393E40E9447B060934C0C7093AC
:1087B0004D0C80934E0C90934F0C0E94A7B1CE01AC
:1087C0008B960E9489506BEE78E0CE0185960E94D0
:1087D000634CBE01655D7F4FCE01859690D7BC018D
:1087E000CE01C796F7D7CE0185960E94FF4BCE01EA
:1087F0008B960E94FF4B69E27BE05DC020E030E099
:1088000047E853E4C701B6010E94B8AE1816FCF061
:1088100020E030E044E353E4C701B6010E9447B0D2
:1088200020E030E040E05FE30E9448B060934C0CF1
:1088300070934D0C80934E0C90934F0C0E94A7B1F7
:10884000CE018B960E9489506BEE78E01EC0A70186
:10885000960160E070E084EB93E40E9447B020E072
:1088600030E040E05FE30E9448B060934C0C7093AE
:108870004D0C80934E0C90934F0C0E94A7B1CE01EB
:108880008B960E94895068EE78E0CE0185960E9412
:10889000634CBE01655D7F4FCE01859630D7BC012C
:1088A000CE01C79697D7CE018596A9D7CE018B96D4
:1088B000A6D76EEE78E0CE01CD9677D7BE01695C83
:1088C0007F4FCE018596F7D74AE050E060E070E038
:1088D000CE0185960E94BF8FCE01859690D70E94CB
:1088E0008B87C0909613D0909713E0909813F090D8
:1088F0009913A4E6CA0ED11CE11CF11CC616D706BA
:10890000E806F90608F4E7C10E948B870E94BCAE16
:108910006B017C016091961370919713809198136D
:10892000909199130E94BEAE20E030E048EC51E4F3
:108930000E9448B09B01AC01C701B6010E94B8AECD
:1089400087FDC9C169ED7BE0CE018596BCD7BE012C
:10895000635C7F4FCE018596D2D6BC01CE01C7960F
:1089600065D6CE0185964BD7C8010297029708F0CD
:108970008EC120E030E040E251E4C501B4010E9424
:108980001DAF6B017C0120E030E040E251E4C30107
:10899000B2010E941DAF4B015C0120E030E040E2DB
:1089A00051E427966CAD7DAD8EAD9FAD27970E94AB
:1089B0001DAF2B013C010E948B872091EC0B309165
:1089C000ED0B4091EE0B5091EF0B621B730B840B80
:1089D000950B0E94BCAE20E030E04AE754E40E94D0
:1089E0000EB1AB01BC0123E0CE018B960DD769EF30
:1089F00078E0CE01859667D7BE01655D7F4FCE01D9
:108A000085967DD66DEF7AE063D6BC0187E192E171
:108A1000E1D6CE018596F3D6CE018B96F0D667E1EE
:108A200072E1CE01859647D769E272E1CE01859663
:108A300066D6BE01695C7F4F62D6BC01CE01C79687
:108A4000C9D6CE018596DBD661E87DE083E292E16E
:108A500067D621E0B701A601CE018596D5D6BE0125
:108A60006B5D7F4F83E292E1E1D5CE018596C7D65B
:108A700021E0B301A201CE01C196C6D621E0B50125
:108A8000A401CE018B96C0D669ED7BE0CE01859620
:108A90001AD7BE01655D7F4FCE01859630D669ED50
:108AA0007BE016D6BE016F5C7F4F29D660EF78E081
:108AB0000FD6BC0183E292E1B9D5CE0185969FD64F
:108AC000CE018B969CD6CE01C19699D6A701960170
:108AD000C701B6010E941DAF6B017C01A501940185
:108AE000C501B4010E941DAF9B01AC01C701B601D5
:108AF0000E9448B06B017C01A3019201C301B20145
:108B00000E941DAF9B01AC01C701B6010E9448B095
:108B10000E9406B36B017C016093480C7093490C72
:108B200080934A0C90934B0C64EF78E083E292E1DF
:108B30006FD521E0B701A601CE01859665D6BE01AD
:108B40006B5D7F4FCE018B96B6D665E079E0CE01A6
:108B50008B96BED5BC0189E292E13CD6CE018B96C4
:108B60004ED6CE0185964BD669E272E183E292E160
:108B70005DD5C090480CD090490CE0904A0CF09024
:108B80004B0C20E030E04AE754E4C701B6010E94F4
:108B9000FDB187FD23C020E030E04AE754E4C7017F
:108BA000B6010E940EB1AB01BC0123E0CE01859657
:108BB0002BD6BE016B5D7F4FCE018B967CD666E0D7
:108BC00079E0CE018B9684D5BC0189E292E102D690
:108BD000CE018B9614D6CE01859611D620E030E6D4
:108BE0004AE656E46091480C7091490C80914A0C19
:108BF00090914B0C0E94B8AEBE01695C7F4F87FF1D
:108C000043C0CE01859657D668EF78E0CE018596B1
:108C10005FD563E272E173D5BC0183E292E1DAD5FC
:108C2000CE018596ECD50330110589F463E272E13B
:108C3000CE01859640D6CE0185960E942971CE013F
:108C40008596DDD56EEB79E083E292E1AED56BEFF0
:108C500078E0CE01859637D669E272E1CE0185963D
:108C60004ED5BC01CE018B9626D64AE050E06FEF80
:108C70007FEFCE018B960E94778DCE018B96BFD56C
:108C8000CE018596BCD503C083E292E1A3D56AE00C
:108C900070E080E090E00E942F86CE01CD96AFD5A7
:108CA000CE01C796ACD5CA5BDF4F0FB6F894DEBFD6
:108CB0000FBECDBFDF91CF911F910F91FF90EF902D
:108CC000DF90CF90BF90AF909F908F907F906F90EC
:108CD0005F904F9008956EEB79E0CE018596F3D5C5
:108CE000CE0185960E94F38DCE01859688D5BE0172
:108CF000635C7F4F84E293E144D624CE1F93CF93ED
:108D0000DF93CDB7DEB7A8970FB6F894DEBF0FBEDE
:108D1000CDBF182F0E9457508EE10E945A6A62E020
:108D20008FEA9FE00E94515660E08FEA9FE00E9428
:108D300051560E94536A8EE10E945A6A61E08FEA9E
:108D40009FE00E94515660E28FEA9FE00E945156D8
:108D50000E94536A80E290E09093621280936112C5
:108D600080E090E8A9E8B4E48093670290936802F9
:108D7000A0936902B0936A0280E090E0A5E7B4E4B2
:108D80008093630290936402A0936502B09366029D
:108D9000BE016F5F7F4F8EE592E129D2112309F466
:108DA0007CC066E57DE082E19FE0F9D582E19FE04D
:108DB0000E94E26966E47DE082E19FE0F0D5BE01B9
:108DC0006F5F7F4F82E19FE00E94CD6A66E37DE0A6
:108DD00082E19FE0E4D56D857E858F8598890E942C
:108DE000DE6A66E27DE082E19FE0D9D569897A8911
:108DF0008B899C890E94DE6A66E17DE082E19FE0CA
:108E0000CED520E030E040E251E4698D7A8D8B8D43
:108E10009C8D0E941DAF42E00E94116B64E079E0DE
:108E200082E19FE00E94CD6A66E07DE082E19FE002
:108E3000B6D520E030E040E251E46D8D7E8D8F8D1F
:108E400098A10E941DAF42E00E94116B64E079E09E
:108E500082E19FE00E94CD6A66EF7CE082E19FE0C4
:108E60009ED520E030E040E251E469A17AA18BA1D7
:108E70009CA10E941DAF42E00E94116B64E079E06A
:108E800082E19FE00E94CD6A60ED7CE082E19FE09C
:108E900086D582E19FE00E94E26964EF71E080E0A4
:108EA00090E00E942F86A8960FB6F894DEBF0FBE02
:108EB000CDBFDF91CF911F9108950895CF92DF929A
:108EC000EF92FF920F931F93CF93DF936C017A0180
:108ED0008B01C0E0D0E0CE15DF0581F0D8016D91A7
:108EE0008D01D601ED91FC910190F081E02DC6013C
:108EF0001995892B11F02196EECF7E01C701DF91E4
:108F0000CF911F910F91FF90EF90DF90CF90089538
:108F1000FC01538D448D252F30E0842F90E0821B7F
:108F2000930B541710F0CF96089501970895FC0104
:108F3000918D828D981761F0828DDF01A80FB11D90
:108F40005D968C91928D9F5F9F73928F90E00895B4
:108F50008FEF9FEF0895FC01918D828D981731F06E
:108F6000828DE80FF11D858D90E008958FEF9FEFC2
:108F70000895FC01918D228D892F90E0805C9F4F98
:108F8000821B91098F73992708958BE39DE0F1DF90
:108F900021E0892B09F420E0822F089588ED9DE0DF
:108FA000E8DF21E0892B09F420E0822F089585E78E
:108FB0009EE0DFDF21E0892B09F420E0822F089575
:108FC00082E19FE0D6DF21E0892B09F420E0822FA7
:108FD0000895FC01848DDF01A80FB11DA35ABF4F76
:108FE0002C91848D90E001968F739927848FA689A8
:108FF000B7892C93A089B1898C91837080648C93FC
:10900000938D848D981306C00288F389E02D8081AA
:109010008F7D80830895EF92FF920F931F93CF93DC
:10902000DF93EC0181E0888F9B8D8C8D981305C0B8
:10903000E889F989808185FD25C0F62E0B8D10E029
:109040000F5F1F4F0F731127E02E8C8DE8120BC09E
:109050000FB607FCFACFE889F989808185FFF5CF43
:10906000CE01B7DFF2CF8B8DFE01E80FF11DE35A81
:10907000FF4FF0829FB7F8940B8FEA89FB898081BC
:1090800080620AC09FB7F894EE89FF896083E889FF
:10909000F98980818370806480839FBF81E090E044
:1090A000DF91CF911F910F91FF90EF900895CF9393
:1090B000DF93EC01888D8823C1F0EA89FB898081E8
:1090C00085FD05C0A889B9898C9186FD0EC00FB6B3
:1090D00007FCF5CF808185FFF2CFA889B9898C91F3
:1090E00085FFEDCFCE0175DFE8CFDF91CF910895F9
:1090F00080E090E0892B19F063DF811116C080E0D9
:1091000090E0892B19F053DF811112C080E090E0CC
:10911000892B19F043DF81110EC080E090E0892B8C
:1091200079F033DF81110AC008950E940000E7CF73
:109130000E940000EBCF0E940000EFCF0C940000D3
:1091400008950E94D6B50F931F93CF93DF93EC0140
:1091500088819981009729F02A813B81261737075A
:1091600088F48B016F5F7F4F0E94F6B4009761F027
:10917000998388831B830A832C813D81232B11F4DF
:10918000FC01108281E001C080E0DF91CF911F914E
:109190000F910895EF92FF920F931F93CF93DF9358
:1091A0006115710511F480E01BC041155105B9F03E
:1091B0007B01EC018C819D818A01080F191FB80188
:1091C000CE01C1DF882379F3288139818C819D818B
:1091D000B701820F931F0E940DB61D830C8381E09F
:1091E000DF91CF911F910F91FF90EF9008950F9312
:1091F0001F93CF93DF938C01EB0188E2FB01119267
:109200008A95E9F74BE050E068E079E0CE010E94F2
:1092100022B61B8681E090E0A0E0B0E08C879D87BD
:10922000AE87BF87F80185899689A789B08D888B1D
:10923000998BAA8BBB8B82E090E0A0E0B0E08C8B96
:109240009D8BAE8BBF8B1CA21DA21EA21FA280E015
:1092500090E0A8E4B4E4888F998FAA8FBB8F80E058
:1092600090E0A8E4B4EC8C8F9D8FAE8FBF8F8DEC17
:109270009CECACE4BEE388A399A3AAA3BBA3DF91B3
:10928000CF911F910F9108954F925F926F927F92AD
:109290008F929F92AF92BF92CF92DF92EF92FF9206
:1092A0000F931F93CF93DF938C01EB0184E2FB01BB
:1092B00011928A95E9F78EE10E945A6A83E090E064
:1092C0000E94556A0E94536A66E08EE14DD78091F4
:1092D000701390E020917113821B910986309105E3
:1092E000ECF38FEA9FE00E940956882E8FEA9FE0F8
:1092F0000E940956982E8FEA9FE00E940956682E18
:109300008FEA9FE00E940956782E8FEA9FE00E9424
:109310000956482E8FEA9FE00E940956582EB82C15
:10932000A12CB5016929072E000C880B990B0E940E
:10933000BEAE4B015C01F80165837683878390871D
:10934000D42CC12CB6016529072E000C880B990B73
:109350000E94BEAEF8016187728783879487F62CDE
:10936000E12CB7016729072E000C880B990B0E948E
:10937000BEAEF801658776878787908B118A128A3F
:10938000138A148A84E290E0A0E0B0E08883998395
:10939000AA83BB8385899689A789B08D8C839D8399
:1093A000AE83BF8382E090E0A0E0B0E08887998739
:1093B000AA87BB87188A198A1A8A1B8AC0906702F3
:1093C000D0906802E0906902F0906A02A7019601CD
:1093D000C501B4010E940EB120E030E048EC52E437
:1093E0000E941DAF6C8B7D8B8E8B9F8BA70196018E
:1093F000F80161857285838594850E940EB120E015
:1094000030E048EC52E40E941DAF688F798F8A8F5C
:109410009B8F2091630230916402409165025091CC
:109420006602F80165857685878590890E940EB170
:1094300020E030E048EC52E40E941DAF6C8F7D8F3D
:109440008E8F9F8F81E0DF91CF911F910F91FF90C1
:10945000EF90DF90CF90BF90AF909F908F907F90D4
:109460006F905F904F900895862F0C945385862FB0
:10947000642F0C947B85862F642F0C94A985FC01A6
:1094800080819181009711F00C9447AA60E070E010
:10949000CB010895FC0180819181009711F00C941B
:1094A0004AAA60E070E0CB010895AF92BF92CF92DC
:1094B000DF92EF92FF920F931F93CF93DF93DC0124
:1094C000CD90DC901197C114D10409F443C01496D7
:1094D000CD91DC9115972097E9F18C017601570128
:1094E000BFEFAB1ABB0AF7018081082E000C990B65
:1094F0000E9488AE892B11F07501F1CF2197CC0D18
:10950000DD1D8881082E000C990B0E9488AE892BE6
:1095100029F0CE15DF0510F02197F3CFAE014F5F94
:109520005F4F4E195F09D80115965C934E931497BF
:10953000CE14DF0420F4B701C6010E94FBB5D801A8
:10954000ED91FC91119714968D919C911597E80FD0
:10955000F91F1082DF91CF911F910F91FF90EF9033
:10956000DF90CF90BF90AF900895FC0124813581AA
:109570006217730748F480819181009729F0FC01FC
:10958000E60FF71F8081089580E00895EF92FF9223
:109590000F931F93CF93DF936115710511F480E052
:1095A0001DC08B01EC01CB010E9477AA0097A9F0A6
:1095B0002C813D817C01E20EF31EB701CE01C3DD9B
:1095C000882369F3288139818C819D81B801820FBC
:1095D000931F0E9470AAFD82EC8281E0DF91CF91FF
:1095E0001F910F91FF90EF900895CF93DF931F92FB
:1095F0001F92CDB7DEB769831A8241E050E0BE0109
:109600006F5F7F4FC7DD0F900F90DF91CF9108956F
:109610006115710549F0FB0101900020E9F73197D0
:10962000AF01461B570BB6CD80E00895FB01448186
:10963000558160817181AECD0F931F93CF93DF93DE
:109640008C01EB01FC0180819181009739F06881E8
:10965000798161157105A1F40E946DB488819981A9
:10966000F801918380838A819B81938382838C819B
:109670009D8195838483198218821B821A820FC070
:10968000F801428153812C813D814217530720F319
:109690000E940DB68C819D81F801958384831D8283
:1096A0001C82DF91CF911F910F910895CF93DF938B
:1096B000EC0188819981009711F00E946DB41982A4
:1096C00018821D821C821B821A82DF91CF9108951D
:1096D000CF93DF93EC016115710559F0FB01019007
:1096E0000020E9F73197AF01461B570B53DD81117D
:1096F00002C0CE01DBDFCE01DF91CF910895CF9381
:10970000DF93EC01FB01448155816081718142DD71
:10971000811102C0CE01CADFCE01DF91CF91089541
:10972000EF92FF920F931F93CF93DF93EC018B0186
:109730006115710549F0CB010E9477AA7C01BC013B
:10974000CE0101DD811103C0CE01B0DF07C0FD8273
:10975000EC82B801888199810E9470AACE01DF91C4
:10976000CF911F910F91FF90EF900895EF92FF928C
:109770000F931F93CF93DF93EC017B018A01BA0112
:10978000E2DC811103C0CE0191DF07C01D830C8391
:10979000B701888199810E940DB6CE01DF91CF91EA
:1097A0001F910F91FF90EF900895CF93DF93EC01FD
:1097B0006115710551F0FB0101900020E9F7319727
:1097C000AF01461B570BD2DF01C070DFCE01DF9126
:1097D000CF910895CF93DF93EC01FB018617970794
:1097E00051F0608171816115710521F044815581CD
:1097F000BDDF01C05BDFCE01DF91CF910895FC0199
:10980000808191810C946DB4EF92FF920F931F931E
:10981000CF93DF93CDB7DEB7A1970FB6F894DEBF35
:109820000FBECDBF7C01CB01BA01F70111821082BE
:10983000138212821582148242E0420F8E010F5F62
:109840001F4F0E9428AABC01C701AFDFA1960FB627
:10985000F894DEBF0FBECDBFDF91CF911F910F9166
:10986000FF90EF900895CF93DF931F921F92CDB793
:10987000DEB7FC01118210821382128215821482DB
:1098800069831A82BE016F5F7F4F8FDF0F900F9049
:10989000DF91CF910895FC01118210821382128210
:1098A00015821482C9CEFC011182108213821282A9
:1098B0001582148235CFFC0111821082138212822C
:1098C0001582148287CFFC011182108213821282CA
:1098D000158214826115710549F0FB010190002089
:1098E000E9F73197AF01461B570B40CF0895BF9260
:1098F000CF92DF92EF92FF920F931F93CF93DF935C
:109900007C016B018A01E9012417350720F4812FBE
:109910008901C42FD82F6EEB79E0C701D4DFD601BF
:1099200014968D919C91159708171907C0F48C1700
:109930009D0708F4EC01D601ED91FC911197EC0F15
:10994000FD1FB08010826D917C91600F711FC70167
:109950002CDFD601ED91FC91EC0FFD1FB082C70109
:10996000DF91CF911F910F91FF90EF90DF90CF90FB
:10997000BF900895DC01ED91FC910190F081E02D04
:109980001994DB0114964D915C9115976D917C9122
:10999000DC01ED91FC910280F381E02D1994EF92AE
:1099A000FF920F931F93CF93DF938C017B01C0E055
:1099B000D0E0F701EC0FFD1F6491662361F0D80140
:1099C000ED91FC910190F081E02DC8011995892B52
:1099D00011F02196EECFCE01DF91CF911F910F9123
:1099E000FF90EF9008956115710579F0FB010190EA
:1099F0000020E9F73197AF01461B570BDC01ED91D1
:109A0000FC910280F381E02D199480E090E00895AC
:109A10008F929F92AF92BF92EF92FF920F931F93FC
:109A2000CF93DF93CDB7DEB7A1970FB6F894DEBF23
:109A30000FBECDBF7C01FA01CB0119A2223008F480
:109A40002AE08E010F5D1F4F822E912CA12CB12C8C
:109A5000BF01A50194010E9416B0F901CA0101508D
:109A600011096A3014F4605D01C0695CD8016C931F
:109A7000232B242B252B61F7B801C701B4DFA19656
:109A80000FB6F894DEBF0FBECDBFDF91CF911F910F
:109A90000F91FF90EF90BF90AF909F908F9008959F
:109AA000CF92DF92EF92FF920F931F93CF93DF93AA
:109AB0004115510579F4DC01ED91FC910190F081A3
:109AC000E02DDF91CF911F910F91FF90EF90DF90EC
:109AD000CF9019946B01770FEE08FF084A305105BB
:109AE000E9F4F7FE19C0EC016DE244DF8C01442774
:109AF0005527BA014C195D096E097F092AE0CE018C
:109B000087DF800F911FDF91CF911F910F91FF9001
:109B1000EF90DF90CF9008952AE001C0242FB70185
:109B2000A601DF91CF911F910F91FF90EF90DF90F1
:109B3000CF906ECF58CF1F920F920FB60F92112475
:109B40000BB60F922F933F934F935F936F937F9337
:109B50008F939F93AF93BF93EF93FF938BE39DE01E
:109B600038DAFF91EF91BF91AF919F918F917F91E3
:109B70006F915F914F913F912F910F900BBE0F907E
:109B80000FBE0F901F9018951F920F920FB60F9255
:109B900011240BB60F922F933F934F935F936F93C4
:109BA0007F938F939F93AF93BF93EF93FF938BE339
:109BB0009DE00E943A85FF91EF91BF91AF919F91F7
:109BC0008F917F916F915F914F913F912F910F9066
:109BD0000BBE0F900FBE0F901F9018951F920F9203
:109BE0000FB60F9211240BB60F922F933F934F9302
:109BF0005F936F937F938F939F93AF93BF93EF93F5
:109C0000FF9388ED9DE0E5D9FF91EF91BF91AF9172
:109C10009F918F917F916F915F914F913F912F9184
:109C20000F900BBE0F900FBE0F901F9018951F92B4
:109C30000F920FB60F9211240BB60F922F933F93F2
:109C40004F935F936F937F938F939F93AF93BF9344
:109C5000EF93FF9388ED9DE00E943A85FF91EF918D
:109C6000BF91AF919F918F917F916F915F914F9134
:109C70003F912F910F900BBE0F900FBE0F901F9032
:109C800018951F920F920FB60F9211240BB60F92D8
:109C90002F933F934F935F936F937F938F939F93F4
:109CA000AF93BF93EF93FF9385E79EE092D9FF9127
:109CB000EF91BF91AF919F918F917F916F915F9144
:109CC0004F913F912F910F900BBE0F900FBE0F90B1
:109CD0001F9018951F920F920FB60F9211240BB67A
:109CE0000F922F933F934F935F936F937F938F9335
:109CF0009F93AF93BF93EF93FF9385E79EE00E94FE
:109D00003A85FF91EF91BF91AF919F918F917F9194
:109D10006F915F914F913F912F910F900BBE0F90DC
:109D20000FBE0F901F9018951F920F920FB60F92B3
:109D300011240BB60F922F933F934F935F936F9322
:109D40007F938F939F93AF93BF93EF93FF9382E1A2
:109D50009FE03FD9FF91EF91BF91AF919F918F917C
:109D60007F916F915F914F913F912F910F900BBE1B
:109D70000F900FBE0F901F9018951F920F920FB665
:109D80000F9211240BB60F922F933F934F935F9333
:109D90006F937F938F939F93AF93BF93EF93FF93B3
:109DA00082E19FE00E943A85FF91EF91BF91AF91D0
:109DB0009F918F917F916F915F914F913F912F91E3
:109DC0000F900BBE0F900FBE0F901F901895DC01E7
:109DD00080E0615098F02D91982F9227E92FEF7035
:109DE000F0E0E258F04F249192959F70E92FF0E057
:109DF000E257F04FE491822F8E27EBCF0895EF9238
:109E0000FF920F931F93CF93DF938C017B0140E070
:109E100065E5CDD7E70188E0E80EF11C699140E0E7
:109E2000C801C5D7CE15DF05C9F7DF91CF911F91C6
:109E30000F91FF90EF9008956F927F928F929F9273
:109E4000AF92BF92CF92DF92EF92FF920F931F9348
:109E5000CF93DF93EC017B018A018E819F81DAD75A
:109E6000882389F1B7018E819F81C9DF40E06EEBC5
:109E70008E819F819CD77801680189E0C80ED11C32
:109E8000AE80BF8088E0882E912C712C662463946C
:109E9000C5013AD781117628660CE1E08E1A910847
:109EA000B9F7F70171927F01EC15FD0549F78E8135
:109EB0009F81B0D7813039F468E0C80188DF91E034
:109EC000F8012085281390E0892FDF91CF911F9111
:109ED0000F91FF90EF90DF90CF90BF90AF909F9049
:109EE0008F907F906F900895CF93DF93CDB7DEB7BB
:109EF00029970FB6F894DEBF0FBECDBFAE014F5FFE
:109F00005F4F9ADF882389F08D818F3361F020F4D1
:109F10008F3159F489E00CC08F3519F08F3739F043
:109F200004C08BE005C08AE003C080E001C08CE083
:109F300029960FB6F894DEBF0FBECDBFDF91CF914B
:109F40000895BF92CF92DF92EF92FF920F931F93EB
:109F5000CF93DF93EC016B018D85811104C0CE019D
:109F600059D7811105C01B861D861C8680E05CC008
:109F700040E060EFCE011BD701E0E12CB12C11E0F5
:109F8000CE01C2D6F82ECE01BFD691E0F91203C0A1
:109F90008130B1F433C02E2D30E0F8121BC08B8518
:109FA000181738F4FE01E20FF31F8381802341F478
:109FB00002C0811729F0F12C193058F41C8709C010
:109FC000FE01EE0DF11D8381802B8383FF24F3942A
:109FD00009C0B12EFE01E20FF31F9381802F8095FF
:109FE000892383836F2DCE01B3D61F5F000F11F439
:109FF000E39401E087E08E1508F0C2CF113408F435
:10A00000B2CFBB86B11002C081E08D878B818823DF
:10A0100009F4A9CFDE011396F6012B968D91819359
:10A02000CA17DB07D9F781E0DF91CF911F910F911C
:10A03000FF90EF90DF90CF90BF900895DF92EF9266
:10A04000FF920F931F93CF93DF937C018B01D42E4C
:10A05000DC011696ED91FC911797138615861486F0
:10A06000DF011B9633961E92EA17FB07E1F7C0E06B
:10A07000B801F7018681978164DFD82F882369F0C2
:10A08000DC1208C067E0C801A2DED80117969C91D7
:10A09000891721F0CF5FDC1658F7D0E08D2FDF91C4
:10A0A000CF911F910F91FF90EF90DF900895109244
:10A0B0007113109270131092190D10923A0D1092A4
:10A0C000170D81E08093160D1092F10C61E084E190
:10A0D0000E947B8561E085E10E947B85E9EBF0E0F1
:10A0E00080818E7F808380818D7F808388E48093D0
:10A0F000B80085E48093BC0087EF95E59093570CFA
:10A100008093560C88EF95E59093550C8093540CF2
:10A1100008950F931F93CF93DF93CDB7DEB7629768
:10A120000FB6F894DEBF0FBECDBF8C01CB01F80196
:10A130001182108213821282158214824AE0BE01BB
:10A140006F5F7F4F0E9480AABE016F5F7F4FC80183
:10A150002CDB62960FB6F894DEBF0FBECDBFDF9149
:10A16000CF911F910F910895613208F060E20E9433
:10A17000EB8E10927113809370130895AF92BF927B
:10A18000CF92DF92EF92FF920F931F93CF93DF93C3
:10A19000C82FD62F10928512109286121092871215
:10A1A000109288121092891261E00E94A98560E0E5
:10A1B0008C2F0E947B856D2F70E080E090E00E94E4
:10A1C0002F8660E08C2F0E94A9858BE990E0019793
:10A1D000F1F700E911E08C2F0E945385892B31F4AF
:10A1E00001501109C1F78EEF9FEF4CC000E911E05B
:10A1F0008C2F0E945385019709F43FC018E2D0E8E4
:10A2000000E090E9E92EFF24F3948C2F0E945385FF
:10A21000892B29F481E0E81AF108B9F7E4CF0E940C
:10A220000A866B017C0180E9A82EBB24B3948C2F95
:10A230000E945385019729F481E0A81AB108B9F763
:10A24000D2CF0E940A86DC01CB018C199D09AE0990
:10A25000BF098997A105B10538F0E02FF0E0E35878
:10A26000FD4E80858D2B8087D69511F40F5FD0E849
:10A27000115039F680E090E005C00150110909F055
:10A28000B7CFB1CFDF91CF911F910F91FF90EF909A
:10A29000DF90CF90BF90AF900895EF92FF920F9311
:10A2A0001F93CF93DF93C82F8B017A0183E50E9420
:10A2B0005A6A6C2F8FEA9FE0F4D40E94536A83E5B8
:10A2C0000E945A6AB80183E590E00E942D8FE70151
:10A2D000CE018E199F09309170132091711332179E
:10A2E00029F08FEA9FE095D48993F2CF08171907D8
:10A2F00029F010928B1281E080938C12DF91CF9124
:10A300001F910F91FF90EF900C94536ACF93DF93BE
:10A310004AE050E0BC0182E19FE0C2DBEC0182E157
:10A320009FE00E94E2698C0F9D1FDF91CF910895FD
:10A330001F93CF93DF931F92CDB7DEB7162FAE01D9
:10A340004F5F5F4F61E070E0A8DF898190E002C05D
:10A35000959587951A95E2F781700F90DF91CF91CF
:10A360001F910895CF93DF93D82FC62F83E50E94C6
:10A370005A6A6D2F8FEA9FE094D46C2F8FEA9FE08A
:10A3800090D4DF91CF910C94536AFF920F931F9357
:10A39000CF93DF931F92CDB7DEB7182F062FF42E81
:10A3A000AE014F5F5F4F61E070E077DF4981FF20D2
:10A3B00049F021E030E001C0220F0A95EAF7242B92
:10A3C000298309C081E090E001C0880F0A95EAF76F
:10A3D0008095842389836981812FC4DF0F90DF9169
:10A3E000CF911F910F91FF9008950F931F93CF93DB
:10A3F000DF93EC019A01452B19F40E940B4805C02C
:10A40000462F50E060E070E003DB8C01CE010E943B
:10A41000E269800F911FDF91CF911F910F910895F5
:10A42000CF93DF9342E00E94116BEC0182E19FE049
:10A430000E94E2698C0F9D1FDF91CF9108958F924A
:10A440009F92AF92BF92CF92DF92EF92FF920F93C3
:10A450001F93CF93DF9300D000D0CDB7DEB75C0160
:10A4600049E952E166E070E082E317DF80919912DA
:10A4700090919A129A83898380919B1290919C1259
:10A480009C838B8380919D1290919E129E838D83DD
:10A49000CE0101966C018DE8E82E82E1F82E85014F
:10A4A000F601619171916F01F70181909190A190F6
:10A4B000B1907F01072E000C880B990B0E94BEAE55
:10A4C000A50194010E941DAFF801619371938193DE
:10A4D00091938F01F9E9EF16F2E1FF0609F726964D
:10A4E0000FB6F894DEBF0FBECDBFDF91CF911F91A5
:10A4F0000F91FF90EF90DF90CF90BF90AF909F9023
:10A500008F900895CF93DF93C82F809111130E94ED
:10A510005A6A6C2F8FEA9FE0C4D380E00E94F769EB
:10A5200063E08091111320DE8FEA9FE072D3EC018B
:10A530008FEA9FE06ED320E030E0382FC9018C2BEA
:10A540009D2BDF91CF9108950F931F93CF93DF93AE
:10A55000CDB7DEB761970FB6F894DEBF0FBECDBFA3
:10A560008C01462FBE01665F7F4F68DD811105C0FB
:10A5700060E070E08EEF92EC4BC0AE014F5F5F4F3A
:10A58000BE01665F7F4FC80157DC882361F12A81D5
:10A5900030E0C901982F8827990F990F990F698189
:10A5A00028E0629FB00111249C01262B372B8A855D
:10A5B0008031E1F4688570E08F81AB01481B51095F
:10A5C000CA019695982F8827979587950E9483B3FF
:10A5D00060517109207F53E0220F331F5A95E1F734
:10A5E000620F731F04C060E874EE01C0B9016138E6
:10A5F00054EE75070CF4BCCF072E000C880B990B9A
:10A600000E94BEAE20E030E040E05CE30E941DAF5F
:10A6100061960FB6F894DEBF0FBECDBFDF91CF912C
:10A620001F910F9108959F92AF92BF92CF92DF92A8
:10A63000EF92FF920F931F93CF93DF93CDB7DEB7C7
:10A6400061970FB6F894DEBF0FBECDBF8C018CE0D2
:10A65000F8018183C12CD12C2FE5E22E3FE7B32EE8
:10A660004FE1A42E5FE3952EF801848190E0C81697
:10A67000D9060CF095C04C2DBE01665F7F4FC80116
:10A68000DDDCF8018181893038F0F82EFCE0F81724
:10A6900028F49CE0F92E02C089E0F82E8A858031EA
:10A6A00031F0BE01665F7F4FC8011EDC01C08CE047
:10A6B000F81609F471C0AE014F5F5F4FBE01665FCF
:10A6C0007F4FC801B9DB882309F466C08A858031D1
:10A6D00009F462C08BE0F81651F0ECE0FE1629F0A8
:10A6E000FAE0FF1206C09D8205C0BD8203C0ED8264
:10A6F00001C0AD82F801868197818CD3BE01665F6F
:10A700007F4FF801868197817ADB40E06EE4F801A3
:10A71000868197814CD340E06B81F80186819781D7
:10A7200046D340E06C81F8018681978140D38A85C9
:10A73000803131F040E06D81F8018681978137D317
:10A74000F8018681978166D3BE01665F7F4FF8016D
:10A750008681978154DBF801408168E48681978186
:10A7600026D364E170E080E090E00E942F86F8013B
:10A770008081882331F06AE070E080E090E00E9400
:10A780002F86F8018681978145D3F80181818F1545
:10A7900008F48F2DF8018183FFEFCF1ADF0A64CF11
:10A7A00061960FB6F894DEBF0FBECDBFDF91CF919B
:10A7B0001F910F91FF90EF90DF90CF90BF90AF90DF
:10A7C0009F9008958F929F92AF92BF92CF92DF9207
:10A7D000EF92FF920F931F93CF93DF93EC018E8143
:10A7E0009F8118D340E06CEC8E819F81E0D248813C
:10A7F00064E48E819F81DBD28A81882309F441C081
:10A80000E981E950E33040F4F0E0EE0FFF1FEB5C2C
:10A81000FA4F0081118102C00EEE12E08B81882375
:10A82000F1F0888181111BC00E948B874B015C0174
:10A830006801110FEE08FF088E819F8165D281307B
:10A8400001F10E948B87DC01CB018C199D09AE09B7
:10A85000BF0988159905AA05BB0570F312C0B80198
:10A86000110F880B990BDF91CF911F910F91FF90E2
:10A87000EF90DF90CF90BF90AF909F908F900C940F
:10A880002F86DF91CF911F910F91FF90EF90DF9076
:10A89000CF90BF90AF909F908F900895EF92FF92CE
:10A8A0000F931F93CF93DF93CDB7DEB728970FB6E3
:10A8B000F894DEBF0FBECDBF8C01DC011696ED9182
:10A8C000FC911797138615861486DF011B96339625
:10A8D0001E92EA17FB07E1F7F80114821582EE24B5
:10A8E000E394BE016F5F7F4FD80116968D919C91C6
:10A8F000179727DB882309F46DC067E0CE01019626
:10A9000066DA98858913EDCFF801808181111FC027
:10A91000868197817FD2BE016F5F7F4FD8011696E7
:10A920008D919C9117976BDA40E064EBF80186817A
:10A9300097813DD2D80116968D919C911797E4D1BD
:10A94000F82EF8018681978165D2FF20A1F1D80108
:10A950001196FC9089818031C9F1BE016F5F7F4FF4
:10A96000C801C2DA8F1518F4F80181810AC0898103
:10A97000803111F48CE005C0BE016F5F7F4FC801CC
:10A98000B3DAD80111968C93119714968C91149781
:10A990008F5F14968C938981883281F030F48031F6
:10A9A00069F0823209F09DCF09C08B3339F08234CF
:10A9B00009F097CF03C0F801E082C9CFD8011596FE
:10A9C0008C9115978F5F15968C938BCFBCE0BF153C
:10A9D00058F2D0CF28960FB6F894DEBF0FBECDBF89
:10A9E000DF91CF911F910F91FF90EF9008956F929B
:10A9F0007F928F929F92AF92BF92CF92DF92EF920F
:10AA0000FF920F931F93CF93DF93CDB7DEB72C97B1
:10AA10000FB6F894DEBF0FBECDBF7C015B014A01CB
:10AA20006EEB79E00E94634C6EEB79E0CE01079605
:10AA30000E94634CC12CD12C35018FEF681A780A23
:10AA40008E010F5F1F4FC814D9040CF084C0F701AA
:10AA5000848195818615970508F07DC0B501C801F0
:10AA60000E94338BB801CE0107960E941C4BC8018F
:10AA70000E94FF4B64E170E080E090E00E942F862E
:10AA80008B859C85892B61F4B501C8010E94D18911
:10AA9000B801CE0107960E941C4BC8010E94FF4BD3
:10AAA0008B859C85892B79F060EF77E08F81988585
:10AAB0000E9404B6892BD9F4F70124813581211530
:10AAC000310569F514C064E170E080E090E00E9417
:10AAD0002F86F701848195818A159B0520F4EFEF7D
:10AAE000CE1ADE0AB0CFF5E1CF0ED11CACCFBE013D
:10AAF000695F7F4FC7010E94164BF2E3CF1AD1085E
:10AB0000B701C8010E945B4C42E350E06FEF7FEF5A
:10AB1000C8010E94778DC8010E94FF4BDACF223016
:10AB2000310530F46EEB79E0C7010E94D54BE5CFDB
:10AB30002150310940E050E0B701C8010E94774C34
:10AB40000E151F0521F0B801C7010E941C4BC8015A
:10AB50000E94FF4BD2CFCE0107960E94FF4BC70148
:10AB60002C960FB6F894DEBF0FBECDBFDF91CF910C
:10AB70001F910F91FF90EF90DF90CF90BF90AF901B
:10AB80009F908F907F906F90089585ED8093BC008B
:10AB90008091BC0084FDFCCF1092170D0895409168
:10ABA000780C262F30E0240F311D21323105DCF4E2
:10ABB0002091170D2430C9F4FC0180E090E0861745
:10ABC00058F43091780C2191DC01A85AB34FA30FAF
:10ABD000B11D2C930196F3CF8091780C680F609390
:10ABE000780C80E0089581E0089582E0089508954A
:10ABF00008950895E091711380917013E81730F46F
:10AC0000F0E0EE58FC4E808190E008958FEF9FEFCA
:10AC100008959091711380917013981750F4E92F53
:10AC2000F0E0EE58FC4E208130E09F5F909371136E
:10AC300002C02FEF3FEFC90108958091701390E09B
:10AC400020917113821B91090895CF92DF92EF92A8
:10AC5000FF920F931F93CF93DF937C01CB018A0167
:10AC60002091180D222389F0EB016B01C40ED51E33
:10AC7000CC15DD0561F06991D701ED91FC91019052
:10AC8000F081E02DC7011995F3CF642F88DFC8014B
:10AC9000DF91CF911F910F91FF90EF90DF90CF90B8
:10ACA0000895CF93DF931F92CDB7DEB769832091CC
:10ACB000180D2223D1F020913A0D203240F021E0EE
:10ACC00030E0FC013383228380E090E014C0809167
:10ACD000190DE82FF0E0E65EF24F998190838F5FC7
:10ACE0008093190D80933A0D04C061E0CE01019666
:10ACF00056DF81E090E00F90DF91CF91089580E0E2
:10AD000090E008950C946DB4FC0190810180F28173
:10AD1000E02DF8948181892B81832281892F809570
:10AD200028232283A7E0B0E01197F1F72181822345
:10AD30008183A3E2B0E01197F1F780817894EFEC82
:10AD4000F0E03197F1F7982381E009F480E008956D
:10AD5000FC0190810180F281E02D892F809560FFB8
:10AD600012C0F8942281822382838181892B81837E
:10AD7000A3E2B0E01197F1F78281982B9283789447
:10AD800087ED90E011C0F894228182238283818133
:10AD9000892B8183AFEFB0E01197F1F78281982B77
:10ADA000928378948FE090E00197F1F70895DF9215
:10ADB000EF92FF920F931F93CF93DF93EC01D62E68
:10ADC000E42E08E010E0FF24F39461E08D2D8F2144
:10ADD00009F460E0CE01BCDFFF0C01501109A9F7B6
:10ADE000E11010C0F894E981FA8191818881809501
:10ADF00089238183E981FA819281888180958923E1
:10AE000082837894DF91CF911F910F91FF90EF9003
:10AE1000DF900895DC012C911196ED91FC91129731
:10AE2000F8948181922F90958923818378948DE77E
:10AE300043E050E0815021F1DA011197F1F73081C0
:10AE40003223C1F3F8948281892382838181822B0A
:10AE500081837894ABE7B7E01197F1F7F89481819B
:10AE60009823918383E191E00197F1F78081282372
:10AE700081E009F080E07894E3E6F6E03197F1F7BD
:10AE800008951F93CF93DF93EC01162F60E0812F7D
:10AE90000E94A985612F70E0FB01E05BFC4EE4910C
:10AEA000E883FB01E65FFC4EE491F0E0EE0FFF1F4C
:10AEB000E051FD4E859194919A8389831B861D866E
:10AEC0001C86FE013B9623961292EC17FD07E1F7D4
:10AED000DF91CF911F9108951F93CF93DF93EC01E2
:10AEE000162F8C810E945A6A6B85812F862B90E0E9
:10AEF0000E94556ADF91CF911F910C94536A0F9372
:10AF00001F93CF938C01C62FE7DF6C2F6460C801BD
:10AF1000E3DF6C2F6B7FC801DFDF83EC90E00197EC
:10AF2000F1F7CF911F910F9108950F931F93CF9336
:10AF30008C01C62F607F6160E2DF80E1C89FB001B5
:10AF400011246160C801DBDF81E090E0CF911F91A7
:10AF50000F9108951F920F920FB60F9211240BB606
:10AF60000F922F933F934F935F936F937F938F93A2
:10AF70009F93AF93BF93EF93FF938091BC0F0E9479
:10AF800053852091C00F3091C10F2F5F3F4F3093F9
:10AF9000C10F2093C00F9091BF0F953618F096E027
:10AFA0009093BB0F9091BB0F9430C9F128F492306D
:10AFB00069F09330D1F05EC0953009F451C09630FD
:10AFC00009F058C091E090938C1051C0811152C08B
:10AFD0002091C00F3091C10F2436310508F442C0D2
:10AFE00010928C101092BF0F1CC0813009F042C02B
:10AFF000E091BF0F91E09E0F9093BF0FF0E0209182
:10B00000C00F3091C10FEE0FFF1FE554F04F308796
:10B0100027831092C10F1092C00F94E029C08111B4
:10B0200017C0E091BF0F91E09E0F9093BF0FF0E02B
:10B030002091C00F3091C10FEE0FFF1FE554F04F6C
:10B04000308727831092C10F1092C00F93E010C079
:10B050002091C00F3091C10F2536310558F007C03F
:10B06000811108C01092C10F1092C00F03C095E06B
:10B070009093BB0F9091BE0F9923B9F081110AC034
:10B080008091BD0F882321F08091BD0F61E009C040
:10B090002F9A0BC08091BD0F882331F08091BD0F96
:10B0A00060E00E947B8501C02F98FF91EF91BF91D6
:10B0B000AF919F918F917F916F915F914F913F9150
:10B0C0002F910F900BBE0F900FBE0F901F901895F1
:10B0D000CF92DF92EF92FF92CF93DF93EC01072E96
:10B0E000000C880B990B0E94BEAE6B017C0120E026
:10B0F00030E040E45FE30E941DAF20E030E048E430
:10B1000052E40E940EB10E94A7B1C617D707D4F02F
:10B1100020E030E040EA5FE3C701B6010E941DAFC6
:10B1200020E030E048E452E40E940EB120E030E03C
:10B1300040E85FE30E9448B00E94A7B121E06C178D
:10B140007D070CF420E0822F90E0DF91CF91FF90FB
:10B15000EF90DF90CF9008950F931F93CF93DF93DD
:10B16000082F60E476E082E19FE00E949A4DC7E0FC
:10B17000D0E010E0B8010C2E02C0759567950A94D6
:10B18000E2F76170772742E050E082E19FE00E94A1
:10B19000504D219778F7DF91CF911F910F9108952E
:10B1A0001F920F920FB60F9211240BB60F922F938E
:10B1B0003F934F935F936F937F938F939F93AF933F
:10B1C000BF93EF93FF938091B900887F803609F495
:10B1D0009CC068F5883209F45BC090F4803109F4B2
:10B1E00054C038F4882309F4F6C0883009F44DC0FF
:10B1F000F5C0883109F44CC0803209F45DC0EEC05E
:10B20000803409F468C048F4803309F455C08833A9
:10B2100009F0E4C08093150DD8C0803509F44FC003
:10B22000883509F45DC0883409F0D8C0D6C08839A3
:10B2300009F4C7C0A8F4883709F467C038F4883621
:10B2400009F463C0803709F460C0C8C0883809F4C5
:10B25000B8C0803909F45FC0803809F0BFC05BC056
:10B26000803B09F486C038F4803A09F466C0883A15
:10B2700009F47FC0B3C0803C09F4A7C0883C09F43E
:10B28000A4C0883B09F48AC0A9C08091F20C10C008
:10B290009091140D8091130D981770F5E091140D95
:10B2A00081E08E0F8093140DF0E0ED50F34F80811C
:10B2B0008093BB0085EC86C08093150D8EC0E09115
:10B2C000140D81E08E0F8093140D8091BB00F0E08F
:10B2D000ED50F34F80839091140D8091130D6EC04B
:10B2E000E091140D81E08E0F8093140D8091BB00CE
:10B2F000F0E0ED50F34F80838091160D81116DC009
:10B3000081E08093F10C84EA61C083E08093170DA3
:10B3100010929A0CCFCF80919A0C803208F051C0D5
:10B32000E0919A0C81E08E0F80939A0C8091BB0083
:10B33000F0E0E658F34F8083BDCF85EC8093BC00EE
:10B340001092170D80919A0C803230F4E0919A0C93
:10B35000F0E0E658F34F108260919A0C70E0E091B3
:10B36000540CF091550C8AE79CE0199510929A0CB8
:10B3700035C084E08093170D1092790C1092780CF0
:10B38000E091560CF091570C19958091780C811131
:10B3900005C081E08093780C1092580CE091790CF4
:10B3A00081E08E0F8093790CF0E0E85AF34F8081B2
:10B3B0008093BB009091790C8091780C981708F4D9
:10B3C00079CF85E88093BC0009C085EC8093BC00F0
:10B3D0001092170D03C01092150DD7DBFF91EF915E
:10B3E000BF91AF919F918F917F916F915F914F919D
:10B3F0003F912F910F900BBE0F900FBE0F901F909B
:10B4000018950895EEE8F0E114A215A216A217A26D
:10B4100010A611A612A613A681E084A729E130E0A8
:10B4200036A725A787A780E090E0A0EAB0E480AB2C
:10B4300091ABA2ABB3AB80E090E0A8EAB1E484ABFF
:10B4400095ABA6ABB7AB8093250290932602A09351
:10B450002702B093280280E090E0A0E8BFE3809349
:10B46000D8109093D910A093DA10B093DB1080938A
:10B47000210290932202A0932302B09324021092FF
:10B480000511109204118BE090E0909307118093C6
:10B49000061190932A028093290210923C0C10927C
:10B4A0003B0C80E090E00C94A26EEF92FF920F9321
:10B4B0001F93CF93DF93CDB7DEB768970FB6F8949D
:10B4C000DEBF0FBECDBF8C0169ED7BE0CE010D96D6
:10B4D0000E94634C60E179E0CE0143960E94634C88
:10B4E00061EF7FE0C8010E94534CBE016D5E7F4F4B
:10B4F000C8010E94164B68EE7FE0C8010E94C64A50
:10B500008DE1E82E81E1F82EF701608170E0CE0137
:10B5100001960E948950BE016F5F7F4FCE01079652
:10B520000E945B4CBE01635F7F4FCE0107960E9475
:10B530007F4BBC01C8010E94164BCE0107960E94AA
:10B54000FF4BCE0101960E94FF4B6BED7FE0C801DF
:10B550000E94C64AF7016181062E000C770BCE01CE
:10B5600001960E948950BE016F5F7F4FCE01079602
:10B570000E945B4CBE01635F7F4FCE0107960E9425
:10B580007F4BBC01C8010E94164BCE0107960E945A
:10B59000FF4BCE0101960E94FF4B61ED7FE0C80199
:10B5A0000E94C64AF7016281062E000C770BCE017D
:10B5B00001960E948950BE016F5F7F4FCE010796B2
:10B5C0000E945B4CBE01635F7F4FCE0107960E94D5
:10B5D0007F4BBC01C8010E94164BCE0107960E940A
:10B5E000FF4BCE0101960E94FF4B69EC7FE0C80142
:10B5F0000E94C64AF70163817481CE0101960E94C0
:10B600008950BE016F5F7F4FCE0107960E945B4C51
:10B61000BE016D5E7F4FCE0107960E947F4BBC013D
:10B62000C8010E94164BCE0107960E94FF4BCE0127
:10B6300001960E94FF4B62EB7FE0C8010E94C64A60
:10B64000F70165817681CE0101960E948950BE0185
:10B650006F5F7F4FCE0107960E945B4CBE01635F18
:10B660007F4FCE0107960E947F4BBC01C8010E940C
:10B67000164BCE0107960E94FF4BCE0101960E9409
:10B68000FF4B69EA7FE0C8010E94C64AF701678163
:10B69000062E000C770B6F5F7F4FCE0101960E9444
:10B6A0008950BE016F5F7F4FCE0107960E945B4CB1
:10B6B000BE01635F7F4FCE0107960E947F4BBC01A6
:10B6C000C8010E94164BCE0107960E94FF4BCE0187
:10B6D00001960E94FF4B6EE97FE0C8010E94C64AB6
:10B6E000F7016085062E000C770BCE0101960E94B3
:10B6F0008950BE016F5F7F4FC8010E94164BCE017B
:10B7000001960E94FF4BCE0143960E94FF4BCE0153
:10B710000D960E94FF4BC80168960FB6F894DEBFE5
:10B720000FBECDBFDF91CF911F910F91FF90EF9092
:10B7300008950F931F9360E0809102020E947B8521
:10B7400083E090E00197F1F761E0809102020E94AE
:10B750007B8583E290E00197F1F760E0809102023F
:10B760000E947B8580910002909101029927FC0143
:10B77000E05BFC4E6491FC01E65FFC4EE491F0E07E
:10B78000EE0FFF1FE051FD4E8591949100E412E40D
:10B790002FE030E0462F0E940B9A6115710581055C
:10B7A000910549F0DC01CB010196A11DB11DBC0141
:10B7B000CD019F7003C060E070E0CB010E94BCAE81
:10B7C00020E030E048EC52E40E940EB120919B0C46
:10B7D00030919C0C40919D0C50919E0C0E941DAF8D
:10B7E00020E030E44CE156E40E940EB120E030E06D
:10B7F00040E05FE30E941DAF1F910F91089523E386
:10B8000033E948E853E40E940EB120E030E040E81C
:10B810005FE30E9448B00E9406B326E636EA45EA96
:10B8200053E40E941DAF60939B0C70939C0C80931B
:10B830009D0C90939E0C0895CF92DF92EF92FF9211
:10B8400078DF6B017C0120E030E040E050E40E94B2
:10B85000FDB118161CF46DDF6B017C0120E030E0B7
:10B8600040E050E4C701B6010E94FDB118161CF477
:10B8700060DF6B017C0120E030E040E050E4C70174
:10B88000B6010E94FDB118161CF453DF6B017C0158
:10B8900020E030E040E050E4C701B6010E94FDB175
:10B8A00018162CF4FF90EF90DF90CF9042CFC70195
:10B8B000B601FF90EF90DF90CF900895BF92CF92A6
:10B8C000DF92EF92FF920F931F93CF93DF93CDB749
:10B8D000DEB762970FB6F894DEBF0FBECDBF8C0106
:10B8E0006B0169ED7BE0CE010D960E94634C67E32E
:10B8F00070E1C8010E94534C76012FEFE21AF20A60
:10B90000B701CE0101960E948950BE016F5F7F4F43
:10B91000CE0107960E945B4C66E177E0CE01079668
:10B920000E94684BBC01C8010E94164BCE010796CD
:10B930000E94FF4BCE0101960E94FF4B8AE0B82E79
:10B94000BE9CC001BF9C900D1124FC01E35EFE4E25
:10B950007F018081082E000C990B0E94EDB5892B88
:10B9600009F4B2C0B701CE0101960E94634CBE013A
:10B970006F5F7F4FCE0107960E945B4C68EF7AE0C5
:10B98000CE0107960E94684BBC01C8010E94164B6D
:10B99000CE0107960E94FF4BCE0101960E94FF4BFD
:10B9A000BC9CC001BD9C900D11249C01235E3E4EA9
:10B9B0007901F9016685062E000C770BCE01019600
:10B9C0000E948950BE016F5F7F4FCE0107960E9493
:10B9D0005B4C63E179E0CE0107960E94684BBE01A3
:10B9E000635F7F4F0E947F4BBC01C8010E94164BD2
:10B9F000CE0107960E94FF4BCE0101960E94FF4B9D
:10BA000060E370E1C8010E94C64AF7016785062E0F
:10BA1000000C770BCE0101960E948950BE016F5F2A
:10BA20007F4FCE0107960E945B4CBE01635F7F4F44
:10BA3000CE0107960E947F4BBC01C8010E94164BA5
:10BA4000CE0107960E94FF4BCE0101960E94FF4B4C
:10BA50006AE270E1C8010E94C64AF70160897189F3
:10BA6000CE0101960E948950BE016F5F7F4FCE01CB
:10BA700007960E945B4CBE01635F7F4FCE01079625
:10BA80000E947F4BBC01C8010E94164BCE01079655
:10BA90000E94FF4BCE0101960E94FF4B65E270E1D0
:10BAA000C8010E94C64AF70162897389CE010196D6
:10BAB0000E948950BE016F5F7F4FC8010E94164BE4
:10BAC000CE0101960E94FF4BCE010D960E94FF4BC6
:10BAD000C80162960FB6F894DEBF0FBECDBFDF91EE
:10BAE000CF911F910F91FF90EF90DF90CF90BF907B
:10BAF00008950F931F93CF93DF93CDB7DEB72C97A5
:10BB00000FB6F894DEBF0FBECDBF8C016EEB79E0AF
:10BB100081E492E10E94D54B0830110509F0DFC0A5
:10BB200066E271E1CE0101960E94534C44E650E07A
:10BB30006FEF7FEFCE0101960E94BF8FCE0101967D
:10BB40000E94FF4B6AE171E1CE0101960E94534CC5
:10BB500044E650E060E070E0CE0101960E94778DEF
:10BB6000CE0101960E94FF4B8BE39DE00E94574857
:10BB70004CE251E061E070E0CE0101960E94F75482
:10BB800080919A138823D1F065E179E0CE01079680
:10BB90000E94634CBE016F5F7F4FCE0107960E94EB
:10BBA0007F4B61E277E00E94684BBC0182E19FE03D
:10BBB0000E94E669CE0107960E94FF4B6DEC78E08B
:10BBC000CE0107960E94634CBE01695F7F4FCE0194
:10BBD00001960E941F85182FCE0107960E94FF4BE9
:10BBE000112309F4A5C268E179E081E492E10E94A1
:10BBF000D54B88E090E090930C0C80930B0C0E9446
:10BC00003D35182F6DE071E1CE0107960E94534C2F
:10BC100044E650E060E070E0CE0107960E94778D28
:10BC2000CE0107960E94FF4B8BE39DE00E94574890
:10BC300048E552E061E070E0CE0107960E94F754BB
:10BC4000BE01695F7F4FCE0101960E941C4BCE0161
:10BC500007960E94FF4B80919A138823D1F065E1EB
:10BC600079E0CE0107960E94634CBE016F5F7F4F63
:10BC7000CE0107960E947F4B61E277E00E94684BFD
:10BC8000BC0182E19FE00E94E669CE0107960E9416
:10BC9000FF4B60E476E0CE0107960E94634CBE0144
:10BCA000695F7F4FCE0101960E941F85082FCE014C
:10BCB00007960E94FF4B002309F43AC26DE179E038
:10BCC00081E492E10E94D54B0E943D35882309F41E
:10BCD0002FC2112309F42CC260E071E1F9C0093FC1
:10BCE0002FEF120709F00BC16FEE70E1CE01019644
:10BCF0000E94534C44E650E06FEF7FEFCE01019677
:10BD00000E94BF8FCE0101960E94FF4B61EE70E151
:10BD1000CE0101960E94534C44E650E060E070E092
:10BD2000CE0101960E94778DCE0101960E94FF4BB5
:10BD30008BE39DE00E9457484CE251E064E070E0E4
:10BD4000CE0101960E94F75480919A138823D1F076
:10BD500065E179E0CE0107960E94634CBE016F5FFA
:10BD60007F4FCE0107960E947F4B61E277E00E94F1
:10BD7000684BBC0182E19FE00E94E669CE01079614
:10BD80000E94FF4B60E070E0CE0101960E94B54A30
:10BD9000082E000C990BC0970A9708F0CCC163E2FB
:10BDA00079E0CE0107960E94634CBE016F5F7F4F22
:10BDB000CE0107960E947F4BBC0181E492E10E9474
:10BDC000EA4BCE0107960E94FF4B89EF9FEF9093BD
:10BDD0000C0C80930B0C0E943D35182F63ED70E125
:10BDE000CE0107960E94534C44E650E060E070E0BC
:10BDF000CE0107960E94778DCE0107960E94FF4BD9
:10BE00008BE39DE00E94574848E552E065E070E012
:10BE1000CE0107960E94F754BE01695F7F4FCE01A5
:10BE200001960E941C4BCE0107960E94FF4B809109
:10BE30009A138823D1F065E179E0CE0107960E943C
:10BE4000634CBE016F5F7F4FCE0107960E947F4B10
:10BE500061E277E00E94684BBC0182E19FE00E94B2
:10BE6000E669CE0107960E94FF4B60E070E0CE01CC
:10BE700001960E94B54A082E000C990BC0970A97AC
:10BE800008F059C168E279E0CE0107960E94634C40
:10BE9000BE016F5F7F4FCE0107960E947F4BBC01B2
:10BEA00081E492E10E94EA4BCE0107960E94FF4B8B
:10BEB00089EF9FEF90930C0C80930B0C0E943D3503
:10BEC000882309F438C1112309F435C166EC70E107
:10BED000CE0107960E94534C44E650E060E070E0CB
:10BEE000CE0107960E94778DCE0107960E94FF4BE8
:10BEF0006EEB79E081E492E10E94D54B14C165EBD1
:10BF000070E1CE0101960E94534C44E650E06FEF81
:10BF10007FEFCE0101960E94BF8FCE0101960E9455
:10BF2000FF4B6EEB79E081E492E10E94D54B053F37
:10BF30008FEF180749F46DE678E081E492E10E9402
:10BF4000D54B6BEA70E126C0063F2FEF120749F48C
:10BF500067E678E081E492E10E94D54B61EA70E106
:10BF600019C0013F8FEF180749F461E778E081E4D9
:10BF700092E10E94D54B62E970E10CC0023F2FEFC5
:10BF80001207B9F46DE279E081E492E10E94D54BA9
:10BF900062E870E1CE0101960E94534C44E650E005
:10BFA0006FEF7FEFCE0101960E94778DCE01019653
:10BFB000C5C00230110509F07EC066E770E1CE0110
:10BFC00001960E94534C44E650E06FEF7FEFCE01A4
:10BFD00001960E94BF8FCE0101960E94FF4B66E63C
:10BFE00070E1CE0101960E94534C44E650E06FEFA1
:10BFF0007FEFCE0101960E94778DCE0101960E94BF
:10C00000FF4B44EF51E066E070E0CE0101960E94E4
:10C01000F754BE016F5F7F4F81E492E10E941C4B99
:10C02000CE0101960E94FF4B8091451290914612DD
:10C03000059708F486C060E070E081E492E10E9418
:10C04000B54A082E000C990BC0970A9708F079C0E2
:10C0500081E492E10E944A4A613523EC720781052E
:10C0600091050CF46EC00E94BEAE20E030E048ECBA
:10C0700052E40E940EB1AB01BC0122E0CE01079652
:10C080000E94044C6EE478E0CE0101960E94634C5D
:10C09000BE01695F7F4FCE0101960E947F4BBC01BC
:10C0A00081E492E10E94EA4BCE0101960E94FF4B8F
:10C0B000CE01079643C06FE470E1CE0101960E9465
:10C0C000534C44E650E06FEF7FEFCE0101960E94A3
:10C0D000778DCE0101960E94FF4B6EEB79E081E4F3
:10C0E00092E10E94D54B0B3E8FEF180709F465C013
:10C0F0008091451290914612892BE1F55EC068EC63
:10C1000070E080E090E00E942F8669E370E1CE014C
:10C1100001960E94534C44EF51E06FEF7FEFCE0148
:10C1200001960E94778DCE0101960E94FF4B45C07B
:10C1300069EF70E1CDCE6FEB70E1CACE0E94FF4B8C
:10C14000D7CF68E570E1CE0101960E94534C48EECE
:10C1500053E06FEF7FEFCE0101960E94778DCE0105
:10C1600001960E94FF4B6EEB79E081E492E10E9420
:10C17000D54BBECF0E943D35882309F268EC70E0B4
:10C1800080E090E00E942F8665E470E1CE01019688
:10C190000E94534C44EF51E06FEF7FEFCE010196C8
:10C1A0000E94778DCE0101960E94FF4B10930C0CDC
:10C1B00000930B0CC8010E94D70A2C960FB6F89476
:10C1C000DEBF0FBECDBFDF91CF911F910F910895BC
:10C1D0006F927F928F929F92AF92BF92CF92DF9297
:10C1E000EF92FF920F931F93CF93DF93CDB7DEB7FC
:10C1F00068970FB6F894DEBF0FBECDBF6C0180917B
:10C20000041190910511019731F06EEB79E0C601B0
:10C210000E94634C46C169E379E0CE010D960E940D
:10C22000634CBE01635F7F4F8BE39DE00E94C14C76
:10C230006CE271E080E090E00E942F86CE01439690
:10C240000E94EB7564E670E080E090E00E942F862B
:10C25000E12CF12C85E0A82EB12C9AE0892E912CAE
:10C2600064E479E0CE0101960E94634C8F89988D39
:10C27000892B69F06B887C8869817A81C3010E946F
:10C2800031B6009721F08C010619170902C00FEF93
:10C290001FEFCE0101960E94FF4BA8014F5F5F4F39
:10C2A000BE016D5E7F4FCE0101960E94343FBE01FC
:10C2B0006F5F7F4FCE010D960E941C4BCE01019601
:10C2C0000E94FF4B89899A89892B69F060E070E0B0
:10C2D000CE010D960E94B54A082E000C990BC0970E
:10C2E0000A9708F4C7C010E065E170E1CE0101963D
:10C2F0000E94534C44E150E06FEF7FEFCE01019676
:10C300000E946490CE0101960E94FF4B8FEFE81AC5
:10C31000F80A62E370E080E090E00E942F86C70197
:10C32000B5010E9483B3019771F5CE0101960E9479
:10C33000A2748D819E81892B59F0BE016F5F7F4F62
:10C3400081E492E10E94EA4B0E949C7E11E017C0BA
:10C3500084E1E816F1049CF0C701B4010E9483B3A4
:10C36000892B69F4BE01635F7F4F8BE39DE00E94E0
:10C37000C14C68EC70E080E090E00E942F86CE0116
:10C3800001960E94FF4BCE0101960E94EB75BE0103
:10C390006F5F7F4FCE0143960E941C4BCE010196EA
:10C3A0000E94FF4B62E370E080E090E00E942F86E5
:10C3B00084E6E816F10419F0112309F451CF8091B5
:10C3C0009A138823F1F061E179E0CE0101960E9491
:10C3D000634CBE01635F7F4FCE0101960E947F4B8D
:10C3E000BC01CE0107960E945B4CCE0107960E94CD
:10C3F0002971CE0107960E94FF4BCE0101960E9443
:10C40000FF4B89899A89892B61F060E070E0CE0149
:10C410000D960E94B54A082E000C990BC0970A97FA
:10C4200030F066E479E0C6010E94634C1AC062E510
:10C4300079E0CE0101960E94634CBE016F5F7F4F91
:10C44000CE010D960E941F85182FCE0101960E94E5
:10C45000FF4B1111E6CFBE01635F7F4FC6010E9403
:10C460004B4CCE0143960E94FF4BCE010D960E948D
:10C47000FF4B17C062E579E0CE0101960E94634C44
:10C48000BE016F5F7F4FCE010D960E941F85082F62
:10C49000CE0101960E94FF4B11E0002309F424CF46
:10C4A00022CFC60168960FB6F894DEBF0FBECDBF8F
:10C4B000DF91CF911F910F91FF90EF90DF90CF9080
:10C4C000BF90AF909F908F907F906F900895AF92A4
:10C4D000BF92CF92DF92EF92FF920F931F93CF9371
:10C4E000DF93CDB7DEB72C970FB6F894DEBF0FBE43
:10C4F000CDBF8091470C811102C00E94E93E80911E
:10C50000050290910602029751F08091110C9091D2
:10C51000120C009709F48DC1039709F48AC16FE5E5
:10C5200071E18DE192E10E94904B6DE172E1CE01EB
:10C5300001960E945B4C44E150E060E070E0CE0167
:10C5400001960E94BF8FCE0101960E94FF4B60E5CD
:10C5500071E18DE192E10E94904B6DE172E1CE01BB
:10C5600001960E945B4C44E150E06FEF7FEFCE01FB
:10C5700001960E94778DCE0101960E94FF4B87E0C5
:10C580000E9482528C0186E00E948252BC0180E0AF
:10C5900090E00E94BCAE2AE037ED43EA5CE30E94E3
:10C5A0001DAF23E333E948E853E40E9447B06B0131
:10C5B0007C0184E0A82EB12C20E030E048EC52E46D
:10C5C000C701B6010E94FDB1181614F581E0A81A42
:10C5D000B10809F4F4C064E670E080E090E00E94E5
:10C5E0002F8686E00E948252BC0180E090E00E948B
:10C5F000BCAE2AE037ED43EA5CE30E941DAF23E3C3
:10C6000033E948E853E40E9447B06B017C01D4CF82
:10C61000B80180E090E00E94BCAE2AE037ED43EA2A
:10C620005CE30E941DAF23E333E948E853E40E9432
:10C6300047B0AB01BC0121E0CE0101960E94044C41
:10C640006CE679E0CE0107960E94634CBE016F5FF5
:10C650007F4FCE0107960E947F4BBC0183E292E19F
:10C660000E94EA4BCE0107960E94FF4BCE01019635
:10C670000E94FF4B63E272E1CE0101960E945B4C87
:10C6800042E350E06FEF7FEFCE0101960E94778D7D
:10C69000CE0101960E94FF4B66E779E0CE0101963C
:10C6A0000E94634CCE0101960E94F38DCE0101964B
:10C6B0000E94FF4B65E779E083E292E10E94084B1C
:10C6C00021E0B701A601CE0101960E94044C6CE066
:10C6D0007AE0CE0107960E94634CBE016F5F7F4FE8
:10C6E000CE0107960E947F4BBC0189E292E10E9435
:10C6F000EA4BCE0107960E94FF4BCE0101960E94A5
:10C70000FF4B69ED7BE0CE0101960E94634C69E22C
:10C7100072E1CE0101960E947F4BBC018DE192E156
:10C720000E94EA4BCE0101960E94FF4B6DE172E13F
:10C73000CE0101960E945B4C4AE050E060E070E060
:10C74000CE0101960E946490CE0101960E94FF4B9B
:10C7500066E779E0CE0101960E94634CCE01019616
:10C760000E94F38DCE0101960E94FF4B65E779E0B0
:10C7700089E292E10E94084B69E272E1CE010196E2
:10C780000E945B4C69ED7BE0CE0101960E94684BF4
:10C7900063E272E10E947F4BBC0183E292E10E945E
:10C7A000EA4BCE0101960E94FF4B8091110C9091B3
:10C7B000120C039709F006C184E090E0FFC065E425
:10C7C00071E18DE192E10E94904B6DE172E1CE0149
:10C7D00001960E945B4C4AE050E060E070E0CE01C0
:10C7E00001960E94BF8FCE0101960E94FF4B6AE521
:10C7F00079E0CE0101960E94634C6DE172E1CE01B9
:10C8000001960E947F4BBC0183E292E10E94EA4BB9
:10C81000CE0101960E94FF4B8091110C9091120C59
:10C82000049721F41092120C1092110C81E090E008
:10C8300018C188ED9DE00E94118E64E670E080E0F2
:10C8400090E00E942F8665E871E18DE192E10E94FF
:10C85000904B6DE172E1CE0101960E945B4C44E188
:10C8600050E060E070E0CE0101960E94BF8FCE01E3
:10C8700001960E94FF4B66E771E18DE192E10E9413
:10C88000904B6DE172E1CE0101960E945B4C44E158
:10C8900050E06FEF7FEFCE0101960E94778DCE01C1
:10C8A00001960E94FF4B8CE40E942F8E6B017C014D
:10C8B00004E010E0A7019601C701B6010E9447B34A
:10C8C000811192C021E0B701A601CE0107960E9416
:10C8D000044C6CE679E0CE0101960E94634CBE01E7
:10C8E000695F7F4FCE0101960E947F4BBC0183E2BE
:10C8F00092E10E94EA4BCE0101960E94FF4BCE01CD
:10C9000007960E94FF4B63E272E1CE0101960E94FE
:10C910005B4C42E350E06FEF7FEFCE0101960E9447
:10C92000778DCE0101960E94FF4B66E779E0CE013C
:10C9300001960E94634CCE0101960E94F38DCE01B8
:10C9400001960E94FF4B65E779E083E292E10E9445
:10C95000084B86E60E942F8E6B017C0104E010E0FC
:10C96000A7019601C701B6010E9447B3882309F4C5
:10C970007DC00150110909F0E2C06EEB79E089E257
:10C9800092E10E94D54B69E272E1CE0101960E94CC
:10C990005B4C69ED7BE0CE0101960E94684B63E23F
:10C9A00072E10E947F4BBC0183E292E10E94EA4B5C
:10C9B000CE0101960E94FF4B83E090E09093120C11
:10C9C0008093110C64E670E080E090E00E942F8676
:10C9D0008091470C882309F4BEC060E273E080E0D8
:10C9E00090E00E942F86B7C00150110909F09BC04A
:10C9F0006BE671E18DE192E10E94904B6DE172E195
:10CA0000CE0101960E945B4C4AE050E060E070E08D
:10CA1000CE0101960E94BF8FCE0101960E94FF4B6E
:10CA20006AE579E0CE0101960E94634C6DE172E106
:10CA3000CE0101960E947F4BBC0183E292E10E94ED
:10CA4000EA4BCE0101960E94FF4B8091110C909110
:10CA5000120C039721F41092120C1092110C82E028
:10CA600090E09093060280930502ACCF21E0B701DD
:10CA7000A601CE0107960E94044C6CE07AE0CE013C
:10CA800001960E94634CBE01695F7F4FCE01019603
:10CA90000E947F4BBC0189E292E10E94EA4BCE01E9
:10CAA00001960E94FF4BCE0107960E94FF4B69ED55
:10CAB0007BE0CE0101960E94634C69E272E1CE01F7
:10CAC00001960E947F4BBC018DE192E10E94EA4BEE
:10CAD000CE0101960E94FF4B6DE172E1CE010196FD
:10CAE0000E945B4C4AE050E06FEF7FEFCE01019671
:10CAF0000E946490CE0101960E94FF4B66E779E0A8
:10CB0000CE0101960E94634CCE0101960E94F38DE6
:10CB1000CE0101960E94FF4B65E779E089E292E140
:10CB20000E94084B30CF68EC70E080E090E00E94FB
:10CB30002F868CE40E942F8E6B017C01BBCE68ECAB
:10CB400070E080E090E00E942F8686E60E942F8EA3
:10CB50006B017C0105CF2C960FB6F894DEBF0FBE9B
:10CB6000CDBFDF91CF911F910F91FF90EF90DF909C
:10CB7000CF90BF90AF9008952F923F924F925F92C7
:10CB80006F927F928F929F92AF92BF92CF92DF92DD
:10CB9000EF92FF920F931F93CF93DF93CDB7DEB742
:10CBA000C554D1090FB6F894DEBF0FBECDBF2B011F
:10CBB0003C0169017A010E948B8722966CAF7DAFA0
:10CBC0008EAF9FAF229720E9421621E05206610402
:10CBD000710434F090E9492E55245394612C712C42
:10CBE00030E1C31637E2D306E104F1042CF4CDA6FC
:10CBF000DEA6EFA6F8AA08C080E197E2A0E0B0E0C8
:10CC00008DA79EA7AFA7B8AB8091470C882321F0D2
:10CC1000CDA6DEA6EFA6F8AA22966CAD7DAD8EADB0
:10CC20009FAD229728EE33E040E050E00E94EAAF4B
:10CC300026962CAF3DAF4EAF5FAF269791E09DABF0
:10CC400019A61AA61BA61CA68E01035F1F4FCC2493
:10CC5000DD247601C418D508E608F708C9AADAAABF
:10CC6000EBAAFCAAC9A4DAA4EBA4FCA42DA53EA5BA
:10CC70004FA558A9C216D306E406F5060CF02BC33F
:10CC8000C701B6010E94BEAE20E030E04AE754E49E
:10CC90000E940EB1AB01BC0123E0C8010E94044C0C
:10CCA000B8018DE192E10E941C4BC8010E94FF4B2C
:10CCB0008DA59EA5AFA5B8A90A97A105B10584F4D5
:10CCC00026964CAD5DAD6EAD7FAD2697C80138D4CC
:10CCD000B8018DE192E10E941C4BC8010E94FF4BFC
:10CCE000CE0101960E941F5268E371E183E292E156
:10CCF0000E94904BDE0111961D01C12CD12C7601B2
:10CD0000F10181909190A190B1901F01A501940132
:10CD1000C501B4010E941DAF9B01AC01C701B60162
:10CD20000E9448B06B017C0123E0B501A401C80159
:10CD30000E94044CB801CE0143960E945B4C69ED01
:10CD40007BE0CE0143960E94684BBC0183E292E1F6
:10CD50000E94164BCE0143960E94FF4BC8010E94D1
:10CD6000FF4B0215130561F6C701B6010E9406B319
:10CD70006B017C01FDE24F16F1E05F066104710476
:10CD80002CF00E94E93E60E080E0AFD323E0B701E1
:10CD9000A601CE0143960E94044C68EF78E0C801DA
:10CDA0000E94634C6DE172E1C8010E947F4B68E70D
:10CDB00079E00E94684BBE016D5E7F4F0E947F4B01
:10CDC0006DE779E00E94684BBC0183E292E10E942A
:10CDD000164BC8010E94FF4BCE0143960E94FF4BA9
:10CDE0002DEC3CEC4CE45FE3C701B6010E94FDB1C1
:10CDF00029813A814B815C812DA33EA34FA358A783
:10CE000018160CF0ACC12AE939E949E95FE3C7011A
:10CE1000B6010E94B8AE87FFA2C1CDA8CC2009F40C
:10CE20009EC189849A84AB84BC8420E030E0A9014F
:10CE3000C501B4010E94B8AECD80DE80EF80F884D9
:10CE4000882309F12DA13EA14FA158A5CA01B9011E
:10CE50000E941DAF6EAB7FAB88AF99AFA701960163
:10CE6000C701B6010E941DAF9B01AC016EA97FA94D
:10CE700088AD99AD0E9448B00E9406B3A501940107
:10CE80000E94BBB004C06BED7FE089EC9FE320EE15
:10CE90003EE245E652E40E941DAF6EAB7FAB88AF29
:10CEA00099AF20E030E0A901C701B6010E94B8AEF9
:10CEB000882309F12DA13EA14FA158A5CA01B901AE
:10CEC0000E941DAF6AAF7BAF8CAF9DAFA5019401EF
:10CED000C501B4010E941DAF9B01AC016AAD7BADE1
:10CEE0008CAD9DAD0E9448B00E9406B3A70196018B
:10CEF0000E94BBB004C06BED7FE089EC9FE320EEA5
:10CF00003EE245E652E40E941DAF6AAF7BAF8CAFB4
:10CF10009DAF20E030E0A9016DA17EA18FA198A571
:10CF20000E94B8AE8823F9F0A5019401C501B401AF
:10CF30000E941DAF4B015C01A7019601C701B6011C
:10CF40000E941DAF9B01AC01C501B4010E9448B015
:10CF50000E9406B32DA13EA14FA158A50E94BBB0CF
:10CF60006B017C0108C08BEDC82E8FE0D82E89ECB8
:10CF7000E82E8FE3F82E69EF78E0C8010E94634C39
:10CF80006DE172E1C8010E947F4B60E879E00E9488
:10CF9000684BBC0183E292E10E94EA4BC8010E9407
:10CFA000FF4B69EF78E0C8010E94634C6DE172E1CC
:10CFB000C8010E947F4B6AE979E00E94684BBC017E
:10CFC0008DE192E10E94EA4BC8010E94FF4B21E0F3
:10CFD0004EA95FA968AD79ADCE014F960E94044C71
:10CFE00021E04AAD5BAD6CAD7DADCE0149960E94AE
:10CFF000044C20EE3EE245E652E4C701B6010E9431
:10D000001DAFAB01BC0121E0C8010E94044CB80176
:10D01000CE0143960E945B4C69ED7BE0CE014396C6
:10D020000E94684BBE01675E7F4F0E947F4B69ED97
:10D030007BE00E94684BBE01615E7F4F0E947F4B88
:10D04000BC0187E192E10E94EA4BCE0143960E9427
:10D05000FF4BC8010E94FF4BCE0149960E94FF4B37
:10D06000CE014F960E94FF4B2DE2421621E0520660
:10D070006104710474F469A57AA58BA59CA525E0CB
:10D0800030E040E050E00E94EAAF672B682B692B4C
:10D09000C1F56DE172E1C8010E945B4C45E050E0D2
:10D0A0006FEF7FEFC8010E946490C8010E94FF4BA0
:10D0B00063EA79E0C8010E94634C45E050E061EF0B
:10D0C0007FEFC8010E94BF8FC8010E94FF4B6EEB2B
:10D0D00079E0C8010E94634CC8010E94F38DC80129
:10D0E0000E94FF4B67E172E1C8010E945B4C45E082
:10D0F00050E060E070E0C8010E94778DC8010E9496
:10D10000FF4B67E172E183E292E10E94164B3FE13F
:10D11000431651046104710434F4C9A4DAA4EBA4E5
:10D12000FCA4F7FC11C063E272E1C8010E945B4CF1
:10D13000C8010E942971C8010E94FF4B6EEB79E083
:10D1400083E292E10E94D54BB201C30177FE04C095
:10D1500069A97AA98BA99CA90E942F86A9C023E05E
:10D160004DA15EA16FA178A5CE0143960E94044C0B
:10D1700069EF78E0C8010E94634C6DE172E1C8017B
:10D180000E947F4B65EA79E00E94684BBE016D5EAC
:10D190007F4F0E947F4B6EE779E00E94684BBC0195
:10D1A0008DE192E10E94EA4BC8010E94FF4BCE0143
:10D1B00043960E94FF4B49855A856B857C8523E009
:10D1C000CE0149960E94044C4D815E816F81788525
:10D1D00023E0C8010E94044CB801CE0143960E948E
:10D1E0005B4C6AEA79E0CE0143960E94684BBE012F
:10D1F000675E7F4F0E947F4B6EE779E00E94684B2D
:10D20000BC0187E192E10E94EA4BCE0143960E9465
:10D21000FF4BC8010E94FF4BCE0149960E94FF4B75
:10D220002DE2421621E052066104710474F469A5EE
:10D230007AA58BA59CA525E030E040E050E00E9457
:10D24000EAAF672B682B692BF1F46DE172E1C8013D
:10D250000E945B4C4AE050E06FEF7FEFC8010E94F4
:10D260006490C8010E94FF4B67E172E1C8010E940F
:10D270005B4C4AE050E060E070E0C8010E94778DAE
:10D28000C8010E94FF4B63E272E1C8010E945B4C3F
:10D29000C801DFD7C8010E94FF4B6EEB79E083E243
:10D2A00092E10E94D54BC301B2010E942F861DAAB4
:10D2B0000E948B876B017C0122962CAD3DAD4EAD5B
:10D2C0005FAD2297C21AD30AE40AF50AC9A6DAA604
:10D2D000EBA6FCA6C7CC6DE172E1CE010D960E94D3
:10D2E0005B4C4AE050E06FEF7FEFCE010D960E945D
:10D2F000BF8FCE010D960E94FF4BCDA8CC20B1F17F
:10D3000063EA79E0CE010D960E94634C45E050E05F
:10D3100061EF7FEFCE010D960E94BF8FCE010D967B
:10D320000E94FF4B8091470C882391F060E371E1EC
:10D33000CE010D960E94534C45E050E060E070E055
:10D34000CE010D960E94BF8FCE010D960E94FF4B1D
:10D350006EEB79E0CE010D960E94634CCE010D96E6
:10D360000E94F38DCE010D960E94FF4B67E172E1A2
:10D37000CE010D960E945B4C4AE050E06FEF7FEFCC
:10D38000CE010D960E94778DCE010D960E94FF4B27
:10D39000CB5BDF4F0FB6F894DEBF0FBECDBFDF9182
:10D3A000CF911F910F91FF90EF90DF90CF90BF90A2
:10D3B000AF909F908F907F906F905F904F903F9035
:10D3C0002F9008956CEB79E00C94F34C0F931F931E
:10D3D000CF93DF93EC010E94C14C8C01CE01F2DFB0
:10D3E000800F911FDF91CF911F910F910895282FEA
:10D3F00030913A0D313208F04AC08091170D8111F9
:10D40000FCCF9091301342E04093170D2093160DFE
:10D410002FEF2093150D1092140D3093130DEAE1A8
:10D42000FDE0A3EFBCE020E0321721F041914D93E5
:10D430002F5FFACF1092F20C2091F20C990F922BE1
:10D440009093F20C9091F10C913061F41092F10CE8
:10D450009091F20C9093BB009091BC0093FDF8CF9B
:10D4600095EC01C095EE9093BC009091170D923011
:10D47000E1F39091150D9F3F79F08091150D803269
:10D4800041F08091150D803331F084E005C081E0DA
:10D4900003C082E001C083E01092190D10923A0D92
:10D4A0001092180D089581E0A2CF682F8FEA9FE0B7
:10D4B0000C94515691E09093180D80933013109274
:10D4C000190D10923A0D0895CF93C82F682F607FE1
:10D4D00084E293E10E947F5780E1C89FB00111244C
:10D4E00084E293E1CF910C947F57CF93DF93CDB734
:10D4F000DEB728970FB6F894DEBF0FBECDBF98E019
:10D50000EBE3F5E0DE01119601900D929A95E1F7BB
:10D5100090912D13961710F46FEF690FFE0131965D
:10D52000E60FF11DE60FF11D9081890F80682896A6
:10D530000FB6F894DEBF0FBECDBFDF91CF91C4CF41
:10D540000F931F93CF93DF93CDB7DEB7A2970FB69C
:10D55000F894DEBF0FBECDBF8C01CB01BA01F8013C
:10D560001182108213821282158214822AE0AE0187
:10D570004F5F5F4F0E948AAABE016F5F7F4FC80155
:10D580000E94D54BA2960FB6F894DEBF0FBECDBF5A
:10D59000DF91CF911F910F9108950F931F93CF9318
:10D5A000DF93EC010E94F34C8C01CE010BDF800F66
:10D5B000911FDF91CF911F910F910895CF92DF922C
:10D5C000EF92FF92CF93DF936B017C0197FF15C021
:10D5D0006DE282E19FE00E94BA4CEC01442755279E
:10D5E000BA014C195D096E097F092AE082E19FE0CA
:10D5F0000E94084DC80FD91F08C02AE0AB01BC012A
:10D6000082E19FE00E94084DEC0182E19FE0DADEBA
:10D610008C0F9D1FDF91CF91FF90EF90DF90CF9007
:10D6200008958F929F92AF92BF92CF92DF92EF9226
:10D63000FF920F931F93CF93DF936B017C01142F05
:10D640009B01AC010E9447B3882319F06FEB79E08E
:10D6500027C046015701E894B7F82FEF3FEF4FE797
:10D660005FE7C501B4010E9447B381110DC02FEFE0
:10D670003FEF4FE75FE7C501B4010E94B8AE18164F
:10D680001CF463EC79E00CC02FEF3FEF4FE75FE451
:10D69000C701B6010E94FDB1181694F467EC79E059
:10D6A00082E19FE0DF91CF911F910F91FF90EF906A
:10D6B000DF90CF90BF90AF909F908F900C94F34CE1
:10D6C0002FEF3FEF4FE75FECC701B6010E94B8AE06
:10D6D00087FDE4CF20E030E0A901C701B6010E9438
:10D6E000B8AE87FF0BC06DE282E19FE00E94BA4CAA
:10D6F000EC01F7FAF094F7F8F09402C0C0E0D0E043
:10D7000000E060E070E080E09FE3101741F020E06F
:10D7100030E040E251E40E940EB10F5FF6CFA70166
:10D7200096010E9448B06B017C010E94ACB14B0194
:10D730005C012AE0AB01BC0182E19FE00E94084D40
:10D74000C80FD91F1123C9F1C501B4010E94BCAE95
:10D750009B01AC01C701B6010E9447B06B017C017F
:10D760006EE282E19FE00E94BA4CC80FD91F20E010
:10D7700030E040E251E4C701B6010E941DAF4B0109
:10D780005C010E94ACB16B01E12CF12C2AE0B701E5
:10D79000A60182E19FE00E94084DC80FD91FC70172
:10D7A000B6010E94BCAE9B01AC01C501B4010E9450
:10D7B00047B06B017C011150D1F6CE01DF91CF91C2
:10D7C0001F910F91FF90EF90DF90CF90BF90AF909F
:10D7D0009F908F9008952F923F924F925F926F92F9
:10D7E0007F928F929F92AF92BF92CF92DF92EF92F1
:10D7F000FF920F931F93CF93DF93CDB7DEB7289798
:10D800000FB6F894DEBF0FBECDBFC090A10CD09074
:10D81000A20C4091A30C5091A40CC416D5062CF474
:10D820003C2D2D2D6A01432F522FE5EAFCE060E0EC
:10D8300070E0CB01019111910417150754F44A01CE
:10D84000550FAA08BB08680D791D8A1D9B1DA801EC
:10D8500015C0C016D10654F40D2C000CEE08FF08BC
:10D860006C0D7D1D8E1D9F1D680108C0012E000CD2
:10D87000220B330B600F711F821F931F2CE0E13FBF
:10D88000F207C1F60E94BEAE20E030E048E152E46B
:10D890000E940EB18B0188879F8381EAE82E8CE07D
:10D8A000F82E812C912C5401D7016D917D917D0131
:10D8B000072E000C880B990B0E94BEAE980148857C
:10D8C0005F810E9447B09B01AC010E941DAF9B018C
:10D8D000AC01C501B4010E9448B04B015C01E1EF0D
:10D8E000FCE0EE15FF0501F720E030E04CE152E4EA
:10D8F0000E940EB10E9406B36B017C0120E030E073
:10D9000040E85FE30E94FDB118160CF069C021EAFF
:10D910003CE03A832983212C312C412C512C3201BB
:10D92000A981BA818D919D91BA83A9839C01990F98
:10D93000440B550B2B833C834D835E83CA01B90195
:10D940000E94BEAE980148855F810E9447B04B019E
:10D950005C0120E030E0A9010E94FDB1181624F01E
:10D96000B7FAB094B7F8B094A7019601C501B40115
:10D970000E94B8AE87FF0BC08B819C81AD81BE81B8
:10D98000480E591E6A1E7B1E9FEF291A390AA1EF05
:10D99000BCE0E981FA81AE17BF0711F620E030E064
:10D9A00040EC5FE3C701B6010E941DAF6B017C0133
:10D9B000F5E02F1631040CF4AACFC301B2010E9486
:10D9C000BEAE6B017C01B101330C880B990B0E9438
:10D9D000BEAE9B01AC01C701B6010E940EB103C0EF
:10D9E000B80188859F816B017C01C701B60128962B
:10D9F0000FB6F894DEBF0FBECDBFDF91CF911F9160
:10DA00000F91FF90EF90DF90CF90BF90AF909F90DD
:10DA10008F907F906F905F904F903F902F900895E0
:10DA20004F925F926F927F928F929F92AF92BF922E
:10DA3000CF92DF92EF92FF921F93CF93DF93CDB7F8
:10DA4000DEB728970FB6F894DEBF0FBECDBF4B01EF
:10DA50005C0111E0612E712C9301220F331F220F04
:10DA6000331F3A832983F901ED57FD4FC080D180E0
:10DA7000E280F380A5019401C701B6010E94B8AE0F
:10DA800087FF02C01F5FE6CFA5019401C701B60161
:10DA90000E94B8AE49815A8145595D4F5E834D83DE
:10DAA000811106C0FA0160817181828193814DC02C
:10DAB000F1E06F1AF0EC7F0AC301880F991F880FFD
:10DAC000991FFC01ED57FD4F208131814281538127
:10DAD00029833A834B835C83FC01E559FD4F4080E9
:10DAE000518062807380A3019201ED81FE8160818B
:10DAF0007181828193810E9447B06D837E838F8381
:10DB0000988729813A814B815C81C501B4010E94CB
:10DB100047B09B01AC016D817E818F8198850E9409
:10DB20001DAF4B015C0129813A814B815C81C701AA
:10DB3000B6010E9447B09B01AC01C501B4010E942F
:10DB40000EB1A30192010E9448B028960FB6F89436
:10DB5000DEBF0FBECDBFDF91CF911F91FF90EF9041
:10DB6000DF90CF90BF90AF909F908F907F906F90FD
:10DB70005F904F9008950F931F930E948B8760933F
:10DB8000E00D7093E10D8093E20D9093E30D88ED2D
:10DB90009DE00E94974797FF1FC00E948B870091CE
:10DBA000E00D1091E10D2091E20D3091E30DDC01CB
:10DBB000CB01801B910BA20BB30B0091DC0D1091DC
:10DBC000DD0D2091DE0D3091DF0D80179107A2074A
:10DBD000B307E8F28FEF9FEF1F910F910895CF9257
:10DBE000DF92EF92FF92CF93DF93EC016A017B010A
:10DBF000E889F98982E080834115514E61057105FC
:10DC0000B1F060E079E08DE390E0A70196010E9419
:10DC100016B0DA01C9010197A109B109B695A79516
:10DC2000979587959C01211580E13807A8F0E88930
:10DC3000F989108260E874E88EE190E0A70196010E
:10DC40000E9416B0DA01C9010197A109B109B69580
:10DC5000A795979587959C01EC85FD853083EE858A
:10DC6000FF852083188EEC89FD8986E08083EA8910
:10DC7000FB89808180618083EA89FB89808188605B
:10DC80008083EA89FB89808180688083EA89FB89B7
:10DC900080818F7D8083DF91CF91FF90EF90DF9027
:10DCA000CF9008950F931F93CF93DF931F921F92EE
:10DCB000CDB7DEB70FE91CE0F80160818EED93E08F
:10DCC0009A838983CE0101960E941B3FF8016181EE
:10DCD0008FED93E09A838983CE0101960E941B3FCA
:10DCE000C8010F900F90DF91CF911F910F91089570
:10DCF000EF92FF920F931F93CF93DF931F921F9288
:10DD0000CDB7DEB70DE111E18D5191417C01C70125
:10DD1000800F911FF80161918F019A838983CE0151
:10DD200001960E941B3FF1E107321F0781F78DE149
:10DD300091E10F900F90DF91CF911F910F91FF9084
:10DD4000EF900895EF92FF920F931F93CF93DF937D
:10DD50001F921F92CDB7DEB70EE810E18E589041AA
:10DD60007C01C701800F911FF80161918F019A8397
:10DD70008983CE0101960E941B3FF1E104311F0708
:10DD800081F78EE890E10F900F90DF91CF911F9176
:10DD90000F91FF90EF900895EF92FF920F931F93D2
:10DDA000CF93DF931F921F92CDB7DEB70DE111E144
:10DDB0008D5191417C01C701800F911FF801619144
:10DDC0008F019A838983CE0101960E941B3FF2E165
:10DDD00007311F0781F78DE191E10F900F90DF91DF
:10DDE000CF911F910F91FF90EF9008958F929F9286
:10DDF000AF92BF92CF92DF92EF92FF920F931F9359
:10DE0000CF93DF938C01862F0B30110509F06FC083
:10DE100090918A12992309F0F89462E10E94BE5011
:10DE200020918A12222309F07894009709F072C099
:10DE3000E0908512F09086126F2D70E080E090E007
:10DE40000E94BEAE2DEC3CEC4CEC5DE30E941DAF9D
:10DE50004B015C016E2D70E080E090E00E94BEAE50
:10DE60009B01AC01C501B4010E9448B060937D12D2
:10DE700070937E1280937F1290938012C0918712CC
:10DE8000D09188126C2F6F7770E080E090E00E9454
:10DE9000BEAE4B015C016D2F70E080E090E00E940F
:10DEA000BEAE2DEC3CEC4CEC5DE30E941DAF9B0143
:10DEB000AC01C501B4010E9448B0C7FD09C0609320
:10DEC00081127093821280938312909384120BC0FC
:10DED000DC01CB01B0588093811290938212A09301
:10DEE0008312B0938412FE0CCF0DCD0F71C006319A
:10DEF000110509F0B4C090918A12992309F0F894A1
:10DF000061E00E94BE5020918A12222309F0789489
:10DF10000097A9F040E050EC69E774EC40937D1263
:10DF200050937E1260937F127093801240938112FF
:10DF300050938212609383127093841295C0F09074
:10DF40008612D09185126091851270918612762783
:10DF50006727762780E090E00E94BCAE2DEC3CEC79
:10DF60004CEC5DE30E941DAF60937D1270937E12B6
:10DF700080937F1290938012E0908812C091871254
:10DF80008C2F8F776E2D70E0782B80E090E00E94D0
:10DF9000BCAE2DEC3CEC4CEC5DE30E941DAFC7FD2C
:10DFA00009C06093811270938212809383129093C0
:10DFB00084120BC0DC01CB01B05880938112909386
:10DFC0008212A0938312B0938412DF0DED0ECE0D5A
:10DFD00080918912C81346C0C0907D12D0907E12E5
:10DFE000E0907F12F090801220E030E048EC52E4A4
:10DFF000C701B6010E94FDB118161CF0C0E0D0E0C8
:10E0000002C0CBEFDFEF20E030E0A901C701B6018D
:10E010000E94B8AE87FF02C0CAEFDFEFC090811246
:10E02000D0908212E0908312F090841220E030E0D1
:10E0300048EC52ECC701B6010E94B8AE87FF02C09F
:10E04000C9EFDFEF20E030E040EF52E4C701B60156
:10E050000E94FDB11816ACF4C8EFDFEF12C0CFEF8D
:10E06000DFEF0FC08FEF9FEF8F3FFFEF9F0709F4A8
:10E07000D3C0009709F4B0CF029609F4D9C0CCEF11
:10E08000DFEF0C30110509F0D6C08CE513DA80E023
:10E0900090E00BDA08DA65E08CE50E94B450C82FF6
:10E0A000D0E02097A1F0C530D105A4F001E313E141
:10E0B0008FEA9FE00E940956F80180870F5F1F4F8B
:10E0C000C801815393418C179D0794F306C0CEEF8E
:10E0D000DFEFB1C0CDEFDFEFAEC0C09139130091DB
:10E0E0003A13602F70E080E090E00E94BEAE2DEC0D
:10E0F0003CEC4CEC5DE30E941DAF6B017C016C2F8E
:10E1000070E080E090E00E94BEAE9B01AC01C701D0
:10E11000B6010E9448B0609331137093321380931C
:10E12000331390933413D0913B1310913C136D2F04
:10E130006F7770E080E090E00E94BEAE6B017C01E2
:10E14000612F70E080E090E00E94BEAE2DEC3CECD0
:10E150004CEC5DE30E941DAF9B01AC01C701B60111
:10E160000E9448B0D7FF5BC0DC01CB01B058809360
:10E17000351390933613A0933713B09338138C2F25
:10E18000800FC82FCD0FC10F80913D13C81344C01D
:10E19000C0903113D0903213E0903313F0903413C9
:10E1A00020E030E048EC52E4C701B6010E94FDB126
:10E1B00018161CF0C0E0D0E002C0CBEFDFEF20E08B
:10E1C00030E040EA50E4C701B6010E94B8AE87FFD4
:10E1D00002C0CAEFDFEFC0903513D0903613E09045
:10E1E0003713F090381320E030E040EF51ECC701D6
:10E1F000B6010E94B8AE87FF02C0C9EFDFEF20E092
:10E2000030E040EF52E4C701B6010E94FDB118169C
:10E2100094F4C8EFDFEF0FC0CFEFDFEF0CC06093D7
:10E220003513709336138093371390933813A7CF19
:10E23000CEEFDFEF26CFCE01DF91CF911F910F916F
:10E24000FF90EF90DF90CF90BF90AF909F908F9016
:10E250000895CF93DF93FC0124813581232B89F02E
:10E26000EC01BC018BE39DE0B1D86EE170E080E091
:10E2700090E00E942F86BE0182E19FE0DF91CF9166
:10E28000A5C8DF91CF910895CF92DF92EF92FF92D0
:10E29000CF93C091BD10C4300CF5C1300CF04BC011
:10E2A000C11176C091D7BC01990F880B990B0E94C0
:10E2B000BEAE20E030E040EA50E40E941DAF20E016
:10E2C00030EC4FE754E40E940EB12091BE10309123
:10E2D000BF104091C0105091C11057C0C43009F018
:10E2E00057C072D7BC01990F880B990B0E94BEAE24
:10E2F00020E030E040EA50E40E941DAF20E030EC26
:10E300004FE754E40E940EB120E030E040EA50E4D0
:10E310000E940EB120E030E040E851E40E941DAFC1
:10E3200020E030E040E850E40E9448B020E030E0D7
:10E330004AE754E42AC048D7BC01990F880B990BCF
:10E340000E94BEAE2AE137E64CE950E40E941DAFC0
:10E350002091BE103091BF104091C0105091C1105B
:10E360000E9447B06B017C01EC2FEE0FFF0BE955CB
:10E37000FA4F60817181072E000C880B990B0E9467
:10E38000BEAE9B01AC01C701B6010E940EB103C035
:10E3900060E070E0CB01CF91FF90EF90DF90CF90E5
:10E3A00008958F929F92AF92BF92CF92DF92EF9299
:10E3B000FF92CF93DF93CDB7DEB72C970FB6F894CB
:10E3C000DEBF0FBECDBF66E472E1CE0101960E94B2
:10E3D000534C4CE251E06FEF7FEFCE0101960E946B
:10E3E000778DCE0101960E94FF4B6091B70270912C
:10E3F000B8028091290290912A02F8DC84E1882EEB
:10E40000912CA12CB12CE12CF12C2FEFE21AF20A65
:10E41000C501B4010E942F866091B7027091B802C5
:10E420008091290290912A02E1DC23E0E216F104B6
:10E4300034F02AE0E216F10444F4892B49F084E137
:10E44000880E911CA11CB11CE0CF892B09F08BC157
:10E450008091290290912A028B309105C9F4809114
:10E46000811290918212A0918312B09184128093B4
:10E47000421390934313A0934413B0934513809198
:10E480007D1290917E12A0917F12B09180121DC0DA
:10E490008631910521F30C9701F580913513909108
:10E4A0003613A0913713B091381380934213909391
:10E4B0004313A0934413B09345138091311390916B
:10E4C0003213A0913313B091341380933E13909381
:10E4D0003F13A0934013B0934113409142135091C6
:10E4E0004313609144137091451321E0CE010796C8
:10E4F0000E94044C6CE07AE0CE0101960E94634CCD
:10E50000BE01695F7F4FCE0101960E947F4BBC0127
:10E5100083E292E10E94EA4BCE0101960E94FF4BFA
:10E52000CE0107960E94FF4B40913E1350913F133E
:10E53000609140137091411321E0CE0107960E9433
:10E54000044C62E476E0CE0101960E94634CBE0169
:10E55000695F7F4FCE0101960E947F4BBC0183E231
:10E5600092E10E94164BCE0101960E94FF4BCE0114
:10E5700007960E94FF4B64E076E083E292E10E94FE
:10E58000084B6EEB79E0CE0101960E94634C44E1AA
:10E5900050E060E070E0CE0101960E94BF8FCE0196
:10E5A00001960E94FF4BC0904213D0904313E0901D
:10E5B0004413F090451320E030E0A901C701B601F3
:10E5C0000E94FDB120E030E040E05FE387FD05C040
:10E5D000C701B6010E9448B004C0C701B6010E943D
:10E5E00047B00E94A7B1AB01BC01CE0101960E94C9
:10E5F000A06ABE016F5F7F4F8DE192E10E941C4BCC
:10E60000CE0101960E94FF4B60E087E00E94756A90
:10E610006DE172E184E293E10E94C14C6FED84E20E
:10E6200093E10E94BA4C68E476E084E293E10E94B0
:10E630009A4D60913E1370913F13809140139091D9
:10E6400041130E94A7B14AE050E084E293E10E94A6
:10E65000504D64E076E084E293E10E949A4D64E6D6
:10E6600070E080E090E00E942F86C0904213D0902E
:10E670004313E0904413F090451320E030E040EF66
:10E6800051E4C701B6010E94FDB187FD03C067E3F5
:10E6900072E154C020E030E040ED51E4C701B60122
:10E6A0000E94FDB187FD1FC067E272E1CE010196B5
:10E6B0000E94534C4AE050E06FEF7FEFCE0101968D
:10E6C0000E94778DCE0101960E94FF4B80914702F8
:10E6D000882331F06CED75E080E090E00E942F8699
:10E6E00067E172E12BC020E030E040EB51E4C7016C
:10E6F000B6010E94FDB187FD03C069E072E11EC052
:10E700006AEF71E1CE0101960E94534C4AE050E05D
:10E710006FEF7FEFCE0101960E94778DCE010196BB
:10E720000E94FF4B80914702882331F06CED75E029
:10E7300080E090E00E942F866CEE71E1CE010196A0
:10E740000E94534C4AE050E06FEF7FEFCE010196FC
:10E750000E94778DCE0101960E94FF4B62E370E02C
:10E7600080E090E0DCC00E94E93E6EE170E080E075
:10E7700090E00E942F860E949E976B017C0164E6C8
:10E7800070E080E090E00E942F866CE07AE083E207
:10E7900092E10E94D54B21E0B701A601CE0101967E
:10E7A0000E94044CBE016F5F7F4F83E292E10E94A2
:10E7B000164BCE0101960E94FF4B63E272E1CE013F
:10E7C00001960E945B4C4AE050E060E070E0CE01B0
:10E7D00001960E94BF8FCE0101960E94FF4B80914F
:10E7E0002E05882379F080912D05882359F06FED4F
:10E7F00084E293E10E94BA4C66E779E084E293E117
:10E800000E949A4D65E779E083E292E10E94084B0D
:10E81000C0924213D0924313E0924413F0924513F6
:10E8200020E030E040EF51E4C701B6010E94FDB1A5
:10E8300087FD03C06CED71E154C020E030E040ED95
:10E8400051E4C701B6010E94FDB187FD1FC06CEC09
:10E8500071E1CE0101960E94534C4AE050E06FEF07
:10E860007FEFCE0101960E94778DCE0101960E9426
:10E87000FF4B80914702882331F06CED75E080E01A
:10E8800090E00E942F866CEB71E12BC020E030E01D
:10E8900040EB51E4C701B6010E94FDB187FD03C002
:10E8A0006EEA71E11EC06FE971E1CE0101960E942E
:10E8B000534C4AE050E06FEF7FEFCE0101960E948B
:10E8C000778DCE0101960E94FF4B809147028823ED
:10E8D00031F06CED75E080E090E00E942F8661E9F8
:10E8E00071E1CE0101960E94534C4AE050E06FEF77
:10E8F0007FEFCE0101960E94778DCE0101960E9496
:10E90000FF4B6CE271E080E090E00E942F868091E6
:10E910004702882331F068EE73E080E090E00E94C7
:10E920002F862C960FB6F894DEBF0FBECDBFDF91B9
:10E93000CF91FF90EF90DF90CF90BF90AF909F90DE
:10E940008F900895DF92EF92FF920F931F93CF93D2
:10E95000DF93CDB7DEB762970FB6F894DEBF0FBE78
:10E96000CDBF8C01109246136EEB79E0CE010D966F
:10E970000E94634CFF24F39482E19FE00E94B94718
:10E980002091461318161906DCF5211139C082E1D1
:10E990009FE00E9497478A3041F08D3031F0682F18
:10E9A000CE010D960E94F54A24C089899A89892B47
:10E9B00001F1F09246136BEC79E0CE0101960E94D2
:10E9C000634CBE01635F7F4FCE0101960E947F4B77
:10E9D000BC01CE0107960E945B4CCE0107960E94B7
:10E9E000938FCE0107960E94FF4BCE0101960E94A5
:10E9F000FF4B6AE070E080E090E00E942F86BCCF81
:10EA0000211185C0E12CF12CDD24D3948BE39DE012
:10EA10000E94B9471816190614F58BE39DE00E9471
:10EA200097478A3079F08D3069F0909146139111B3
:10EA300009C0682FCE010D960E94F54A8FEFE81AA3
:10EA4000F80A06C089899A89892B11F0D092461359
:10EA500065E070E080E090E00E942F86D7CF64E10F
:10EA600070E080E090E00E942F86EF28D1F1898944
:10EA70009A89892BB1F180919A13882361F161E120
:10EA800079E0CE0101960E94634CBE016F5F7F4F1B
:10EA9000CE010D960E941F85F82ECE0101960E9490
:10EAA000FF4BF11018C064ED79E082E19FE00E9415
:10EAB0009A4DBE01635F7F4FCE0101960E945B4C71
:10EAC000BE016F5F7F4F82E19FE00E94E669CE0149
:10EAD00001960E94FF4B64E170E080E090E00E94AC
:10EAE0002F8680914613811112C089899A89892BBA
:10EAF00071F464E670E080E090E00E942F860E944E
:10EB00008B876EEB79E0C8010E94634C51C0898904
:10EB10009A89019709F046C06BED75E0CE01079622
:10EB20000E94634CBE01695F7F4FCE010D960E942B
:10EB30001F85811116C06EE577E0CE0101960E9417
:10EB4000634CBE016F5F7F4FCE010D960E941F8503
:10EB5000FF24F3948111F12CCE0101960E94FF4B0A
:10EB600001C0F12CCE0107960E94FF4BFF20A1F0BF
:10EB700040E050E0BE01635F7F4FCE0101960E94EE
:10EB8000343FBE016F5F7F4F8FE292E10E941C4BCA
:10EB9000CE0101960E94FF4B64E170E080E090E0BE
:10EBA0000E942F86BE01635F7F4FC8010E944B4CBD
:10EBB000CE010D960E94FF4BC80162960FB6F894E5
:10EBC000DEBF0FBECDBFDF91CF911F910F91FF90A0
:10EBD000EF90DF900895DF92EF92FF920F931F93D3
:10EBE000CF93DF93CDB7DEB72C970FB6F894DEBF87
:10EBF0000FBECDBF8C01109246136EEB79E0CE01B3
:10EC000007960E94634CE12CF12CDD24D3948BE316
:10EC10009DE00E94B9471816190614F58091461315
:10EC200081111EC08BE39DE00E9497478A3059F006
:10EC30008D3049F0682FCE0107960E94F54A8FEF7C
:10EC4000E81AF80A06C08B859C85892B11F0D092B2
:10EC500046136FE070E080E090E00E942F86D7CFEF
:10EC600062E370E080E090E00E942F86EF2851F090
:10EC70008BE39DE00E94574864E670E080E090E0FE
:10EC80000E942F868091461381110AC08B859C8536
:10EC9000892B31F46EEB79E0C8010E94634C18C0F7
:10ECA00080919A13882371F0BE01695F7F4FCE0176
:10ECB00001960E945B4CCE010196CBDACE01019603
:10ECC0000E94FF4BBE01695F7F4FC8010E944B4C01
:10ECD000CE0107960E94FF4BC8012C960FB6F89400
:10ECE000DEBF0FBECDBFDF91CF911F910F91FF907F
:10ECF000EF90DF90089581E080932D0580912E059F
:10ED0000882341F088E080932F1360E084E293E150
:10ED10000C946C57089580912E0581110FC081E0ED
:10ED200080932E0580932D0580912A13982F94604F
:10ED300090932A138C600E94646A18C080912D05FC
:10ED40008823A1F010922F1360E084E293E10E94E7
:10ED50006C5710922D0580912A138B7F80932A1374
:10ED600088600E94646A10922E050895C4CF2F9285
:10ED70003F924F925F926F927F928F929F92AF924B
:10ED8000BF92CF92DF92EF92FF920F931F93CF9398
:10ED9000DF93CDB7DEB766970FB6F894DEBF0FBE30
:10EDA000CDBF1C0185E79EE00E94118E40E855E230
:10EDB00060E070E085E79EE00E94EF6D64E670E041
:10EDC00080E090E00E942F868CED95E0A0E0B0E01E
:10EDD0008093790E90937A0EA0937B0EB0937C0E65
:10EDE00064E670E080E090E00E942F868FEF8A87D3
:10EDF00081E08B8786E88C871D861E861F86188A91
:10EE0000198A89E78A8BC101880F991F9E8B8D8B88
:10EE1000C12CD12CE12CF12C412C512C320185E755
:10EE20009EE0E214F3046CF5ED89FE89CE16DF0650
:10EE300044F50E94884708974CF049E050E0BE0135
:10EE4000665F7F4F85E79EE00E945E4765E070E069
:10EE500080E090E00E942F8600E010E0812C912C51
:10EE6000540185E79EE00E94B947892B31F4F4E014
:10EE70008F169104A104B104ACF50230110594F58C
:10EE800035C00E94118EE114F10409F47101C3012F
:10EE9000B2010E94BEAE4B015C01B701FF0C880BB2
:10EEA000990B0E94BEAE9B01AC01C501B4010E944A
:10EEB0000EB166960FB6F894DEBF0FBECDBFDF91E0
:10EEC000CF911F910F91FF90EF90DF90CF90BF9067
:10EED000AF909F908F907F906F905F904F903F90FA
:10EEE0002F9008958FEFC81AD80A99CF85E79EE032
:10EEF0000E94B947892B69F085E79EE00E949747F9
:10EF0000E1E0F0E0EC0FFD1FE00FF11F80830F5FE9
:10EF10001F4F65E070E080E090E00E942F86023095
:10EF2000110569F599818A85981329C09A818C8584
:10EF3000981325C0CE0103969C8B8B8B85E79EE0B2
:10EF40000E94B947892B31F494E089169104A104F9
:10EF5000B1043CF509301105C1F48B8190E0982F84
:10EF600088272C81820F911D092E000CAA0BBB0B48
:10EF7000480E591E6A1E7B1EEFEFEE1AFE0AFFEFC7
:10EF80008F1A9F0AAF0ABF0A6CCF85E79EE00E94E6
:10EF90009747EB89FC898193FC8BEB8B0F5F1F4FAD
:10EFA000CDCF0430110544F3D8CF2F923F924F922A
:10EFB0005F926F927F928F929F92AF92BF92CF9209
:10EFC000DF92EF92FF920F931F93CF93DF936C0129
:10EFD000CFEAD5E089E0882E82E0982E0EE810E195
:10EFE000EE24E394F12C22E1222E312C33E1432E46
:10EFF000512C40E1642E712C51E1A52EB12C809151
:10F000000702909108028E159F050CF4CAC021E0FA
:10F01000C216D10439F4F80182AD93ADF4019183A5
:10F0200080830AC0F2E0CF16D10431F4F40180816C
:10F030009181F80193AF82AFF401808191810097B3
:10F0400039F48A819B819093BA028093B90222C0DD
:10F050008130910539F48A819B819093B802809325
:10F06000B70218C08230910539F48A819B81909350
:10F07000B6028093B5020EC0039761F48A819B812A
:10F080009093B4028093B3026EEB79E087E792E14C
:10F090000E94D54BF401819191914F0184309105EB
:10F0A00039F42A813B81309362022093610212C0BD
:10F0B0008530910539F42A813B8130935A0220939F
:10F0C000590208C086309105C9F00EC08A309105FA
:10F0D00009F448C08531910589F42A813B81309338
:10F0E0005E0220935D023EC08730910579F72A8148
:10F0F0003B813093600220935F020AC08631910504
:10F1000039F42A813B8130935C0220935B022AC050
:10F110008731910539F52A813B812830310549F441
:10F120007092030260920202B0920102A092000269
:10F1300019C02730310549F43092030220920202AF
:10F1400050920102409200020DC02630310551F468
:10F1500021E030E03093030220930202109201027A
:10F16000109200029C012B5031092A30310590F495
:10F170002A813B813093B4022093B30239E1389F56
:10F18000B001399F700D112465547D4F87E792E1DE
:10F190000E94D54B8FEFE81AF80A22960E5F1F4F98
:10F1A0002ECFDF91CF911F910F91FF90EF90DF90C5
:10F1B000CF90BF90AF909F908F907F906F905F9017
:10F1C0004F903F902F9008957F928F929F92AF9291
:10F1D000BF92CF92DF92EF92FF920F931F93CF9344
:10F1E000DF93782E8AE0A82EB12CEE24EA9493E0E7
:10F1F000F92E88248A9423E0922E00E010E0C12C9E
:10F20000D12CC0E0D0E0872D0E94E585C816D90634
:10F2100028F00817190718F48C0101C06C01881533
:10F22000990528F08E159F0518F47C0101C04C014A
:10F23000C80FD91F65E070E080E090E00E942F8643
:10F2400081E0A81AB108F9F60C0D1D1DCE01801B36
:10F25000910B8E199F098819990966E070E00E9448
:10F260006FB3CB01DF91CF911F910F91FF90EF9082
:10F27000DF90CF90BF90AF909F908F907F90089538
:10F280004F925F926F927F92AF92BF92CF92DF9236
:10F29000FF920F931F93CF93DF9300D000D0CDB791
:10F2A000DEB75C0185E79EE00E94118E40E052ECE3
:10F2B00061E070E085E79EE00E94EF6D8CED95E0E7
:10F2C000A0E0B0E08093790E90937A0EA0937B0E2D
:10F2D000B0937C0E64E670E080E090E00E942F86A0
:10F2E000C12CD12CF12CCA14DB040CF051C065E008
:10F2F00070E080E090E00E942F8600E010E0412C5A
:10F30000512C3201F1100FC085E79EE00E94B947F1
:10F31000892B31F485E148165104610471041CF411
:10F320000330110554F08FEFC81AD80A64E670E074
:10F3300080E090E00E942F86D6CF85E79EE00E9475
:10F34000B947892B69F085E79EE00E949747E1E085
:10F35000F0E0EC0FFD1FE00FF11F80830F5F1F4FE8
:10F3600065E070E080E090E00E942F860230110599
:10F370004CF089818B3B31F4FF24F3948A818A3AE3
:10F3800009F0F12C8FEF481A580A680A780ABACFA8
:10F390008F2D26960FB6F894DEBF0FBECDBFDF913E
:10F3A000CF911F910F91FF90DF90CF90BF90AF90C2
:10F3B0007F906F905F904F9008951F93CF93DF934E
:10F3C000182FC1EADCE0812F0E94E585899399938B
:10F3D0006CE370E080E090E00E942F868CE0C13FFB
:10F3E000D80789F70E94EB6B20E030E040EA50E458
:10F3F0000E941DAF20E030E040E85AE30E941DAFBC
:10F40000DF91CF911F9108954F925F926F927F92FB
:10F410008F929F92AF92BF92CF92DF92EF92FF9224
:10F42000CF93DF93CDB7DEB768970FB6F894DEBF02
:10F430000FBECDBF6B017C010E948B87698B7A8BDD
:10F440008B8B9C8B88ED9DE00E94118E61E08091FA
:10F4500002020E94A98560E0809100020E94A985B5
:10F460000E949E970E94FF5B0E941C5C6D877E87B6
:10F470008F87988B0E940A864B015C016AE070E0DE
:10F4800080E090E00E942F866BED79E083E292E1CC
:10F490000E94D54B20E030E04AE754E4C701B601B2
:10F4A0000E941DAF6D8B7E8B8F8B988F412C512CC2
:10F4B0003201C12CD12C7601C701B6010E94BEAE2B
:10F4C0002D893E894F89588D0E94B8AE87FF85C12E
:10F4D0000E948B8729893A894B895C89621B730B4F
:10F4E000840B950B0E94BCAE20E030E04AE754E468
:10F4F0000E940EB1AB01BC0123E0CE0101960E9437
:10F50000044CBE016F5F7F4F8DE192E10E941C4B66
:10F51000CE0101960E94FF4B0E941C5C6B017C0196
:10F520000E940A869B01AC01281939094A095B0926
:10F5300049015A0131ED831637E09306A104B10465
:10F540000CF441C020E030E0A901C701B6010E94DF
:10F55000FDB118165CF426EA3BE944EC5BE3C70115
:10F56000B6010E94B8AE87FF0BC02DC026EA3BE96A
:10F5700044EC5BEBC701B6010E94FDB118161CF10B
:10F58000C501B40128EE33E040E050E00E94EAAF4C
:10F59000CA01B9010E94BEAE4B015C012D853E85BA
:10F5A0004F855889C701B6010E9447B020E030E07E
:10F5B0004AE754E40E941DAFA50194010E940EB1D8
:10F5C0004B015C0103C0812C912C54016DE172E16F
:10F5D000CE0101960E945B4C6BED75E0CE01019669
:10F5E0000E94684BBC018DE192E10E94EA4BCE0182
:10F5F00001960E94FF4B23E0B701A601CE010196C0
:10F600000E94044CBE016F5F7F4FCE0107960E949F
:10F610005B4C68EC78E0CE0107960E94684BBC0119
:10F6200087E192E10E94EA4BCE0107960E94FF4BD0
:10F63000CE0101960E94FF4B22E0B501A401CE014C
:10F6400007960E94044C69EF78E0CE0101960E9473
:10F65000634C6DE172E1CE0101960E947F4B69EF30
:10F6600079E00E94684B67E172E10E947F4B6EED8A
:10F6700075E00E94684BBE01695F7F4F0E947F4B1F
:10F6800069ED75E00E94684BBC0183E292E10E9443
:10F69000164BCE0101960E94FF4BCE0107960E94A9
:10F6A000FF4B20E030E0A901C501B4010E94FDB18B
:10F6B00087FD06C069ED7BE087E192E10E94084B7F
:10F6C00022E0B501A401CE0101960E94044CBE01C6
:10F6D0006F5F7F4FCE0107960E945B4C69ED75E02E
:10F6E000CE0107960E94684BBC0187E192E10E941F
:10F6F000164BCE0107960E94FF4BCE0101960E9449
:10F70000FF4B63E272E1CE0101960E945B4CCE0199
:10F7100001960E942971CE0101960E94FF4BC30100
:10F72000B20125E030E040E050E00E94EAAF672BF4
:10F73000682B692B21F56CE772E1CE0101960E94DE
:10F74000534C45E050E060E070E0CE0101960E942D
:10F75000BF8FCE0101960E94FF4B67E172E1CE019F
:10F7600001960E945B4C45E050E06FEF7FEFCE01C9
:10F7700001960E94778DCE0101960E94FF4B6EEBA1
:10F7800079E083E292E10E94D54B65E070E080E091
:10F7900090E00E942F860E948B876B017C01298953
:10F7A0003A894B895C89C21AD30AE40AF50A0E9495
:10F7B0001C5C6D877E878F87988B0E940A864B0121
:10F7C0005C016AE070E080E090E00E942F863FEFED
:10F7D000431A530A630A730A6FCE60E080910202F3
:10F7E0000E94A98568960FB6F894DEBF0FBECDBF04
:10F7F000DF91CF91FF90EF90DF90CF90BF90AF90CF
:10F800009F908F907F906F905F904F9008954F9250
:10F810005F926F927F92AF92BF92CF92DF92EF9200
:10F82000FF920F931F93CF93DF93CDB7DEB7EA9785
:10F830000FB6F894DEBF0FBECDBFF82E6EEB79E0A9
:10F84000CE01C5960E94634C8E010B5E1F4F6F2D3B
:10F85000C8010E94415718870F831D821E8219829A
:10F8600089E08A8381E08B838C831C8A1B8ACE018A
:10F8700001960E944E54CE0101960E94E253CE01A1
:10F8800001960E9413530E8110E00330110509F414
:10F890006EC162E772E1CE01C5960E94904B6EEB9D
:10F8A00079E083E292E10E94D54BBE016B5C7F4F11
:10F8B000CE0183960E945B4C4AE050E060E070E02D
:10F8C000CE0183960E94BF8FCE0183960E94FF4B8C
:10F8D00061E080E00E94756A6CE07AE0CE01C59636
:10F8E0000E94D54B83E1A82E8CE0B82ECC24C39483
:10F8F000D12CE12CF12CE016F1060CF0EEC06E2DAF
:10F90000CE0101960E94A452F501219131914191BD
:10F9100051915F010E9448B02B013C0120E030E092
:10F920004CEF52EC0E94B8AE87FF24C0B601CE0166
:10F9300089960E9489506AEA77E0CE0183960E94F8
:10F94000634CBE01675D7F4FCE0183960E947F4B63
:10F950006DEF79E00E94684BBC0183E292E10E9466
:10F96000164BCE0183960E94FF4BCE0189960E94D2
:10F97000FF4B48C022E0B301A201CE018F960E9446
:10F98000044CB601CE0189960E9489506AEA77E05C
:10F99000CE0183960E94634CBE01675D7F4FCE010E
:10F9A00083960E947F4B63ED7AE00E94684BBE0114
:10F9B000615D7F4F0E947F4BBC0187E192E10E9415
:10F9C000EA4BCE0183960E94FF4BCE0189960E949E
:10F9D000FF4BCE018F960E94FF4B67E172E1CE0193
:10F9E00083960E945B4C69ED7BE0CE0183960E947A
:10F9F000684BBC0183E292E10E94164BCE018396D4
:10FA00000E94FF4B0130110559F4E114F10409F093
:10FA10005DC063E272E1CE01C5960E94EA4B56C01A
:10FA20000230110511F522E0B301A201CE01839647
:10FA30000E94044CBE016D5D7F4FCE0189960E94ED
:10FA40005B4C69ED7BE0CE0189960E94684BBC015E
:10FA5000CE01C5960E94164BCE0189960E94FF4B9F
:10FA6000CE0183960E94FF4B31C00330110571F126
:10FA700067E172E1CE0183960E945B4C44E150E065
:10FA80006FEF7FEFCE0183960E94778DCE01839634
:10FA90000E94FF4B66E779E0CE0183960E94634C9B
:10FAA000CE0183960E94F38DCE0183960E94FF4B78
:10FAB00080912E05882351F080912D05882331F007
:10FAC00060ED77E080E090E00E942F86FFEFEF1A74
:10FAD000FF0A8FEFC81AD80A0ECFCE01C5960E9432
:10FAE000554A83E292E10E94554A01151105C9F475
:10FAF0006FE572E183E292E10E94904B64E572E16E
:10FB0000CE0183960E94534C4AE050E06FEF7FEFA6
:10FB1000CE0183960E94778DCE0183960E94FF4B83
:10FB2000EBC0043011050CF000C1BE016B5C7F4FCF
:10FB3000CE0183960E945B4C4AE050E06FEF7FEF6E
:10FB4000CE0183960E94778DCE0183960E94FF4B53
:10FB500066E779E0CE0183960E94634CCE018396DE
:10FB60000E94F38DCE0183960E94FF4BDEC069E0B8
:10FB70007AE0CE01C5960E94D54BBE016B5C7F4FEB
:10FB8000CE0183960E945B4C4AE050E060E070E05A
:10FB9000CE0183960E94BF8FCE0183960E94FF4BB9
:10FBA0006EEB79E083E292E10E94D54B63E272E171
:10FBB000CE01C5960E94EA4B00E010E0602FCE0116
:10FBC00001960E94A4526B017C0122E0AB01BC01B2
:10FBD000CE0183960115110551F40E94044CBE011B
:10FBE0006D5D7F4F84E293E10E94C14C18C00E947A
:10FBF000044CBE016D5D7F4FCE0189960E945B4C27
:10FC000069ED7BE0CE0189960E94684BBC01CE0174
:10FC1000C5960E94164BCE0189960E94FF4BCE01DD
:10FC200083960E94FF4B22E0B701A601CE01839686
:10FC30000E94044CBE016D5D7F4FCE0189960E94EB
:10FC40005B4C69ED7BE0CE0189960E94684BBC015C
:10FC500083E292E10E94164BCE0189960E94FF4BEF
:10FC6000CE0183960E94FF4B0F5F1F4F033011059B
:10FC700009F0A4CFCE01C5960E94554ABE016B5C27
:10FC80007F4FCE0183960E945B4C4AE050E06FEFBD
:10FC90007FEFCE0183960E94778DCE0183960E94DE
:10FCA000FF4B66E779E0CE0183960E94634CCE015C
:10FCB00083960E94F38DCE0183960E94FF4B83E2D0
:10FCC00092E10E94554A6FE07AE0CE0183960E944D
:10FCD000634C63E272E1CE0183960E947F4B69E13F
:10FCE0007AE00E94684BBC0183E292E10E94EA4BF9
:10FCF000CE0183960E94FF4BCE01C5960E94FF4B1A
:10FD0000EA960FB6F894DEBF0FBECDBFDF91CF915C
:10FD10001F910F91FF90EF90DF90CF90BF90AF9029
:10FD20007F906F905F904F90089569E17AE083E251
:10FD300092E10E94084BE0CFAF92BF92CF92DF9248
:10FD4000EF92FF920F931F93CF93DF93CDB7DEB760
:10FD5000A4970FB6F894DEBF0FBECDBF80914713B6
:10FD6000882319F01092471377C58091451290911E
:10FD70004612049708F03FC060EF77E0CE0101968D
:10FD80000E94634CBE016F5F7F4F8BE392E157D6B9
:10FD9000182FCE0101960E94FF4B112361F161E003
:10FDA00070E081E492E10E94B54A80330CF4845EF5
:10FDB0006AE270E0681B710987FD7395CE010196B8
:10FDC0000E948950BE016F5F7F4F81E492E10E94E3
:10FDD0001C4BCE0101960E94FF4B61E472E18FE261
:10FDE00092E10E94EA4B81E492E10E944A4ACB01EF
:10FDF0000E94D70A31C561E577E0CE0101960E94E5
:10FE0000634CBE016F5F7F4F8BE392E118D6182FD2
:10FE1000CE0101960E94FF4B112309F482C36CE2CC
:10FE20007AE0CE0101960E94634CCE0101960E94B9
:10FE30002971CE0101960E94FF4B68E37AE0CE0162
:10FE400007960E94634C68E173E1CE0107960E9419
:10FE50007F4BBC01CE0101960E945B4CCE01019606
:10FE60000E942971CE0101960E94FF4BCE01079698
:10FE70000E94FF4B609143027091440280914502C1
:10FE8000909146020E94BEAE20E030E048EC52E481
:10FE90000E940EB1AB01BC0122E0CE0107960E9488
:10FEA000044C6EE47AE0CE010D960E94634CBE01D4
:10FEB000695F7F4FCE010D960E947F4B62E578E02F
:10FEC0000E94684BBC01CE0101960E945B4CCE01A2
:10FED00001960E942971CE0101960E94FF4BCE012E
:10FEE0000D960E94FF4BCE0107960E94FF4B40915A
:10FEF0003F0250914002609141027091420224E021
:10FF0000CE0107960E94044C63E67AE0CE010D967E
:10FF10000E94634CBE01695F7F4FCE010D960E9427
:10FF20007F4BBC01CE0101960E945B4CCE01019635
:10FF30000E942971CE0101960E94FF4BCE010D96C1
:10FF40000E94FF4BCE0107960E94FF4B4091330267
:10FF500050913402609135027091360222E0CE0158
:10FF600007960E94044C40912B0250912C02609104
:10FF70002D0270912E0223E0CE010D960E94044CBA
:10FF800040913702509138026091390270913A02E3
:10FF900022E0CE0143960E94044C40912F025091E2
:10FFA0003002609131027091320223E0CE01499615
:10FFB0000E94044C60E87AE0CE014F960E94634CA8
:10FFC000BE01675E7F4FCE014F960E947F4B65E971
:10FFD0007AE00E94684BBE016D5E7F4F0E947F4BAE
:10FFE00068E97AE00E94684BBE01635F7F4F0E9420
:10FFF0007F4B65E97AE00E94684BBE01695F7F4FE5
:020000021000EC
:100000000E947F4B6EE97AE00E94684BBC01CE01F2
:1000100001960E945B4CCE0101960E942971CE018F
:1000200001960E94FF4BCE014F960E94FF4BCE01DE
:1000300049960E94FF4BCE0143960E94FF4BCE0192
:100040000D960E94FF4BCE0107960E94FF4B6BEA74
:1000500072E1CE0149960E94534CF090BD100F2DD5
:100060000F2C000C110B01151105A1F52091BE10EC
:100070003091BF104091C0105091C11060E070E00D
:1000800080EA90E40E940EB1AB01BC0122E0CE01F7
:1000900001960E94044C65E878E0CE0107960E9424
:1000A000634CBE016F5F7F4FCE0107960E947F4B6E
:1000B00064ED78E00E94684BBC01CE0149960E9435
:1000C000164BCE0107960E94FF4BCE0101960E946F
:1000D000FF4B09C00130110531F46DE972E1CE0129
:1000E00049960E94C64AC8010297029738F58F2D9B
:1000F0009AE08902B0011124CE0101960E94895034
:1001000063EA7AE0CE0107960E94634CBE016F5FFE
:100110007F4FCE0107960E947F4B6DEC78E00E94E6
:10012000684BBC01CE0149960E94164BCE01079642
:100130000E94FF4BCE0101960E94FF4B0430110537
:1001400019F46BE872E105C00530110534F063E87D
:1001500072E1CE0149960E94C64ABE01675E7F4F9A
:10016000CE0101960E945B4CCE0101960E9429713E
:10017000CE0101960E94FF4B6FEA7AE0CE014996CC
:100180000E94D54B8091BA106091BB107091BC1049
:1001900083300CF04FC3CE0101960E9489506AEA69
:1001A0007AE0CE0107960E94634CBE016F5F7F4FDD
:1001B000CE0107960E947F4B63EB7BE00E94684B69
:1001C000BC01CE0149960E94164BCE0107960E94B3
:1001D000FF4BCE0101960E94FF4BBE01675E7F4F31
:1001E000CE0101960E945B4CCE0101960E942971BE
:1001F000CE0101960E94FF4B4091C2105091C31056
:100200006091C4107091C51022E0CE0107960E9443
:10021000044C6FEB7AE0CE010D960E94634CBE0158
:10022000695F7F4FCE010D960E947F4B65ED7AE0AE
:100230000E94684BBC01CE0101960E945B4CCE012E
:1002400001960E942971CE0101960E94FF4BCE01BA
:100250000D960E94FF4BCE0107960E94FF4B4091E6
:10026000D8105091D9106091DA107091DB1022E013
:10027000CE0107960E94044C6CED7AE0CE010D96FB
:100280000E94634CBE01695F7F4FCE010D960E94B4
:100290007F4B6DEC75E00E94684BBC01CE0101966E
:1002A0000E945B4CCE0101960E942971CE010196FD
:1002B0000E94FF4BCE010D960E94FF4BCE01079688
:1002C0000E94FF4B89E0C82E82E0D82E01E010E0AA
:1002D00099E1F92E80910702909108028017910709
:1002E0000CF44DC0F601A190B1906F01B501CE01A3
:1002F00007960E948950B801CE010D960E94895040
:100300006FEE7AE0CE0143960E94634CBE01635FBC
:100310007F4FCE0143960E947F4B67EF7AE00E94A9
:10032000684BBE01695F7F4F0E947F4B6AEF7AE0A6
:100330000E94684BFA9CB001FB9C700D112465541F
:100340007D4F0E94684BBC01CE0101960E945B4C20
:10035000CE0101960E942971CE0101960E94FF4BA9
:10036000CE0143960E94FF4BCE010D960E94FF4B9B
:10037000CE0107960E94FF4B0F5F1F4FABCF8091BE
:10038000041190910511892B71F460E07BE0CE019E
:1003900001960E94634CCE0101960E942971CE0104
:1003A00001960E94FF4B80910411909105110197D5
:1003B00071F46FE07BE0CE0101960E94634CCE01A8
:1003C00001960E942971CE0101960E94FF4B8091F7
:1003D000041190910511029771F469E17BE0CE015F
:1003E00001960E94634CCE0101960E942971CE01B4
:1003F00001960E94FF4B6091290270912A02CE0162
:1004000007960E9489506BE27BE0CE010D960E9418
:10041000634CBE01695F7F4FCE010D960E947F4BFA
:10042000BC01CE0101960E945B4CCE0101960E9458
:100430002971CE0101960E94FF4BCE010D960E94BC
:10044000FF4BCE0107960E94FF4B40915002509106
:100450005102609152027091530222E0CE01079640
:100460000E94044C68E47BE0CE010D960E94634C30
:10047000BE01695F7F4FCE010D960E947F4B6BEDF1
:1004800075E00E94684BBC01CE0101960E945B4C56
:10049000CE0101960E942971CE0101960E94FF4B68
:1004A000CE010D960E94FF4BCE0107960E94FF4B96
:1004B0004091550250915602609157027091580236
:1004C00022E0CE0107960E94044C68E57BE0CE0155
:1004D0000D960E94634CBE01695F7F4FCE010D9661
:1004E0000E947F4B6BED75E00E94684BBC01CE0112
:1004F00001960E945B4CCE0101960E942971CE01AB
:1005000001960E94FF4BCE010D960E94FF4BCE013B
:1005100007960E94FF4B10925402CE0149960E940A
:10052000FF4B80914512909146128330910508F05F
:100530006FC18130910541F460E070E081E492E1A7
:100540000E94B54AE82E57C0029709F054C060EFE8
:1005500077E0CE0101960E94634CBE016F5F7F4F32
:100560008BE392E16CD2182FCE0101960E94FF4BD3
:10057000112309F440C061E070E081E492E10E943F
:10058000B54A682FCE0101960E94334CBE016F5FC1
:100590007F4F8FE292E10E941C4BCE0101960E9498
:1005A000FF4B60E070E081E492E10E94B54AE82EE2
:1005B00080919A138823F9F068E67BE0CE010196DA
:1005C0000E94634C61E472E1CE0101960E947F4B70
:1005D00069ED7BE00E94684BBC0182E19FE00E94D4
:1005E000C14CCE0101960E94FF4B6FE272E182E1A5
:1005F0009FE00E94E6698E2DEE0C990B0E94DAB501
:10060000892BB1F00E947B760E94E93E69ED7BE088
:10061000CE0101960E94634C4AE050E060E070E039
:10062000CE0101960E946490CE0101960E94FF4B7C
:1006300061E472E1CE0107960E945B4C60E070E0DD
:10064000CE0107960E94B54A823409F474C0D4F4EE
:10065000803309F490C07CF4833209F483C08A3279
:1006600009F0A9C061E87BE081E492E10E94D54BEA
:100670008FEF9FEF8EC0813309F48EC0813409F46F
:100680004FC099C0813609F44BC034F4833409F467
:100690005DC0843449F08FC0833609F457C00CF430
:1006A0004AC0843609F087C0809133129091341289
:1006B000892B09F49FC061E070E0CE0107960E948B
:1006C000B54A182F80919A13882361F06EE67BE07B
:1006D00082E19FE00E949A4D6FE272E182E19FE029
:1006E0000E94E66910330CF4145E6AE270E0611B4C
:1006F000710917FD7395CE0101960E948950BE01C4
:100700006F5F7F4F8FE292E10E941C4BCE010196FA
:100710000E94FF4B8FE292E10E944A4ACB0139C00E
:1007200065E77BE081E492E10E94D54B80910B0C60
:1007300090910C0C2EC068E77BE081E492E10E946E
:10074000D54B1092470C8CEF9FEF23C06BE77BE0FB
:1007500081E492E10E94D54B81E08093470C8DEFBC
:100760009FEF17C06EE77BE081E492E10E94D54BDA
:100770008EEF9FEF0EC068E579E08FE292E10E9474
:10078000D54B68E579E081E492E10E94D54B80E0A9
:1007900090E00E94D70A2EC062E87BE08FE292E1EF
:1007A0000E94D54B62E87BE081E492E10E94D54B48
:1007B00081E090E0EECFBE01695F7F4F8FE292E172
:1007C0000E94EA4B60E070E08FE292E10E94B54A3D
:1007D000082E000C990BC0970A9738F48FE292E12B
:1007E0000E944A4ACB010E94D70A64E670E080E08A
:1007F00090E035D2CE0107960E94FF4B8CD36093D8
:100800003D0C70933E0C80933F0C9093400C02C0C3
:100810000E94A72480D360933D0C70933E0C80937C
:100820003F0C9093400C6EEB79E081E492E10E94E2
:10083000D54B12C0CE0101960E94895064E87BE03E
:10084000CE0107960E94634CBE016F5F7F4FCE01C1
:1008500007960E947F4BB4CCA4960FB6F894DEBFE7
:100860000FBECDBFDF91CF911F910F91FF90EF9001
:10087000DF90CF90BF90AF90089590E0FC0131974A
:10088000E231F10508F04EC08827E855FF4F8F4F41
:100890000C9496B3809180008F7703C08091800084
:1008A0008F7D80938000089580918000877FF9CFAD
:1008B00084B58F7702C084B58F7D84BD0895809103
:1008C000B0008F7703C08091B0008F7D8093B0001F
:1008D0000895809190008F7707C0809190008F7D60
:1008E00003C080919000877F80939000089580914D
:1008F000A0008F7707C08091A0008F7D03C08091FA
:10090000A000877F8093A0000895809120018F77B9
:1009100007C0809120018F7D03C080912001877FD7
:10092000809320010895CF93DF93FC0124813581CA
:10093000232B71F0FB01DC01CD91DC916081718191
:10094000CE010E9431B6009719F08C1B9D0B02C09E
:100950008FEF9FEFDF91CF9108950F931F93CF9368
:10096000DF93FC01C481D581209719F4FB0110822B
:1009700011C0415051094C175D0708F4EA018B0181
:10098000FC0160817181AE01C8010E9422B6C00FD6
:10099000D11F1882DF91CF911F910F910895AF92CF
:1009A000BF92CF92DF92EF92FF920F931F93CF935C
:1009B000DF93FC0124813581FB014481558189014C
:1009C000041B150B4115510551F12115310539F164
:1009D0002417350720F10217130718F08901015079
:1009E00011097B01FC01A080B180C501DFEFCFEFD1
:1009F0006501C00ED11EC816D906A0F0F7016081AE
:100A000071810E9431B6009769F09C012A193B0957
:100A10000217130710F0D22FC32F0196ECCF8FEFE0
:100A20009FEF02C08D2F9C2FDF91CF911F910F91CF
:100A3000FF90EF90DF90CF90BF90AF900895FB01B3
:100A400044815581FC01248135812417350778F0D4
:100A500080819181009759F0FB016081718161155E
:100A6000710529F00E9414B621E0892B09F020E0DD
:100A7000822F0895FC01A089B1898C91A689B7893C
:100A800082FD0FC09C91818D8F5F8F73228D8217A5
:100A900049F0218DDF01A20FB11D5D969C93818FDE
:100AA00008958C910895CF93DF93282F30E0F901BA
:100AB000EA56FC4E8491F901E05BFC4ED491F901B9
:100AC000E65FFC4EC491CC2389F08111D6DEEC2F79
:100AD000F0E0EE0FFF1FE051FD4EA591B491EC91B7
:100AE000ED2381E090E021F480E002C080E090E01E
:100AF000DF91CF9108951F93CF93DF93282F30E09C
:100B0000F901EA56FC4E8491F901E05BFC4ED49168
:100B1000F901E65FFC4EC491CC23B9F0162F811188
:100B2000ACDEEC2FF0E0EE0FFF1FEA52FD4EA59178
:100B3000B4919FB7F894111104C08C91D095D8232B
:100B400002C0EC91DE2BDC939FBFDF91CF911F9110
:100B50000895CF93DF9390E0FC01E05BFC4E24917D
:100B6000FC01E65FFC4E8491882361F190E0880FE0
:100B7000991FFC01E454FD4EC591D491FC01EA5249
:100B8000FD4EA591B491611109C09FB7F894888179
:100B9000209582238883EC912E230BC0623061F470
:100BA0009FB7F8948881322F309583238883EC9106
:100BB0002E2B2C939FBF06C08FB7F894E8812E2B65
:100BC00028838FBFDF91CF910895863308F0865335
:100BD00090917B00282F2870977F922B90937B0019
:100BE00020912C0590E4299F900111248770822B7D
:100BF00080937C0080917A00806480937A00809159
:100C00007A0086FDFCCF809178002091790090E0F9
:100C1000922B08953FB7F89480914C1390914D1307
:100C2000A0914E13B0914F1326B5A89B05C02F3F3E
:100C300019F00196A11DB11D3FBFBA2FA92F982F02
:100C40008827820F911DA11DB11DBC01CD0142E07D
:100C5000660F771F881F991F4A95D1F708958F92C5
:100C60009F92AF92BF92CF92DF92EF92FF926B0171
:100C70007C01D0DF4B015C01C114D104E104F1041B
:100C8000E9F0C8DFDC01CB0188199909AA09BB0981
:100C9000883E9340A105B10578F321E0C21AD1083E
:100CA000E108F10888EE880E83E0981EA11CB11CB3
:100CB000C114D104E104F10421F7DECFFF90EF90DD
:100CC000DF90CF90BF90AF909F908F900895FF924C
:100CD0000F931F93CF93DF93CDB7DEB72B970FB64C
:100CE000F894DEBF0FBECDBF85E79EE09AD740E8FF
:100CF00055E260E070E085E79EE00E94EF6D64E6FB
:100D000070E080E090E0ABDF8CED95E0A0E0B0E03B
:100D10008093790E90937A0EA0937B0EB0937C0E05
:100D200064E670E080E090E09ADF8FEF898381E0F5
:100D30008A8386E88B831C821D821E821F8218860E
:100D400089E7898785E79EE00E94574862E370E063
:100D500080E090E084DF85E79EE00E948847089766
:100D60004CF049E050E0BE016F5F7F4F85E79EE0A9
:100D70000E945E4762E370E080E090E070DF85E70C
:100D80009EE00E94B947892B01F185E79EE00E9411
:100D90008847089784F465E070E080E090E05FDFCA
:100DA00000E010E0F12C85E79EE00E94B947023098
:100DB0001105A4F50CC049E050E0BE016F5F7F4F04
:100DC00085E79EE00E945E47E6CFF12C27C085E7CD
:100DD0009EE00E94B947892B99F465E070E080E0BD
:100DE00090E03DDF02301105F1F69A858981981374
:100DF000DACF9B858B819813D6CFFF24F394D3CF82
:100E000085E79EE00E949747EAE0F0E0EC0FFD1FC7
:100E1000E00FF11F80830F5F1F4FDFCF62E370E0B1
:100E200080E090E01CDF85E79EE0FBD68F2D2B96BF
:100E30000FB6F894DEBF0FBECDBFDF91CF911F91EB
:100E40000F91FF900895CF93DF930E945750109217
:100E5000291380912D13823018F098E09093291374
:100E600090912E13992339F0813029F48091291320
:100E700084608093291362E370E080E090E0EFDE0D
:100E800060912F1384E293E10E946C5768EE73E047
:100E900080E090E0E4DE60E384E293E10E947F572B
:100EA000CBE4D6E4CE010197F1F760E384E293E16D
:100EB0000E947F572197F1F760E384E293E10E945B
:100EC0007F5783E592E00197F1F760E284E293E1D6
:100ED0000E947F578091291380620E94646A84E097
:100EE00080932A138CE00E94646A81E00E94646A05
:100EF000CBE3DFE1CE010197F1F782E080932B1382
:100F000086E00E94646A82E00E94646A2197F1F799
:100F1000DF91CF9108952FB7F894609148137091A5
:100F2000491380914A1390914B132FBF08952F922C
:100F30003F924F925F926F927F928F929F92AF9269
:100F4000BF92CF92DF92EF92FF920F931F93CF93B6
:100F5000DF93CDB7DEB766970FB6F894DEBF0FBE4E
:100F6000CDBF7C016D8B7E8B5C8B4B8B19016EEB47
:100F700079E00E94634C8EE1882E912C8E010F5FE8
:100F80001F4F2101032C000C66087708CD88DE88EE
:100F9000A12CB12CA214B3040CF07BC0B501CE017E
:100FA0000D960E948950BE01635F7F4FCE01079668
:100FB0000E945B4C66E177E0CE0107960E94684B89
:100FC0006B897C890E947F4BB6010E947F4BBC01DC
:100FD000C8010E945B4C40ED57E060E070E0C80142
:100FE00086D5C8010E94FF4BCE0107960E94FF4B99
:100FF000CE010D960E94FF4B44E150E061E070E0AD
:10100000C8010E94F7540E151F0521F0B801C70151
:101010000E941C4BC8010E94FF4BF70184819581FF
:10102000892BA9F160E070E0C7010E94B54A082E43
:10103000000C990BC0970A9740F4C7010E944A4AD6
:1010400064157505860597054CF066E779E0F701AC
:10105000808191810E9404B6892B59F481E0FFEFD1
:10106000AF1ABF0A96E0C90ED11C882309F492CFAB
:1010700015C06CED73E1C8010E94534C40ED57E080
:1010800060E070E0C80133D5C8010E94FF4B80E0EA
:10109000E6CFE1E08E1A910809F078CFC701669695
:1010A0000FB6F894DEBF0FBECDBFDF91CF911F9179
:1010B0000F91FF90EF90DF90CF90BF90AF909F90F7
:1010C0008F907F906F905F904F903F902F900895FA
:1010D000CF93DF93EC01483085E058076105710537
:1010E00009F441C108F08DC0493481E05807610519
:1010F000710509F43BC1E0F5443481E0580761050E
:10110000710509F424C1E8F4413481E05807610510
:10111000710509F413C138F440345140610571057B
:1011200009F409C135C1423481E0580761057105F0
:1011300009F407C1433451406105710509F404C144
:1011400027C1463481E058076105710509F405C1DE
:1011500008F400C1473481E058076105710509F4BE
:10116000FFC0483451406105710509F4FCC010C14D
:10117000423085E058076105710509F4E2C0E8F4E2
:10118000443781E058076105710509F4F5C038F46A
:10119000423751406105710509F4F1C0F9C04115AC
:1011A00085E058076105710509F4C5C04130554017
:1011B0006105710509F4C2C0EBC0453085E05807F0
:1011C0006105710509F4C6C070F4433085E0580725
:1011D0006105710509F4B8C04430554061057105D9
:1011E00009F4B5C0D5C0463085E0580761057105E2
:1011F00009F4B3C0473055406105710509F4B0C02A
:10120000C7C04D3B82E458078FEF6807710509F4AA
:10121000BCC008F045C04F3E80E158078FEF68071B
:10122000710509F49DC0E8F4423385E05807610573
:10123000710509F4A4C038F44930554061057105C1
:1012400009F494C0A5C0443385E0580761057105D1
:1012500009F492C04D3F52406F4F710509F48FC0A1
:1012600097C04D3D82E258078FEF6807710509F47A
:1012700083C038F4473E58416F4F710509F46AC086
:1012800087C04F3C80E358078FEF6807710509F46A
:101290005EC0473C58436F4F710509F464C078C085
:1012A000473988E658078FEF6807710509F446C08B
:1012B00000F54D3A82E558078FEF6807710509F48C
:1012C00061C030F4453B5A446F4F7105A1F160C0D5
:1012D000453A8AE558078FEF6807710509F446C05B
:1012E0004D3952466F4F710509F052C066E779E0FB
:1012F00051C0473588EA58078FEF68077105C9F173
:1013000068F445388AE758078FEF6807710529F1B7
:10131000473658496F4F7105A1F03AC04F3480EB02
:1013200058078FEF6807710579F04D33524C6F4FB6
:10133000710529F12DC068E579E02CC062E87BE0F9
:1013400029C06FE77BE026C06CE77BE023C069E73C
:101350007BE020C066E77BE01DC06DE87BE01AC043
:101360006FE87BE017C061E97BE014C063E97BE0D4
:1013700011C060EF77E00EC060E476E00BC06DEC6A
:1013800078E008C061E179E005C065E97BE002C072
:101390006EEB79E0CE010E94634CCE01DF91CF91DC
:1013A00008954F925F926F927F928F929F92AF9229
:1013B000BF92EF92FF920F931F93CF93DF93CDB71E
:1013C000DEB762970FB6F894DEBF0FBECDBF7C01CB
:1013D0005B0180E693E10E94F71D892B31F46EEBEF
:1013E00079E0C7010E94634C28C140916413509179
:1013F00065136091661370916713CE01079668DEDE
:1014000080919A13882359F167E97BE0CE01019618
:101410000E94634CBE01695F7F4FCE0101960E941E
:101420007F4B66E177E00E94684BBC0182E19FE060
:101430000E94C14CCE0101960E94FF4B4091641363
:1014400050916513609166137091671320E182E1FA
:101450009FE00E94084D82E19FE00E94E26960E007
:1014600070E0CE0107960E94B54A182F8A3211F01B
:101470001092471350DD60933D0C70933E0C8093A7
:101480003F0C9093400C6EEB79E0CE010D960E94DC
:10149000634C812F110F990BC0970A9708F05CC01D
:1014A000CE0107960E944A4A633071058105910575
:1014B0000CF094C001E010E082E0982E0A151B05A4
:1014C0000CF08CC06CE271E080E090E0C8DB9092A0
:1014D000BB0F1092BF0F412C512C320180E593E1DC
:1014E0000E94F71D892B41F48EE1481651046104D6
:1014F000710409F08CC01CC08EE1481651046104CF
:101500007104B1F0409154135091551360915613EA
:1015100070915713CE010196DBDDBE016F5F7F4FE7
:10152000CE010D960E941C4BCE0101960E94FF4BEE
:1015300089899A89892B39F0BE01635F7F4FCE017B
:1015400007960E94164B0F5F1F4F6EEB79E0CE019E
:101550000D960E94D54BB2CF6CE271E080E090E036
:101560007EDB82E08093BB0F1092BF0F812C912C09
:10157000540180E593E10E94F71D892B41F48EE12F
:1015800088169104A104B10409F04CC01CC08EE17E
:1015900088169104A104B104B1F040915413509104
:1015A00055136091561370915713CE01019690DD3B
:1015B000BE016F5F7F4FCE010D960E941C4BCE0186
:1015C00001960E94FF4B89899A89892B39F0BE01C7
:1015D000635F7F4FCE0107960E94164B64E670E072
:1015E00080E090E03CDB82E08093BB0F1092BF0F65
:1015F000BE01695F7F4FC7010E944B4CCE010D9623
:101600000E94FF4BCE0107960E94FF4B16C06EE171
:1016100070E080E090E023DB8FEF481A580A680AF8
:10162000780A5CCF6EE170E080E090E018DB8FEF2D
:10163000881A980AA80AB80A9CCFC70162960FB602
:10164000F894DEBF0FBECDBFDF91CF911F910F91F8
:10165000FF90EF90BF90AF909F908F907F906F9092
:101660005F904F900895AF92BF92CF92DF92EF922A
:10167000FF920F931F93CF93DF93CDB7DEB72C97D5
:101680000FB6F894DEBF0FBECDBF7C015B010E9498
:10169000FE97182F811106C06EEB79E0C7010E94FA
:1016A000634C99C08A3211F01092471334DC609376
:1016B0003D0C70933E0C80933F0C9093400C612F37
:1016C000CE0107960E94334C812F012E000C990BFE
:1016D000C0970A9750F5CE0107960E944A4A633098
:1016E0007105810591050CF04BC001E010E00A1571
:1016F0001B050CF045C062E370E080E090E0AFDADB
:101700000E94FE97C12CD12C811152C08FEFC81AB4
:10171000D80A85E1C816D10499F16EE170E080E045
:1017200090E09DDA0E94FE97EFCF612FCE010196E7
:101730000E94334CBE016F5F7F4FCE0107960E941F
:101740001C4BCE0101960E94FF4B62E370E080E0EB
:1017500090E085DA0E94FE9700E010E08823D9F03F
:10176000682FCE0101960E94334CBE016F5F7F4F00
:10177000CE0107960E94164BCE0101960E94FF4BA8
:10178000BE01695F7F4FC7010E944B4CCE01079697
:101790000E94FF4B20C00F5F1F4F0F31110581F3D7
:1017A0006EE170E080E090E05ADA0E94FE97D6CFBA
:1017B000682FCE0101960E94334CBE016F5F7F4FB0
:1017C000CE0107960E94164BCE0101960E94FF4B58
:1017D0000F5F1F4F8CCFC7012C960FB6F894DEBF5A
:1017E0000FBECDBFDF91CF911F910F91FF90EF9072
:1017F000DF90CF90BF90AF9008954F925F926F921D
:101800007F928F929F92AF92BF92CF92DF92EF9290
:10181000FF92CF93DF93CDB7DEB72C970FB6F89436
:10182000DEBF0FBECDBF0E94E93E0E94CC952B01CA
:101830003C010E949E974B015C01609143027091B4
:10184000440280914502909146020E94BEAE6B0117
:101850007C010E94CC950E94BEAEA70196010E9419
:101860000EB121E03EED42E45EE30E94B6B29B0180
:10187000AC0160E070E080E89FE30E9447B020E0A8
:101880003AE24DE257E40E941DAF6B017C01C301B7
:10189000B2010E94BEAE20E030E048EC52E40E946B
:1018A0000EB1AB01BC0122E0CE0101960E94044CB6
:1018B000BE016F5F7F4F87E192E10E941C4BCE011A
:1018C00001960E94FF4B62E578E087E192E10E9479
:1018D000084B67E172E18DE192E10E94EA4B6EE410
:1018E00078E0CE0101960E94634C67E172E1CE017F
:1018F00001960E947F4BBC0187E192E10E94EA4B76
:10190000CE0101960E94FF4B6CE07AE083E292E107
:101910000E94D54B21E0B501A401CE0101960E94A1
:10192000044CBE016F5F7F4F83E292E10E94164B31
:10193000CE0101960E94FF4B6CE97BE083E292E1CD
:101940000E94084B21E0B701A601CE0101960E943A
:10195000044CBE016F5F7F4FCE0107960E945B4C27
:1019600067EF75E0CE0107960E94684BBC0183E2E9
:1019700092E10E94164BCE0107960E94FF4BCE01CA
:1019800001960E94FF4B67E172E1CE0101960E9431
:101990005B4C69ED7BE0CE0101960E94684B63E2EF
:1019A00072E10E947F4BBC0183E292E10E94EA4B0C
:1019B000CE0101960E94FF4B21E0B501A401CE01AA
:1019C00001960E94044CBE016F5F7F4F89E292E155
:1019D0000E941C4BCE0101960E94FF4B69E272E10E
:1019E000CE0101960E945B4C4AE050E060E070E05E
:1019F000CE010196C4D2CE0101960E94FF4B65E054
:101A000070E080E090E02BD966E779E0CE010196A6
:101A10000E94634CCE010196E6D0CE0101960E9451
:101A2000FF4B6DE172E1CE0101960E945B4C4AE0F2
:101A300050E06FEF7FEFCE01019659D0CE010196B5
:101A40000E94FF4B20E0B701A601CE0101960E9443
:101A5000044CBE016F5F7F4FCE0107960E945B4C26
:101A600067EF75E0CE0107960E94684BBC0189E2E2
:101A700092E10E94EA4BCE0107960E94FF4BCE01F5
:101A800001960E94FF4B69E272E1CE0101960E942D
:101A90005B4C4AE050E064EF7FEFCE01019627D027
:101AA000CE0101960E94FF4B65E070E080E090E07F
:101AB000D6D88091470C882329F068E572E080E051
:101AC00090E0CDD82C960FB6F894DEBF0FBECDBFF8
:101AD000DF91CF91FF90EF90DF90CF90BF90AF90CC
:101AE0009F908F907F906F905F904F9008958F920E
:101AF0009F92AF92BF92EF92FF920F931F93CF935B
:101B0000DF9320912E05222309F462C020912D0538
:101B1000222309F45DC08A01EB017C0177FF18C024
:101B2000C095D09561E08C2F0E94756AB70184E260
:101B300093E10E94C14C6AEF73E184E293E10E9459
:101B4000CF4CF701848161E08C0F0E94756A31C02F
:101B5000E2D98090921390909313A0909413B09038
:101B6000951324E6820E911CA11CB11C86169706C3
:101B7000A806B90668F561E08C2F0E94756AB70166
:101B800084E293E10E94C14C69EE73E184E293E147
:101B90000E94CF4CF701848161E08C0F0E94756A2E
:101BA000BAD9609392137093931380939413909384
:101BB0009513B801110F880B990BDF91CF911F91ED
:101BC0000F91FF90EF90BF90AF909F908F9047C87C
:101BD000DF91CF911F910F91FF90EF90BF90AF9049
:101BE0009F908F900895CF93DF9320912E0522230D
:101BF000A9F020912D05222389F0EC016FED84E2FC
:101C000093E10E94BA4C8C819D81892B39F0BE01F1
